:020000040800F2
:10000000000001105D810308A12C0308357101086F
:100010006182030861820308618203080000000016
:10002000000000000000000000000000E9320308AA
:10003000E532030800000000E1320308A58801084A
:1000400061820308618203086182030861820308F8
:1000500061820308618203088D6B0108B96C010895
:100060007D6C0108416C0108056C010815CD000884
:1000700005CD0008F5CC0008E5CC0008D5CC00087B
:10008000C1CC0008ADCC000861820308618203087E
:10009000618203086182030861820308C96B010859
:1000A0006182030861820308618203086182030898
:1000B000057A0108F5790108E579010861820308EC
:1000C0006182030861820308618203086182030878
:1000D000618203087D61010861820308E160010813
:1000E000516B01086182030805330308618203082C
:1000F00061820308618203086182030899CC0008C9
:100100006182030861820308618203086182030837
:100110006182030861820308EDBB0108D1BB0108BD
:1001200085CC000871CC00085DCC000849CC0008E3
:1001300035CC0008618203086182030861820308EC
:10014000618203086182030861820308A52C030809
:1001500021CC00080DCC0008F9CB0008318901083A
:1001600061820308618203086182030861820308D7
:1001700061820308618203086182030861820308C7
:0801800061820308618203089B
:1001880002020300842100208021002000000000DA
:100198000000000027000400A0220020A82300205F
:1001A80000000000D405000816000800A024002064
:1001B800A824002000000000D80500080101040060
:1001C8003C250020BC330020000000000000000097
:1001D8000802090032330020C0330020000000006C
:1001E800DD5D010802000C003C330020CC33002008
:1001F8000000000000000000F70106002C3300207A
:10020800D833002000000000E00500080A020A00B8
:10021800CC250020E033002000000000E60500089F
:100228002C00100008380020F837002000000000DB
:10023800F1F701082B0024003C3800201838002072
:1002480000000000C1F7010829005000EC39002027
:10025800F83D00200000000000000000140002002B
:10026800E8390020483E002000000000F0050008A2
:100278001500700074400020444500200000000074
:10028800000000000300010070400020B445002079
:1002980000000000000000002A006000803F0020ED
:1002A800B845002000000000112B020809020100D7
:1002B800814600206053002000000000F20500087D
:1002C80003123300D7540020A4540020000000007B
:1002D800F405000825005A00F05300204A54002075
:1002E8000000000000000000F6110C00E45300209C
:1002F800D85300200000000028060008012008004C
:10030800505600209C5600200000000034060008CB
:100318001A00080038560020A456002000000000EB
:100328003C0600080002050044570020785A0020C7
:1003380000000000000000001E0004004C570020D0
:10034800805A0020000000004406000822000C002B
:10035800F4590020845A00200000000048060008D4
:100368001F000E00D85B0020F85B00200000000092
:100378005406000805020100C05B0020085C00204C
:10038800000000006206000803010600525B00201E
:100398000C5C002000000000640600080500060050
:1003A8007E5D0020485E0020000000006C0600080A
:1003B8000C002400465D0020505E00200000000074
:1003C80091B201080E20EA003E5C0020745E002015
:1003D800000000006954020813000400945D002026
:1003E800605F0020000000007406000812100C0076
:1003F8001C5C0020645F00200000000078060008F4
:1004080002010300175C0020705F0020000000005C
:10041800B9B201081B00F4007C5F00204062002094
:1004280000000000458A020826000E0044630020F0
:10043800346300200000000035CB020810000300E0
:10044800D0650020D4650020000000008406000864
:1004580028000C00C4650020D865002000000000BA
:100468008806000823001000B4650020E465002019
:10047800000000007513020819000500AC65002093
:10048800F46500200000000094060008F81101003F
:10049800A8650020FC650020000000009A060008FE
:1004A80000010400A4650020006600200000000090
:1004B8009C0600082F0011009065002004660020AB
:1004C80000000000A0060008F9010400C06B00202D
:1004D800C46B002000000000CD5D010818102C003E
:1004E800906B0020C86B0020000000002501020866
:1004F800FB010100686B0020F46B00200000000085
:1005080005700108FC010900346A0020F86B00201E
:1005180000000000C96F01080A101200086A0020D4
:10052800046C002000000000B20600080600160057
:10053800D8660020186C00200000000089540208CA
:100548000B201000846E0020BC6E0020000000000C
:10055800C4060008FD011E003879002094790020A7
:10056800000000005D5D0108FE01080024790020FC
:10057800B4790020000000004D70010804008000DC
:10058800CC9400205C9600200000000000000000D1
:10059800340010008C9D0020609E002000000000A8
:1005A800392B02080D002400689D0020709E002051
:1005B800000000002D9B0108FA0102006C97002042
:0C05C800949E0020000000005970010803
:1005D40020030000C4090000190128281E0100009E
:1005E400000000004A01B400D6010000030013001B
:1005F40000000000000000000000000000000000F7
:1006040000000000000000000000000000000000E6
:1006140000000000000000000000000000000000D6
:1006240000000100000000000000000000000000C5
:10063400E8036400040A00017E05EA05B4053200FB
:1006440000000100C800141E010064002C012800F1
:100654000000000000000100000000050000000090
:10066400040101000000000020000300010000005C
:100674000800000000000001000550494B34000050
:10068400000105000000000100000000000000005F
:100694000000280100000400900100000000000098
:1006A4000000000000000000000000000000003016
:1006B4000100005A0000000090012C01C8006400F1
:1006C4002B21231E64010200000001000A012900FD
:1006D4000101000028DB0308E8060408000000000C
:1006E4000000000038DB030840DB030800000000C2
:1006F4000120000044DB03084CDB03080000000079
:100704000140000050DB03082CF203080000000045
:10071400012000005CDB030868DB03080000000024
:10072400040000006CDB030878DB03080000000011
:10073400040000007CDB03089405040800000000AA
:100744000100000002010000500100000700000049
:100754000200000000000000000000000102030489
:10076400060708090000803F0000803FFF000000EA
:100774003D2B0308F52A0308452A0308000000005E
:1007840035270308B9280308392903082128030851
:100794000000000000000000292703080D270308BB
:1007A4000927030805270308F9260308F526030883
:1007B40001270308FD2603081D2703081127030842
:1007C400F92703080D280308E5270308D1270308A0
:1007D400BD27030828B6030805080400000000002C
:1007E400C8C9030864C9030814B60308000000005C
:1007F40054B6030805080A0000000000C8C903082D
:1008040064C90308E0D0030800000000FFFFFFFFF5
:1008140001010000F51802080000000000000000BB
:1008240000010101010000000101010028FC03088E
:100834000E000000994202080000000000000000C1
:10084400DC020020ECFB03080000000000000000B4
:100854000000000000000000E8060408000000009A
:1008640000000000780700200400000078FB030863
:100874000C00000089BB020854070020000000009F
:100884009CFA03080C00000059BB0208480700202A
:10089400000000000CFC0308080000000000000039
:1008A4003C07002004000000FCFB03080C000000CF
:1008B400D1480208300700200000000088FA03082D
:1008C40003000000B1BD020818070020000000006A
:1008D40004FC030803000000B1BD02080007002067
:1008E400000000008CFA0308010000000000000072
:1008F4000000000000000000000000000D000000E7
:10090400000000000000000000000000ECFB0308F1
:1009140000000000000000000000000000000000D3
:10092400E80604080000000000000000780700202A
:10093400040000001CFB0308030000007D480208BB
:10094400E806002008000000FCFB03080C0000007F
:10095400D1480208300700200000000088FA03088C
:1009640003000000B1BD02081807002000000000C9
:1009740004FC030803000000B1BD020800070020C6
:10098400000000008CFA03080100000000000000D1
:100994000000000000000000000000000D00000046
:1009A40000000000000000000000000014FC030828
:1009B4000000000000000000000000000000000033
:1009C400E80604080000000000000000780700208A
:1009D4000400000024FB030803000000B1BD02086A
:1009E40060070020000000008CFA030801000000EA
:1009F40000000000000000000000000000000000F3
:100A04000D000000000000000000000000000000D5
:100A14002D202D2D202D2D2D2D202D2D2D2D000083
:100A240000000000000000000000000000000000C2
:100A34002246002088130C170100000024460020E1
:100A440088130C170000000060FA0308000000007F
:100A540000000000000000000000000070FA03081D
:100A640008000000000000006C03002004000000E7
:100A74007CFA030808000000000000006003002066
:100A84000000000088FA030804000000B5480208CA
:100A940000000000000000008CFA030801000000C0
:100AA4000000000000000000000000000000000042
:100AB4000D00000000000000000000000000000025
:100AC4002046002088130C17010000001E46002059
:100AD40088130C1700000000CCFA03080E00000075
:100AE400F14202080000000000000000780300202A
:100AF4007E4600200100000088C903081C4600202F
:100B04000100000094C90308BC5B0020020000003F
:100B14009CC903089295002000000000000000001A
:100B24009095002000000000000000008E95002039
:100B340000000000000000008C9500200000000070
:100B4400000000008A950020000000000000000062
:100B5400889500200000000000000000CC07002061
:100B640000000000000000001B46002002000000FE
:100B7400A8C90308D4FA030800000000000000001C
:100B8400000000000000000070FA030808000000E4
:100B940000000000FC030020040000007CFA0308AD
:100BA4000800000000000000F00300200000000026
:100BB40088FA030804000000D14202080000000083
:100BC400000000008CFA030801000000000000008F
:100BD4000000000000000000000000000D00000004
:100BE400000000000000000000000000E4FA030818
:100BF40000000000000000000000000000000000F1
:100C0400F4FA03080C0000005949020838040020D3
:100C14000400000000FB03080C0000001543020858
:100C24002C040020040000000CFB03080C0000004E
:100C340019490208200400200000000018FB0308E2
:100C4400030000009948020808040020080000007E
:100C540024FB030803000000B1BD02086007002064
:100C6400000000008CFA03080100000000000000EE
:100C74000000000000000000000000000D00000063
:100C84000000000000000000000000002CFB03082E
:100C94000000000000000000000000000000000050
:100CA40034FB030804000000B949020800000000F6
:100CB400000000008CFA030801000000000000009E
:100CC4000000000000000000000000000D00000013
:100CD40000000000000000000000000080FB03088A
:100CE4000000000000000000000000000000000000
:100CF400F8FE03080C000000000000009804002027
:100D04000400000090FB030808000000000000003D
:100D14008C040020040000009CFB03080800000071
:100D2400000000008004002004000000A4FB03086D
:100D3400080000000000000074040020040000000B
:100D4400ACFB030808000000000000006804002059
:100D540004000000B4FB03080800000000000000C9
:100D64005C04002004000000BCFB03080800000031
:100D7400000000005004002004000000C4FB03082D
:100D840008000000000000004404002004000000EB
:100D94008CFA0308010000000000000000000000BD
:100DA40000000000000000000D0000000000000032
:100DB4000000000000000000CCFB03080E0000004F
:100DC400E14202080000000000000000A40400202A
:100DD400D4FB03080E000000000000000000000027
:100DE400000000001C050020DCFB03080E000000CE
:100DF400000000000000000000000000BC0500200E
:100E04007D46002004000000B4C903085C530020A0
:100E1400E0150C17000000007F46002008000000C9
:100E240064C903088046002005000000C8C90308FF
:100E3400E4FB03080E0000000000000000000000B6
:100E4400000000000C0600202D202D2D202D2D2D1E
:100E54002D202D2D2D0000000000000000000000BA
:100E640000000000000000000000803F0000803F00
:100E740000FFFF0000000000AA5503009FAA5505CB
:100E8400010000AA550701000001AA550B0100004A
:100E9400AA5509020000000001000000C012000071
:100EA40020700020702D7200C00C04080E00000099
:100EB400000000000000000000000000C415002035
:100EC400FFFFFFFFFA000000010000000100000026
:100ED4002CFB0308000000000000000000000000DC
:100EE4000000000023070408040000000F48020863
:100EF40000000000000000008CFA0308010000005C
:100F040000000000000000000000000000000000DD
:100F14000D000000000000000000000000000000C0
:100F2400B66000200100C40900000000B460002085
:100F34000100C40900000000B26000200100C409DF
:100F440000000000B06000200100C409000000009F
:100F5400AC6000200100C40900000000AE60002065
:100F64000100C40900000000AA6000200100C409B7
:100F740000000000A86000200100C4090000000077
:100F84005C0704080E0000000000000000000000E0
:100F94000000000000080020905B00209CFF2C0152
:100FA400000000005A0100200A000000E0D00308FD
:100FB40018460020E0150C1700000000590100201D
:100FC4000800000064C9030858010020050000005F
:100FD400C8C903081A46002002000000F8D003081C
:100FE400845D00200100FF7F010000007C5D002083
:100FF4000200000004D103082C5C00200300000060
:1010040014D103082B5C00200300000014D1030852
:10101400305D00200000F401010000002E5D00207E
:101024000000F401010000002C5D00200000F40128
:10103400010000002A5D00200000F401010000000E
:10104400285D002000FF0100445D0020E803D00774
:101054000A000000425D0020006401000A00000054
:10106400435D0020006401000A0000003C5D002094
:10107400006401000A000000415D002000640100DA
:101084000A000000405D0020006401000A00000026
:101094003F5D0020006401000A0000003B5D002069
:1010A40000FF01000A0000003A5D002000FF01007B
:1010B4000A0000003A5C00200000F4010100000076
:1010C400385C00200000F40101000000365C0020C0
:1010D4000000F40101000000345C00200000F40171
:1010E40001000000375D002000C80100365D0020CB
:1010F40000C80100355D002000C80100345D0020F7
:10110400006401000A000000335D002000FF0100BC
:101114000A000000735D002000C80100725D002019
:1011240000C80100715D002000C80100705D00204E
:1011340000C801006F5D002000C801006E5D002042
:1011440000C801006D5D002000C801006C5D002036
:1011540000C801006B5D002000C80100640704089A
:10116400000000000000000000000000000000007B
:10117400740704080900000000000000A40800200F
:10118400040000007C0704080900000000000000BF
:101194009808002004000000540B04080900000013
:1011A400000000008C0800200400000084070408EC
:1011B4000900000000000000800800200400000076
:1011C40088070408090000000000000074080020DB
:1011D400040000009007040809000000000000005B
:1011E40068080020040000009807040809000000B3
:1011F400000000005C08002004000000A0070408B0
:101204000900000000000000500800200400000055
:101214008CFA030801000000000000000000000038
:1012240000000000000000000D00000000000000AD
:1012340000000000000000008C080408000000000A
:101244000000000000000000000000009C080408EA
:1012540005000000000000002A5C002000000000DF
:101264008CFA0308010000000000000000000000E8
:1012740000000000000000000D000000000000005D
:101284000000000000000000A408040800000000A2
:10129400000000000000000000000000E806040850
:1012A40000000000000000004003002004000000D3
:1012B400B00804080C000000554802080409002086
:1012C4000000000078FB03080C00000065420208DF
:1012D400F8080020000000009CFA03080C0000003D
:1012E40031420208EC080020000000000CFC030856
:1012F4000800000000000000E008002004000000D6
:10130400FCFB03080C0000001D420208D408002066
:1013140000000000B40804080900000000000000F8
:10132400C80800200400000088FA03080300000035
:10133400B1BD0208B0080020000000008CFA0308C8
:101344000100000000000000000000000000000098
:10135400000000000D00000000000000000000007C
:1013640000000000BC0804080000000000000000A9
:101374000000000000000000CC0804080C0000007D
:10138400000000001C09002000000000D40804082C
:101394000A00000000000000F05D002000000000D2
:1013A400E00804080A00000000000000F85D0020C6
:1013B40000000000E80804080A0000000000000023
:1013C400005E002000000000F0080408080000008F
:1013D400000000001009002000000000F8080408C4
:1013E40004000000F5BE0208000000000000000038
:1013F4008CFA030801000000000000000000000057
:1014040000000000000000000D00000000000000CB
:1014140000000000000000000409040800000000AF
:10142400000000000000000000000000180904088B
:101434000C0000000000000034090020000000003F
:10144400280904080400000001BC02080000000090
:1014540000000000300904080C0000000000000037
:1014640028090020000000004409040804000000CA
:10147400E5BB020800000000000000008CFA03082D
:101484000100000000000000000000000000000057
:10149400000000000D00000000000000000000003B
:1014A400000000004C0904080000000000000000D7
:1014B40000000000000000006009040807000000AC
:1014C4000000000070090020000000006C090408FE
:1014D4000800000000000000640900200000000073
:1014E40078090408080000000000000058090020E2
:1014F4000000000084090408080000000000000047
:101504004C090020000000009009040808000000B5
:101514000000000040090020000000008CFA0308CD
:1015240001000000000000000000000000000000B6
:10153400000000000D00000000000000000000009A
:10154400000000009C0904080000000000000000E6
:10155400D307002000000000A80904080B000000C5
:1015640000000000D809002000000000B0090408B1
:101574000B00000000000000CC0900200000000067
:10158400BC0904080B00000000000000C009002092
:1015940000000000C80904080B000000000000005F
:1015A400B409002000000000D40904080B00000066
:1015B40000000000A809002000000000E009040861
:1015C4000B000000000000009C0900200000000047
:1015D400E80904080B000000000000009009002046
:1015E40000000000F40904080B00000000000000E3
:1015F4008409002000000000000A0408080000001C
:101604000000000078090020000000008CFA0308A4
:1016140001000000000000000000000000000000C5
:10162400000000000D0000000000000000000000A9
:10163400000000000C0A0408000000000000000084
:101644000000000000000000200A04080800000058
:1016540000000000080A0020000000002C0A040812
:101664000800000000000000FC0900200000000049
:10167400380A04080800000000000000F0090020F7
:1016840000000000440A04080800000000000000F4
:10169400E4090020000000008CFA030801000000A7
:1016A4000000000000000000000000000000000036
:1016B4000D00000000000000000000000000000019
:1016C4004C0A04080000000000000000D0070020BD
:1016D400000000005C0A04080B0000000000000089
:1016E400380A002000000000680A04080B0000000B
:1016F400000000002C0A002000000000740A040806
:101704000700000000000000240A00200000000080
:10171400800A040807000000000000001C0A0020E2
:10172400000000008C0A040807000000000000000C
:10173400140A0020000000008CFA030801000000D5
:101744000000000000000000000000000000000095
:101754000D00000000000000000000000000000078
:10176400980A04080000000000000000D0070020D0
:1017740000000000A40A04080700000000000000A4
:10178400840A002000000000AC0A040807000000DE
:10179400000000007C0A002000000000B40A0408D5
:1017A4000700000000000000740A00200000000090
:1017B400BC0A040807000000000000006C0A0020B6
:1017C40000000000C40A0408070000000000000034
:1017D400640A002000000000CC0A0408070000008E
:1017E400000000005C0A002000000000D40A040885
:1017F4000700000000000000540A00200000000060
:10180400DC0A040807000000000000004C0A002065
:1018140000000000E40A04080700000000000000C3
:10182400440A0020000000008CFA030801000000B4
:1018340000000000000000000000000000000000A4
:101844000D00000000000000000000000000000087
:10185400EC0A04080E0000000000000065B802084D
:10186400000000008C0A0020285C00201700000003
:1018740024D103081B5C00200A3201001A5C0020FA
:1018840001FA0100165C002000C80100145C00206D
:10189400E803D0070100000046465F50494B4F461D
:1018A40034000000F40A04080E0000007BB80208AB
:1018B40000000000B9BB0208680B0020FC0A040801
:1018C4000E0000007F41020800000000000000003C
:1018D400B80B0020040B04080E000000D5BE02085B
:1018E400A9BA0208A5BA0208940C00200C0B04083B
:1018F4000E0000009DB80208000000000000000077
:10190400480D0020140B04080E00000025B902083D
:10191400F5B8020800000000D40D00201C0B0408D8
:101924000E000000A1B90208E5B902080000000099
:10193400740E0020385D002001030100280B040808
:101944000E000000C9B80208ADB80208000000008B
:10195400640F0020300B04080E00000055B9020883
:101964001DBC020800000000F00F00203C0B04081E
:101974000E00000011BA020861BC02080000000059
:1019840090100020325D002001030100440B040884
:101994000000000000000000000000000000000043
:1019A400500B04080800000000000000BC110020D7
:1019B40000000000580B04080700000000000000AD
:1019C400B411002000000000680B040807000000A8
:1019D40000000000AC11002000000000740B04089B
:1019E4000700000000000000A41100200000000017
:1019F400800B04080C000000000000009811002077
:101A0400000000008C0B040803000000B1BD0208B4
:101A140080110020000000008CFA0308010000007F
:101A240000000000000000000000000000000000B2
:101A34000D00000000000000000000000000000095
:101A4400940B0408000000000000000000000000E7
:101A540000000000A40B04080A00000000000000BD
:101A6400B0DB030800000000AC0B04080A0000000F
:101A74000000000008DB030800000000B40B0408A9
:101A84000A00000000000000745D00200000000057
:101A9400BC0B04080A00000000000000C81100206C
:101AA400000000008CFA03080100000000000000A0
:101AB4000000000000000000000000000D00000015
:101AC400000000000000000000000000C40B040837
:101AD4000000000000000000000000000000000002
:101AE400D80B040803000000B1BD02080412002052
:101AF40000000000E40B040803000000B1BD02086C
:101B04005C01002000000000EC0B0408030000004E
:101B1400B1BD0208EC11002000000000F40B040821
:101B240003000000B1BD0208D41100200000000031
:101B34008CFA03080100000000000000000000000F
:101B440000000000000000000D0000000000000084
:101B54000000000000000000000C04080000000069
:101B64000000000000000000000000000C0C04084D
:101B740007000000ADBC0208B41200200000000001
:101B8400900E040803000000B1BD02089C1200205E
:101B940000000000180C040803000000B1BD020896
:101BA4008412002000000000200C04080300000040
:101BB400B1BD02086C12002000000000280C0408CB
:101BC4000700000091BC020864120020000000001D
:101BD40094FB030803000000B1BD02084C1200206E
:101BE40000000000340C040803000000B1BD02082A
:101BF4003412002000000000400C04080300000020
:101C0400B1BD02081C120020000000008CFA030879
:101C140001000000000000000000000000000000BF
:101C2400000000000D0000000000000000000000A3
:101C3400000000004C0C04080E00000035B8020837
:101C440005B8020800000000BC120020540C04086F
:101C54000E00000079BA0208000000000000000035
:101C640070130020600C04080E0000000000000047
:101C74000000000000000000FC130020700C0408A9
:101C84000E00000055BA0208C9BC0208000000009A
:101C940088140020780C04080000000000000000F4
:101CA4000000000000000000840C04080300000091
:101CB400B1BD0208AC15002000000000640C04084B
:101CC40003000000B1BD02089415002000000000CC
:101CD4008C0C040803000000B1BD02087C15002030
:101CE40000000000980C040803000000B1BD0208C5
:101CF4006415002000000000A00C0408020000008D
:101D040041BF02080000000000000000A80C040805
:101D14000200000041BF02080100000000000000B2
:101D2400B40C04080200000041BF020802000000D5
:101D340000000000000000000D0000000000000092
:101D4400000000000000000000000101FFFF00008F
:101D5400C4F803080000000000000000919A010884
:101D6400A086010004000000000000000000000044
:101D7400000000000000000000000000000000005F
:101D840000000000900E040818F80308000000008A
:101D940045EA00087D000000060000000000000085
:101DA400000000000000000000000000000000002F
:101DB4000000000000000000CC0C0408000000003B
:101DC40000000000A1560308E8030000030000001F
:101DD40000000000000000000000000000000000FF
:101DE400000000000000000000000000D40C040803
:101DF40000000000000000008955020810270000C0
:101E040003000000000000000000000000000000CB
:101E140000000000000000000000000000000000BE
:101E24007C080408000000004DF60108E5380108AC
:101E3400204E00000500000000000000000000002B
:101E4400000000000000000000000000000000008E
:101E540000000000F8FD030800000000000000007E
:101E64005D5103081027000001000000000000007D
:101E7400000000000000000000000000000000005E
:101E84000000000000000000E00C04080000000056
:101E940000000000956F0108E80300000500000041
:101EA400000000000000000000000000000000002E
:101EB400000000000000000000000000EC0C04081A
:101EC4000000000000000000C1B40108204E000022
:101ED40003000000000000000000000000000000FB
:101EE40000000000000000000000000000000000EE
:101EF400FC0C04080000000000000000CDB2010842
:101F0400204E00000300000000000000000000005C
:101F140000000000000000000000000000000000BD
:101F2400000000000C0D0408000000000000000088
:101F3400ED4E0308400D0300030000000000000004
:101F4400000000000000000000000000000000008D
:101F5400000000000000000078F903080000000001
:101F640000000000C9AE01081027000001000000B5
:101F7400000000000000000000000000000000005D
:101F840000000000000000000000000034F8030816
:101F94000000000000000000499F02081027000014
:101FA400030000000000000000000000000000002A
:101FB400000000000000000000000000000000001D
:101FC40000FE03080000000000000000018000087B
:101FD400A00F00000100000000000000000000004D
:101FE40000000000000000000000000000000000ED
:101FF400000000001C0D04080000000000000000A8
:102004003DCF02081027000001000000000000007E
:1020140000000000000000000000000000000000BC
:10202400000000000000000064FE0308000000003F
:102034000000000071A70208102700000100000042
:10204400000000000000000000000000000000008C
:102054000000000000000000000000000CF803086D
:1020640000000000000000008DC002081A410000BA
:10207400010000000000000000000000000000005B
:10208400000000000000000000000000000000004C
:10209400280D04080000000000000000099B01084E
:1020A400400D0300000000000000000000000000DC
:1020B400000000000000000000000000000000001C
:1020C40000000000300D04080000000000000000C3
:1020D400C59A0108400D0300000000000000000044
:1020E40000000000000000000000000000000000EC
:1020F4000000000000000000380D0408000000008B
:1021040000000000A59B0108A08601000300000058
:1021140000000000000000000000000000000000BB
:1021240000000000000000000000000030303030EB
:102134002D30312D30315430303A30303A30300097
:102144000100000000000000010203040102030476
:1021540006070809040309041201000202020040F0
:1021640083044057000201020301000009024300F6
:10217400020100C03209040000010202010005242A
:1021840000100105240100010424020205240600B4
:1021940001070582030800FF09040100020A000088
:1021A400000705010240000007058102400000000D
:1021B400FF000000252C030865290308E90E030825
:1021C40079270308D12B030889270308A5270308C7
:1021D40069270308592703080000000000000000D5
:1021E400006002401060024000000000000B00008C
:1021F4000000200000000000000000000060024019
:102204002860024000000000060C000000002000CE
:102214000000000000000000006002404060024036
:1022240000000000100D000000002000000000006D
:1022340000000000006002405860024000000000FE
:10224400160E000000002000000000000000000046
:10225400006002407060024000000000200F000097
:1022640000002000000000000000000000600240A8
:1022740088600240000000002610000000002000DA
:10228400000000000000000000600240A060024066
:1022940000000000301100000000200000000000D9
:1022A4000000000000600240B8600240000000002E
:1022B400362F000000002000000000000000000095
:1022C4000064024010640240000000000038000076
:1022D4000000400000000000000000000064024014
:1022E400286402400000000006390000000040009D
:1022F400000000000000000000640240406402404E
:1023040000000000103A000000004000000000003F
:102314000000000000640240586402400000000015
:10232400163B000000004000000000000000000018
:10233400006402407064024000000000203C000081
:1023440000004000000000000000000000640240A3
:1023540088640240000000002644000000004000A1
:10236400000000000000000000640240A06402407D
:1023740000000000304500000000400000000000A4
:102384000000000000640240B86402400000000045
:10239400364600000000400000000000000000007D
:1023A4000000000100000000000000000000000028
:1023B40001000000430000000000000000000000D5
:1023C4000000000000000000000000000000000009
:1023D40000000000430000000000000000000000B6
:1023E40000000000000000000000000000000000E9
:1023F4000000000043000000000000000000000096
:1024040000000000000000000000000000000000C8
:102414000000000043000000000000000000000075
:1024240000000000000000000000000000000000A8
:102434000000000043000000000000000000000055
:102444000000000000000000000000000000000088
:102454000000000043000000000000000000000035
:102464000000000000000000000000000000000068
:102474000000000043000000000000000000000015
:102484000000000000000000000000000000000048
:1024940000000000B9870308F98503080000000064
:1024A4005E1204081E0704086CDF03086CDF0308CF
:1024B4006CDF03086CDF03086CDF03086CDF0308C0
:1024C4006CDF03086CDF03086CDF0308FFFFFFFF0A
:1024D400FFFFFFFFFFFFFFFFFFFF0000010041536D
:1024E4004349490000000000000000000000000013
:1024F4000000000000000000000000000000415344
:1025040043494900000000000000000000000000F2
:1025140000000000000000000000000000000000B7
:10252400541E002000000000000000000000000015
:102534000000000000000000000000000000000097
:102544000000000000000000000000000000000087
:102554000000000000000000000000000000000077
:102564000000000000000000000000000000000067
:102574000000000000000000000000000000000057
:0825840000000000010000004E
:108000002DE9F04F2DED028B93B0834625F074FCE3
:10801000914B1D7825B113B0BDEC028BBDE8F08FFC
:108020008E4B1B685905F6D58D4B8E4E1B6863B180
:108030008D4A31681368CB1A7C2B06D98B481160A6
:108040000378013303702AF071F8894B1B78002BF9
:1080500072D0884C884AD4F81031ABEB03039342BA
:1080600001F2548394F81891B9F1000F35D1DFF87B
:108070003C82D8F800000EF03FF9C0B201280FD9B9
:1080800002287E4F42F066803B78002B42F0B1819F
:10809000D4F81C31ABEB0303B3F57A6F82F0EF82B7
:1080A000D4F82031002B47D094F81831C3B9744B61
:1080B0001B689B7801211E3B00228B4284F818111B
:1080C00084F82C2142F29682D8F800000221043074
:1080D00029F0DEFF94F8243111E0D4F820315BB3AD
:1080E000D4F8283140F6B732ABEB0303934223D9DF
:1080F00094F82431002B01F0F986DFF8B081013BC0
:10810000DBB284F82431002B01F02684D4F82071EE
:1081100094F82C2117F8011B94F82D31D8F80000A1
:10812000C4F820710A44013384F82C2184F82D31DD
:108130000EF0E6F8C4F828B1524B37681B7853B1FB
:10814000DFF86C81D8F8000028B14F4B1B78013B59
:10815000012B41F211844D4B1B7873B1DFF8548130
:10816000D8F800304BB13368424C02931A46D4F829
:108170004431D31A632B01F2B281DFF83C8198F8C5
:108180000030022B01F08A863C4F97F87430032BA5
:1081900001F0CC833E4B1B7873B13E4D2B685BB135
:1081A000344C10F03BFAD4F85031029044F61F6280
:1081B000C31A934200F23081374B1B78002B7DD1DC
:1081C000364B1B7843B12B4CD4F8A03203F5C333A4
:1081D000A0339B4581F03E82314B1B78002B3FF44E
:1081E0001AAF244E2F4C304D06F2C12720680EF0F6
:1081F00083F800283FF40FAF20680EF075F82B7855
:1082000080465A1E33B120682A700EF075F8002897
:10821000F2D100E703223946781E32F064FC96F86A
:10822000C03296F8C12286F8C38283F47F4383F07C
:10823000FF039B1A1FFA88F89BB2B8EB132FD5D116
:1082400096F8C222DBB29A42D0D1781E23F050FABF
:108250002B7818442870C9E74F5900202C6A002059
:10826000586C00208C790020786E0020746E0020FD
:108270009E610020B81E00203F0D0300000000207A
:10828000286E0020A0610020A8610020B0610020BD
:10829000B8610020BC610020286200203962002003
:1082A000C2610020C8610020CC610020246E002043
:1082B0005C6C00201C6E00205E370020484C227849
:1082C000A2B1484B9B7A53B110F0A8F9464B1B68FA
:1082D000C31AA3F57A73B3F5FA6F07D82278434B24
:1082E000434918680DF0D4FF00232370414CD4F8A3
:1082F000983203F5C333A0339B45FFF461AF3E4D85
:10830000C4F898B22B78002B41F035873B4D2B7881
:10831000002B41F08D8694F89C2239498D5CEA0748
:1083200001F1E787AF0701F1A787680702F12B800A
:108330002A0748D5334B344F0B9312AA1146A3F1A9
:108340003D0241F8202D0020A3F140020D4603F824
:10835000400C039102231121517093702846396813
:1083600003F016FC2846796803F012FCFB892749C4
:1083700003EBC3039B00053381FB0321DB17C3EB36
:10838000A101284689B203F01BFC3B8A03EB83035F
:10839000590089B2284603F013FC1D4B039D1B783E
:1083A0009B0743BF398901F57A7189B24FF47A711D
:1083B000284603F005FC0A9B3A7D591C0A91284681
:1083C0001A7025F029FA134A94F89C321178013377
:1083D00093FBF1F201FB123384F89C32F0E600BF0C
:1083E00090610020906B0020CC3600202C62002091
:1083F00050610020B81E0020306200203162002051
:108400003462002050610020A06E0020676666661E
:108410009C6E00203862002094F85631002B41F009
:108420008A85DB4B1A6802F00803002B4AF60B40E2
:1084300048F603414BF60F4349F6074704BF03468E
:108440000F4612F0040F4FF0190118BF1F46900697
:1084500084F8561103D547F4804747F02007CD4BE9
:108460005A79C7F30909002A42F031819B79002B20
:1084700042F03D82984664204FF0FF3A4FF0000CE6
:108480000A970B97ADF834C0CDF83AC0CDF83EC08E
:10849000CDF842C0CDF83090ADF83680ADF838A0B8
:1084A0008DF846000AAF0FCFDFF800E384F805C06F
:1084B000AEE80F0097E80F00AEE807002EF8023B89
:1084C00071464FF0010C1B0CFE271F20C82201F83B
:1084D0001E39A770A27184F807C0E07094F8660195
:1084E000207180F0F10383EA0313DAB2130983F0F9
:1084F000E70343EA022383EAC2031BB283EA0312BF
:10850000D2B2C3F3072383EA121343EA022383EAB6
:10851000C2031BB283F0C80282EA0212D2B2C3F3D2
:10852000072383EA121343EA022383EAC2031BB23E
:1085300083EA0C0787EA0717FFB2C3F3072282EA30
:10854000171242EA072200EB0C0382EAC7070EEB80
:108550000C0084F86631278011F8013B7B4083EAE8
:108560000313DBB21A0982EA172242EA032282EAE3
:10857000C3031BB29FB281422780EDD183F07C03FD
:1085800083EA0313DBB24FEA131E8EEA172E8EEA3C
:10859000032E8EEAC30E0FFA8EFE1FFA8EF9DFF855
:1085A00010C2A4F800905FFA8EFE4FEA192984F8F1
:1085B000289084F827E00CF5C77804F1220ADCF84B
:1085C0000000DCF80410DCF80820DCF80C3047462A
:1085D0000FC70CF1100CD445B846F0D1DCF8000000
:1085E00038606D4F9CF8043088F8043007F1270894
:1085F00084F8B5E184F8B69117F8011F28680DF0EA
:108600007FFEB845F8D194F85731002B41F08E84A5
:108610006249326809780A2084F85701002901F07C
:1086200021865F4F01293888069042F2578102293E
:10863000B7F802E002F06580B8880590032902F0DF
:108640005D81F8880490042902F06E81052938893B
:1086500002F065810629B7F80A9002F05C810729CB
:10866000B7F80C8002F05481FB89039394F86611EB
:108670000A920B4683F0300282EA0212D2B2170944
:108680004849079387F07A0747EA02270988237148
:1086900087EAC202444FC1EB012187FB013A069BE6
:1086A0004FF0000C63F30F0C059B6EF31F4C4FF063
:1086B000000E63F30F0E049BCDF82CC012B28A4457
:1086C0000027C91763F31F4EC1EB6A2A039BCDF83D
:1086D00030E082EA021160F30F070020C9B268F3AC
:1086E0000F00C2F3072269F31F4782EA111263F3F6
:1086F0001F404FF000090D978DF83DA00E908DF8AA
:108700003C9042EA01220DF1280C82EAC107BCE844
:108710000F003FB287F0C80888EA0818DFF88CE03D
:1087200084F805905FFA88F8C7F30727AEE80F00D2
:1087300087EA181747EA08239CE8030083EAC8037E
:108740001BB283F023024EF8040B82EA0212D2B26B
:10875000C3F30723079F83EA1213704643EA0223F9
:1087600083EAC20207F1010C20F814194FF0230824
:108770001621FE27C82384F866C1228084F807806A
:108780000EF1020EA770E170A371114612E000BF56
:10879000986E0020846E002047200020D8350020ED
:1087A000A8600020D060002003082080C01E0020A8
:1087B000BA1E002010F8013B4B4083EA0313DBB2E2
:1087C0001A0982EA112242EA032282EAC3031BB297
:1087D00099B270452180EDD183F0F40383EA03134D
:1087E000DBB24FEA131E8EEA112E8EEA032E8EEABA
:1087F000C30E0FFA8EFE1FFA8EF8CA4FA4F800803F
:108800004FEA182C5FFA8EFE84F81EE084F81FC031
:108810007968BA683868FB6807F5C778A8E80F0078
:1088200038697969BA6904F28F17A8E8070004F279
:10883000AD1884F8ADC184F8ACE117F8011F2868C1
:108840000DF05EFDB845F8D194F85A31002B41F097
:108850007783B54B1B681922990684F85A2140F199
:10886000FC82B24BB24F1B789A0741F128873B7DBF
:10887000042B8CBF4FF003084FF002080FF0CEFE20
:108880003B8A3A890A9003EB83035B00ADF84230E0
:108890004FF47A703B680C93F98997F814E07B6881
:1088A0008DF8448000FB02F24FF0000C0AA84FF054
:1088B000FF398DF845E0CDF82CC0CDF83C900E92F4
:1088C0000D93ADF8401080460390B8E80F00DFF834
:1088D00070E2AEE80F0098E80F00AEE807007246BD
:1088E000182122F81C39E17194F8661184F805C04A
:1088F00081F0780383EA0313D8B2030983F0F60307
:1089000043EA002383EAC0031BB283EA0310C0B228
:10891000C3F3072383EA101343EA002383EAC00367
:108920001BB283F0C80080EA001C5FFA8CFCC3F322
:10893000072080EA1C1040EA0C2080EACC0000B23C
:1089400080F0180383EA0313DBB2C0F3072080EA48
:10895000131040EA032080EAC30301F101081E203E
:108960004FF0FE0C4FF0C809E0700EF1020E2171BD
:1089700084F86681238084F802C084F80690184643
:1089800012F8011B414081EA0111C9B20B0983EAC7
:10899000102343EA012383EAC10109B288B2724578
:1089A0002080EDD181F0180181EA0111C9B20A09D4
:1089B00082EA102383EA012383EAC1031BB29AB23D
:1089C000DFF860A12280DBB2120A0592049384F8DA
:1089D000272084F82630D6460AF5C77904F1220804
:1089E000DEF80000DEF80410DEF80820DEF80C30B7
:1089F000CC46ACE80F000EF1100EC645E146EFD1B3
:108A0000DEF80000CCF800009DF81030DFF834816B
:108A100084F8B4319DF8143084F8B531C14619F8A2
:108A2000011F28680DF06CFC424B4B45F7D10FF04D
:108A3000F5FD414B414AB3F90410B7F808E03B6833
:108A40000B930A907B680C9382FB01274FF47A709A
:108A5000C9174FF0000C00FB0EF0C1EBA701DDF8C9
:108A60000CE0ADF83CC0ADF83EC0ADF840C0ADF88C
:108A700042100D900E90BEE80F00314F84F805C0F3
:108A80000FC79EE807004FF0210C87E807001C2362
:108A9000C8224FF0FE0EE37084F807C084F802E0AD
:108AA000A27194F86611217181F06A0383EA0313BD
:108AB000DAB2130983F0D50343EA022383EAC2033F
:108AC0001BB283EA0312D2B2C3F3072383EA121361
:108AD00043EA022383EAC2031BB283F0C80282EA9C
:108AE0000212D2B2C3F3072383EA121343EA02232A
:108AF00083EAC2031BB283EA0C0282EA0210C0B20C
:108B0000C3F3072282EA101242EA0022013182EA0C
:108B1000C0020C3784F866112280A7F11C011046B0
:108B200012E000BFBA1E0020986E00209C6E00204C
:108B3000A06E00206D2000207C6E002067666666B7
:108B4000C01E00204720002011F8013B434083EA6B
:108B50000313DBB21A0982EA102242EA032282EAF4
:108B6000C3031BB298B2B9422080EDD183F06803F1
:108B700083EA0313DBB2190981EA102282EA032295
:108B800082EAC3031BB29AB2DB4F2280DBB24FEA08
:108B9000122C049384F8243004F1220384F825C0B5
:108BA00007F5C7790593FB6838687968BA68CE46D7
:108BB000AEE80F00059B10379F42F146F3D13B888A
:108BC000AEF800309DF81030CC4F84F8B231C14679
:108BD00084F8B3C119F8011F28680DF091FB4F45C7
:108BE000F8D194F866C1C64AC64F84F804C08CF028
:108BF000EB0383EA0313D9B20B0983F0C50343EAFD
:108C0000012383EAC1031BB283EA0310C0B2C3F39A
:108C1000072181EA101141EA002181EAC0010CCA52
:108C200009B281F0C80E8EEA0E1E5FFA8EFE4FF07A
:108C300000090A92C1F30721039A0B93CDF83090F3
:108C400081EA1E1343EA0E2307CA83EACE031BB24E
:108C500083F0310E87E807008EEA0E1E5FFA8EFE63
:108C6000C3F3072383EA1E1343EA0E2383EACE03EA
:108C700094F808E0607AA17AE27A277B84F805907C
:108C80001BB28EEA030E8EEA0E1E5FFA8EFEC3F34F
:108C9000072383EA1E1343EA0E2383EACE031BB2A3
:108CA000584080EA0010C0B2C3F3072383EA1013D0
:108CB00043EA002383EAC0031BB2594081EA011052
:108CC000C0B2C3F3072181EA101141EA002181EA11
:108CD000C00109B24A4082EA0212D2B2C1F30723AC
:108CE00083EA121343EA022383EAC2031BB25F4002
:108CF00087EA0717FFB2C3F3072383EA171343EA90
:108D00000723607BA17BE27B94F810E094F811903C
:108D100083EAC7031BB2584080EA0010C0B2C3F315
:108D2000072383EA101343EA002383EAC0031BB23C
:108D3000594081EA0111C9B2C3F3072383EA111331
:108D400043EA012383EAC1031BB25A4082EA0212BA
:108D5000D2B2C3F3072383EA121343EA022383EA5E
:108D6000C2031BB28EEA030E8EEA0E1E5FFA8EFE5F
:108D7000C3F3072383EA1E1343EA0E2383EACE03D9
:108D80001BB289EA030989EA09195FFA89F9C3F371
:108D9000072383EA191343EA092383EAC903A17C61
:108DA000E27C594F1BB2594081EA0111C9B2C3F3A9
:108DB000072383EA111343EA012383EAC1031BB2A9
:108DC0005A4082EA0212D2B2C3F3072383EA121393
:108DD00043EA022383EAC2031BB283F0270989EA2C
:108DE0000912D2B2C3F3072989EA121949EA022902
:108DF00089EAC2090FFA89F91FFA89F20CF1010315
:108E00004FEA122E5FFA89F931204FF0FE0C0C2147
:108E100084F86631C8232280E07184F802C0E170D2
:108E2000A37184F8149084F815E0DAF80410DAF8E5
:108E30000820DAF80C30DAF80000BAF810C00FC7D2
:108E400027F803CB84F8A3E184F8A29118F8011F56
:108E500028680DF055FA4745F8D194F85EC1BCF189
:108E6000000F41F07880294B94F866E1B3F90010C7
:108E7000B3F90220B3F904309FED256A214F84F83D
:108E800005C007EE103A33680A938EF06A0383EA4E
:108E9000031306EE901AD9B20B0983F0D50343EA07
:108EA000012383EAC1031BB283EA03115242C9B210
:108EB00007EE902AC3F3072383EA111343EA012341
:108EC000F8EEE77AF8EEE66AB8EEC77A83EAC1030D
:108ED0001BB267EE867A66EE866A27EE067A002077
:108EE00083F0C808CDED0C7ACDED0B6A8DED0D7ACF
:108EF0000E900F900EE000BFBA1E00206B200020E5
:108F000054590020C01E0020482000207C6E002004
:108F100088C3E43A109088EA08160DF12809F6B2E1
:108F2000C3F30728B9E80F0088EA161848EA0628AC
:108F300088EAC6080FFA88F80FC788F01E0699E875
:108F4000070086EA0616F6B2C8F3072383EA16136B
:108F500043EA062387E8070083EAC606C8214FF0E4
:108F600005084FF01E0CFE231C200EF10102A1711A
:108F700084F85E8184F807C0A370E070A7F1100147
:108F800084F804E00C37268084F8662111F8013B50
:108F9000734083EA0313DBB21A0982EA162242EA1B
:108FA000032282EAC3031BB29EB2B9422680EDD1EE
:108FB00083F0270383EA0313DBB24FEA131E8EEA22
:108FC000162E8EEA032E8EEAC30E0FFA8EFE1FFABD
:108FD0008EFCD94FA4F800C05FFA8EFE4FEA1C2C1D
:108FE00084F825C084F824E007F5C77804F1220945
:108FF00038687968BA68FB6846460FC610374F452F
:10900000B046F5D1CD4E3B88A8F8003006F12407D4
:1090100084F8B2E184F8B3C116F8011F28680DF096
:109020006FF9B742F8D194F85F81B8F1000F40F0C2
:109030008C87C34B1B6805229B0684F85F2141F196
:109040000B81C04BDFEDC06ADA891B8907EE902ADD
:1090500007EE103AF8EEE77AB8EE477A67EEA67AAE
:1090600094F866C1B94BBA4AB3F90410B2F90620B4
:10907000B84EB948CDED0B7A8CF0220383EA031386
:10908000DFB23B0983F0590343EA072383EAC703AE
:10909000B2F5FA6F1BB2A8BF4FF4FA6283EA031766
:1090A000FFB2B2F57A7FC3F3072383EA1713B8BF81
:1090B0004FF47A724FF0640E43EA0723A2F57A72F6
:1090C0000EFB02F283EAC70786FB02E680FB01E0A3
:1090D0003FB2C917D217C2EBA612C1EBA0034FF0E3
:1090E00000090AA987F0C8068DED0C7AADF83A2080
:1090F000ADF83830CDF82890CDF834908E4686EA19
:109100000616F6B20391C7F30727BEE80F0087EAF9
:10911000161747EA062787EAC606904FDEF800E0F2
:1091200084F804C00FC736B286F04A0383EA0313FB
:10913000DBB2C6F3072181EA13113A4641EA032163
:109140000CF1010C81EAC303142042F810E9FE2659
:109150004FF04A0E002184F866C14FF0C80CE07051
:109160002380043784F807E0A670617184F806C094
:10917000184612F8011B414081EA0111C9B20B09DE
:1091800083EA102343EA012383EAC10109B288B2CA
:10919000BA422080EDD181F0140181EA0111C9B2F7
:1091A0004FEA111E8EEA102E8EEA012E8EEAC10EB3
:1091B0000FFA8EFE1FFA8EF6DFF87CA126804FEAAA
:1091C000162C5FFA8EFE84F81CE084F81DC0DAF8D5
:1091D0000410DAF80000DAF80820DAF80C30BAF8EF
:1091E00018900AF5C7770FC7DAF81000DAF81410EC
:1091F00003C704F28F16A7F80090374684F8ABC176
:1092000084F8AAE104F2AB1917F8011F28680DF0E1
:1092100077F8B945F8D1524B524A1B781278013B86
:1092200012F00100DBB214BFC0214021172B03D87C
:109230004D4A134493F830804C4B1A8897071ABF55
:10924000002341F01001012312F4027F18BF022312
:1092500012F0100F18BF062312F0200F18BF1023B2
:10926000002841F002824FF0030C94F866E10A9363
:109270008EF0460383EA0313DAB2130983F09203F4
:1092800043EA022383EAC2031BB283EA0310C0B29B
:10929000C3F3072282EA101242EA002282EAC002E5
:1092A00012B282F0C80787EA0717FFB2C2F307229B
:1092B00082EA171200238DF82FC0032042EA072C00
:1092C000039A8DF82C808DF82D308DF82E108DF8A6
:1092D000300007CA8CEAC70C0FFA8CFC1F4FE371F1
:1092E0008CEA0C1803C75FFA88F8CCF3072C8CEAD9
:1092F000181C4CEA082181EAC80894F808C03A70A2
:109300000FFA88F88CEA080C8CEA0C1C5FFA8CFCCB
:10931000C8F3072282EA1C1242EA0C22607AA17A80
:1093200094F80B80637182EACC0212B2504080EA5A
:10933000001C5FFA8CFC1BE0BA1E002047200020B6
:10934000986E0020A06E00200AD7233C7C6E00207F
:10935000A8600020D34D621067666666C01E0020BC
:10936000E83900205C5B002084AC0308D260002058
:10937000C2F3072080EA1C1040EA0C2080EACC00EF
:1093800000B2414081EA0111C9B2C0F3072282EA6A
:10939000111242EA012282EAC10212B288EA0208EC
:1093A00088EA08185FFA88F8C2F3072282EA1812DE
:1093B00042EA082294F80CC0607BA17B84F804E0A8
:1093C00082EAC80212B28CEA020C8CEA0C1C5FFA28
:1093D0008CFCC2F3072282EA1C1242EA0C2282EAC7
:1093E000CC0212B2504080EA0010C0B2C2F3072291
:1093F00082EA101242EA002282EAC00212B251400E
:1094000081EA0111C9B2C2F3072282EA111242EACB
:10941000012282EAC102E17B94F8108013B281EA52
:10942000030282EA0212D2B2C3F3072383EA1213C1
:1094300043EA022383EAC2031BB288EA030282EAF8
:109440000212D2B2C3F3072383EA121343EA0223C0
:1094500083EAC2031BB283F0320282EA0212D2B262
:10946000C3F3072383EA121343EA022383EAC20306
:109470001BB29AB24FF0FE0C0920C8210EF1010E6A
:10948000DBB284F802C04FEA122CE070A17184F8BC
:1094900066E1228084F812C06374DAF80000DAF81A
:1094A0000410DAF80820BAF80C9007F5C07EAEE890
:1094B000070007F5C8778EF80280AEF8009084F8B0
:1094C000A0C184F89F3116F8011F28680CF018FF1E
:1094D000B742F8D1029BC4F85031FEF76DBEDFF8F9
:1094E00024A27C4FDFF82092412028F07DFDBAF9BC
:1094F000023087FB0320DB17C3EBA00080B228F00B
:1095000057FDBAF9003087FB0320DB17C3EBA0003F
:1095100080B228F04DFDBAF9043087FB0320DB1739
:10952000C3EBA00080B228F043FD99F80010D8F8F2
:1095300000000CF0E5FE94F848A11AF0010700F0D5
:109540001085654B1B689A0672D5644B644F1B7877
:109550009B0741F14B803B7D042B8CBF4FF0030AEE
:109560004FF0020A472028F03FFD386828F0ECFC55
:10957000786828F0E9FCFB895A4AD8F80000A2FB79
:109580000323C3F34713194603930CF0B9FE3A893A
:1095900099F80010039B64204B4000FB02F089F80F
:1095A000003028F0D1FC3F7DD8F800004AEA870758
:1095B000FFB239460CF0A4FE99F80030D8F800004C
:1095C0005F40394689F800700CF09AFE94F848A183
:1095D000BAF1000F2CD1444F4F2028F005FD386818
:1095E00028F0B2FC786828F0AFFC504628F0ACFCBC
:1095F0000121D8F800000CF083FE384A99F80030B9
:109600001778D8F8000007F00107394683F0010306
:1096100089F800300CF074FE99F80030D8F800009A
:109620005F40394689F800700CF06AFE94F848A152
:10963000029B2E4AC4F844310AF10103DBB2A2FBBB
:109640000312D20802EB8202A3EB420384F84831F2
:10965000FEF793BD94F8A432254AC4F8A0B202EBF9
:109660008302926C42B312AD04F2AB23214E45F853
:10967000203D002104F2BD2331800B93802115236E
:10968000A52784F8AA32284684F8A91284F8A8727B
:1096900090472846318802F0B9FA0A9D164804F529
:1096A0002A716D1A152DA8BF15252A462EF0B6FF72
:1096B000124A94F8A4321570114A013382FB031246
:1096C000A2EBE37202EB42029B1A84F8A432FEF78B
:1096D00083BD00BF67666666986E00209C6E0020A2
:1096E000A06E00201F85EB5154590020CDCCCCCC6E
:1096F00084AC03080C610020283900203D3900208B
:10970000565555557C6E0020206E0020C24AC34B32
:10971000D4F8141130681B8892F80BE0C04A401A44
:109720004FF47A71DFB201FB0EF11B0A97771775C0
:1097300088424FF00007D37753759770177180F008
:10974000F784B849DFF808C30B688968B648B74F93
:10975000007897F814A08CFB03E8DB178CFB01EC76
:109760004FEAE17EC3EBA80111770912CEEBAC0EF4
:109770005177F4214FEA2E2C82F820E091764FF0B9
:10978000010E302182F81BE082F82210A84B82F8EB
:1097900021C04FF0750E782182F823E082F8241062
:1097A000820783F81AA040F1BF84D7F800C0A14A0D
:1097B000D7F804E0A04882FB0C194FEAEC7182FB59
:1097C0000E82C1EBA9514FEAEE79C9EBA25200FB20
:1097D00001C9029200FB02E009EB4909974A4FEAEE
:1097E000490982FB0982049200EB4000934A400041
:1097F000039082FB0008049A9014029A0490F8895E
:109800003F8902EB820200EBC00002EB820207F507
:10981000FA770692BAF1050F4FEA80021FFA87FA2B
:109820000398049F029201EB81014FEAE97201EB78
:10983000810105914FEAE071A7EB0200804F83F8A8
:1098400015A0024607FB1292059F4FEAA84840B2B6
:1098500000EB8709A8EB0100794F0399804607FBCD
:109860001010069F77494FFA88F84FEADC7C4FEAE0
:10987000DE7E83F809C083F80EE0DFF8D8C108EB7C
:10988000870E029F81FB07814FEAE778BCF80070E2
:109890000397C8EBA1116C4F029187FB021887FB5D
:1098A00000170299DFF8B0C11FFA89F91FFA8EFE7E
:1098B0004FEAE2724FEAE070C2EB681883F80A9050
:1098C000C0EB671283F80FE04FEA19274FEA1E2911
:1098D000C1F3072E0399BCF80000DF7283F81090E3
:1098E0004FEA222783F80C805A749DF80820DA7119
:1098F0004FEA282C4FEA1A2A4FEA112934BF4FF0B9
:1099000032084FF033089DF80C2083F80DC09F7487
:1099100083F816A083F808E0DA7483F8149083F8CB
:109920001B801877C4F810B1FEF79CBBDFF82C91B0
:10993000D9F800000CF0D0FC00283EF42BACD9F88C
:10994000000001210CF0C4FC0222002387F87420DF
:1099500088F80030FEF71EBC94F82C1194F82D31D5
:10996000D8F800004A1C013384F82C2184F82D31EA
:109970000CF0C6FCFEF7DEBB344CDFF8E4904FF091
:10998000000A0BE01B2B00F09F820D2B00F0798169
:109990004FF0010389F80130D8F800000CF0ACFC5E
:1099A00000285FD0D8F800000CF09EFC83B27E2B1C
:1099B00032682AD099F801100029EDD194F82E21AF
:1099C000002ADFD07D2B00F0648294F83CE1BEF1E8
:1099D000000F04D080F02003DBB284F83C11511C4E
:1099E000C9B22244092984F82E1182F8303100F0DE
:1099F00044820829D0D8B4F83A21134403EB132346
:109A000003F0FF03A4F83A31C6E784F82EA184F8E6
:109A10002FA189F801A0BFE7D85B0020D05B002010
:109A2000D0610020646C00209C6E0020A06E00209D
:109A3000FC6100206BCA5F6B806967FF83DE1B439C
:109A400040420F00D34D62101F85EB51B81E00201D
:109A500067666666A4590020A6590020EC370020EE
:109A60000000002094F83D3133B194F8313184F88E
:109A70003D01302B00F0D78594F82F21BA4BBB491C
:109A8000DFF818A3DFF8189302954FF0010E904607
:109A90004246002A00F05B833268D21B012A00F2A2
:109AA0001F8294F83E21002A40F0348294F83FC18E
:109AB00033F81C00F0B984F83FE10A689506E7D551
:109AC0009AF800209007E3D5A94FAA49FA89029D88
:109AD0004FF4F36303FB02F381FB0321DB17C3EBBA
:109AE00061114FF4036028F0B9FA002384F82F3194
:109AF000FEF731BB0CF1010C5FFA8CFCB0F5E06FA6
:109B000084F83FC100F09A801BD8B0F5047F00F0C4
:109B1000498136D8B0F5887F00F0D380B0F5007F5A
:109B200000F0B880B0F5807FB2D10A685207AFD597
:109B30000021029D28F092FA002384F82F31FEF7CD
:109B40000ABBB0F5026F00F05E816CD8B0F5E46F2F
:109B500000F08480B0F5006F00F0DD80B0F5E26FBA
:109B600096D1854B029DDA6B998A642303FB02F33D
:109B700093FBF1F128F072FA002384F82F31FEF7FD
:109B8000EABAB0F5826F00F05581B0F5C06F00F011
:109B90002981B0F5806F7FF47BAF94F84031029D4E
:109BA0000133DBB2032B00F2AF8142F2107184F873
:109BB000403101FB03F1714B1B88002B40F0A28167
:109BC00001316F4B1B78DB076E4B1B8848BF04319C
:109BD000DF0748BF0A31980748BF14311A0648BF4B
:109BE0002831DF0548BF2831580748BF64311A07BC
:109BF00048BFC8319F0548BF01F5C871980648BFE6
:109C000001F57A71DA0648BF01F5FA615F0648BFCF
:109C100001F57A614FF4806028F020FA002384F87F
:109C20002F31FEF798BAB0F5046F1CD0B0F5116F64
:109C300056D0B0F5036F7FF42BAF3EE74E4B029D3D
:109C400090469A6B998A642303FB02F393FBF1F12C
:109C500028F004FA84F82F81FEF77DBA464B029D66
:109C600090461A6CEEE7484B029DB3F9041001EBE5
:109C700081019046490028F0F1F984F82F81FEF720
:109C80006ABA4FF0010184F82E1184F83031A4F83B
:109C90003A2181E699F80620002A3FF4F9AE3B4BC1
:109CA0003B491B68029D81FB0321DB17C3EBA1012C
:109CB0004FF4007028F0D2F9002384F82F31FEF71A
:109CC0004ABA0A6852077FF5E3AE00214FF4887064
:109CD000029D28F0C3F9002384F82F31FEF73BBA28
:109CE00099F80520002A3FF4D3AE2A4A10780028BC
:109CF0003FF4CEAE284B029D1B8803EB8303590033
:109D000091FBF0F14FF4116028F0A8F9002384F8DA
:109D10002F31FEF720BA0A6895067FF5B9AE9AF89A
:109D2000002090077FF5B4AE1CF0010F029D104F8C
:109D3000104900F068847A6882EAE273A3EBE27368
:109D400003EB5303A1FB0331C908002AACBF41F068
:109D5000004141F040414FF4006028F07FF90023BA
:109D600084F82F31FEF7F7B984AC0308986E002011
:109D7000A06E00201F85EB512C6E0020006100209A
:109D80005C5B0020D26000207C6E0020646C0020B0
:109D900067666666E65B0020D05B00209C6E002054
:109DA000846E002099F80520002A3FF471AEC64A5F
:109DB000107800283FF46CAEC44B029D5B7B002BF7
:109DC00000F08184C24B1B8893FBF0F000EB800015
:109DD00041004FF4047028F041F9002384F82F313A
:109DE000FEF7B9B999F80620002A3FF451AEB94BF5
:109DF000029D99684FF4C06028F030F9002384F880
:109E00002F31FEF7A8B90D68AD067FF541AE9AF87F
:109E100000C01CF0020F3FF43BAEAF4F029D3B89E8
:109E20006421904601FB03F128F018F984F82F8192
:109E3000FEF791B90A68900640F10181A74BA64F41
:109E40001878397D029D00F00203002B0CBF00231F
:109E50004FF47A7340F6B83208BF4FF4FA6210F04C
:109E6000010F18BF134619444FF4826028F0F6F82A
:109E7000002384F82F31FEF76EB9B4F83A21C2F10D
:109E8000FF0293427FF484AD4FF0010384F83D312B
:109E90007EE54FF0010384F83C317DE50EF0BEFB1A
:109EA0008F4B1B68C01A40F6B833984200F25881B5
:109EB000DFF858A29AF804303A2B00F0C78200234A
:109EC00088F80030FEF766B9D8F800000CF014FAF4
:109ED00000287FF45DAD4FF0010384F82F315BE57E
:109EE0000023029D84F82F31FEF735B9C4F82031E4
:109EF00084F81831DFF8188228F0FEF894F824313D
:109F0000FEF7FDB802315CE6012384F8403142F2ED
:109F1000107150E67349029D062027F089FE002348
:109F200084F83E0184F82F31FEF715B9013B84F81F
:109F30005731FEF789BC013B84F85631FEF763BB0D
:109F4000013B84F85A31FEF788BF08F1FF3884F8E6
:109F50005F81FFF7BFBA0CF1FF3C84F85EC1FFF7E9
:109F600062B8614B1B88D80513D4D90600F17B83F6
:109F70009A0600F1DA83580600F1DC83190700F134
:109F8000DB83DA0700F1EC8313F0020F0CBF042728
:109F90000C27564B564A1B78D27803F001030AB1BE
:109FA00043F002035320039328F01EF8484A128816
:109FB00002EB820202EB8202900080B227F0F8FFEF
:109FC000002027F0F5FF4B4A4B491288D8F80000D3
:109FD000C2EBC212520081FB023111444FEAE27A15
:109FE000CAEB612A5FFA8AFA51460CF089F999F8AE
:109FF0000020039BD8F800001F438AEA020A0021D0
:10A0000089F800A00CF07CF93946D8F800000CF073
:10A0100077F999F80030D8F800007B40DBB2194698
:10A0200089F800300CF06CF994F848A1FFF7D0BA29
:10A0300032493A2027F0FCFD2870FEF7C1B8304ABB
:10A040001268120600F1F782204A127B002A3FF4C0
:10A050001FAD94F84111029D032900F28383DFE8CC
:10A0600001F059281902274B1B6859799A79DB7935
:10A0700001F1407101EB022101EB0341002384F85F
:10A0800041314FF4826027F0E9FF002384F82F313B
:10A09000FEF761B81C4B1A68137A507992781B044A
:10A0A00003EB002313444A1C84F8412103EB0161B4
:10A0B000E7E7154B1A68D379107952781B0403EB44
:10A0C00000231344EFE700BFE65B0020D85B0020CD
:10A0D000D05B0020646C0020A06E00209C6E0020ED
:10A0E0006437002055200308D26000205C5B00200C
:10A0F000DC600020D06000200308208079D80208AE
:10A100002C6A0020989E0020305C00204C370020F4
:10A11000246E0020BA4B1A689379D07812781B0409
:10A1200003EB00231344BEE72D22DA76FFF7FABBD8
:10A13000B44B31681B78C4F81411013B012B3FF676
:10A1400000AB1021022391701371FFF7FABA029D40
:10A15000FEF701B827F0C0FF01233B70FDF7A0BF59
:10A16000A94AB2F84A3100210133A2F84A3188F8ED
:10A170000010FEF70FB8A54EA54B00930024A6F1E2
:10A180003F01A44BA44A089106F8404CA349099604
:10A190000AA801F013FE089E731C08933470089BF4
:10A1A0002922591C08911A70089BEA22591C08910F
:10A1B0001A70089BC822591C08910AA81A702DF021
:10A1C0000FFB471C0AA93A4608982EF027FA089A6E
:10A1D000D31901330893D455089B5A1C08921C705C
:10A1E000089B5A1C08921C70089B5A1C08921C70F1
:10A1F000089B5A1C08921C70089B5A1C08921C70E1
:10A20000089B5A1C08921C70089B5A1C08921C70D0
:10A21000089B5A1C08921C70089B5A1C08921C70C0
:10A22000089B5A1C08921C70089B5A1C08921C70B0
:10A23000089BFF22591C08911A70089B012299184B
:10A2400012A808911A7050F8283D9B1B337023F018
:10A25000E3FA2C70FDF7B4BFDFED717AB0EE677AE8
:10A26000FEF7FEBE884689460846049105918E4653
:10A2700006910391FEF7FAB9644A6A4B0B9212AE4B
:10A28000A2F13D0046F8200D1988674FA2F1400366
:10A2900000204FF00A0E02F8400C082283F801E07B
:10A2A00030469A7001F08CFC3B686049DA1781FBFC
:10A2B0000313C2EBA30399B2304601F081FC12F004
:10A2C00015F9BF680A9B3A0C591C0A911A700A9B2F
:10A2D0003A0A591C0A911A700A9B5A1C0A921F705A
:10A2E0000A9B5A1C0A921870304623F095FAFEF722
:10A2F0001CB84F4F9FED4F8AB7F9022043480B908F
:10A3000007EE902AF8EEE77A12AE67EE887AA0F1AF
:10A310003D01FDEEE77A46F8201D00F8403C082399
:10A32000CDED027A00F83F3C1E23BDF8081000F87E
:10A330003E3C304601F044FCB7F9003007EE903A5D
:10A34000F8EEE77A304667EE887AFDEEE77ACDEDF3
:10A35000027ABDF8081001F033FCB7F9043007EEBB
:10A36000903AF8EEE77A304667EE887AFDEEE77AC3
:10A37000CDED027ABDF8081001F022FC304623F042
:10A380004BFAFDF7CFBF2C4A204B12680B93A3F179
:10A390004007002103F8401C2123D100BB7040F18D
:10A3A000B88126490326264B1B885A0500F1A68151
:10A3B000D80700F1BC8103F00203224A002B1CBF26
:10A3C00003261146DFF88080324640462EF026F9FB
:10A3D00006EB080312A80133A8F1020140F8203D62
:10A3E00000225B1A06F808207B7023F015FAFDF7AF
:10A3F0009FBFC4F81CB187F80090FDF751BE00BFA5
:10A40000305C0020D8600020B81E00205061002081
:10A41000225C002008DB030810DB03081CDB0308B8
:10A4200000000000D05B0020646C00206766666658
:10A430007C6E002058A08B4168650020F4DA030888
:10A44000D260002004DB0308136100209AF8024068
:10A45000C4B1013CE4B2013454445146002211F825
:10A46000013B534083EA0313DBB2120ADF0042EAE6
:10A4700003228C4287EA131382EA0302EFD1002AF7
:10A480007FF41DADBC4ABD4FBD4B1288BD4CFA6177
:10A49000DFF824931A68FA629B68B4F84A21F866D8
:10A4A0000021FB64D9F80000F963FA650BF042FC67
:10A4B000029000287DF469AE0221D9F800000BF06B
:10A4C00007FF94F84C319AF803200392642B4FF065
:10A4D000040287F8742040F0738194F84D31072B03
:10A4E00004BF9DF8083084F84D3194F84D3106933F
:10A4F00007EB031ADAF80410029108462DF070F900
:10A50000DAF8081005915FFA80FA08462DF068F92C
:10A51000C0B204900AEB0002069B9B48029902908D
:10A520000832C27123F00F0286468272049803F04B
:10A530000F0300EBCA008EF80D3052468EF80E0065
:10A540000EF10F002EF06AF8904B049A05990AF16B
:10A55000090018442EF062F80298C37903F1010A49
:10A56000CBB1013B5FFA83FC0CF1080CDFF84CE245
:10A5700084440023073010F8011B59408B00CA089F
:10A5800083EA410302F018024B404EFA02F25340B4
:10A590008445DBB2EFD17D4A03980AF802302AF0F5
:10A5A00013FA94F84D310022013384F84D3184F8C8
:10A5B0004C21029BDDF808A09B785BB11AF80510CE
:10A5C000D9F800000BF09CFE01359AF80230EDB28C
:10A5D000AB42F3D894F84C310322013384F84C3168
:10A5E00087F8742088F80020FFF7A2B94FF0010A1D
:10A5F000FEF7B8BF0221D8F800000BF069FE94F80E
:10A600002431FDF77CBD3A6882EAE273A3EBE27382
:10A6100003EB5303A1FB0331C908002AB8BF41F083
:10A620008041FFF798BB5A49881F27F0A5FB84F8A3
:10A630003E01FFF721BA10230027042218460AA979
:10A64000029D8DF828308DF829208DF82A708DF81C
:10A650002B708DF82C708DF82D7027F0DFFC84F8AE
:10A660002F71FDF778BD342793E44A4AD278002A47
:10A670000CBF4FF0040C4FF0050CFEF7F6BD0123A4
:10A68000D8F800003B700BF02FFE0746D8F800000A
:10A690000BF02AFE7B067DF403AD8A284ED08E286F
:10A6A0007DF4FEAC94F81831002B7DF416AD3A4BD6
:10A6B000C4F820312D2384F82431FDF7F8BC4FF085
:10A6C0000108FEF7DBB82C4B1888FFF77FBB2A493F
:10A6D0009A790B8803EB830303EB83034FEA830828
:10A6E0001FFA88F8002A00F01081254B1B680FFA2A
:10A6F00083FA11F0FBFE40B2FDF7C0BE03262749E6
:10A7000060E6984699461846049305930393FDF72F
:10A71000ADBF234B234A1B68234903F48003002B5E
:10A7200016BF1146042603263DE6242731E41F49BF
:10A73000042647E610272CE420272AE41C4B1B683C
:10A740009F067DF5ADAC94F81831002B7DF4C5ACB7
:10A75000184BC4F820312D2384F82431FDF7A7BC11
:10A76000082716E44B1CDBB2042B84F841314FEA76
:10A7700001613FF483AC84E4D05B00200000002042
:10A78000646C0020B81E00204092002046920020F9
:10A79000F01F0020DC600020D0610020F8DA030800
:10A7A0002C6A0020F4DA0308ECDA0308FCDA030868
:10A7B000986E0020FC610020EC3700200007090E95
:10A7C00097F875A05B4904951AF00F0F04BF0AF1C2
:10A7D000010A5FFA8AFABAF1070F28BF4FF0010A9F
:10A7E0004FEA0A1C07EB0C03187C534B02930A1820
:10A7F000002392F82410504A93725FFA8CF31A46A1
:10A800004E4B964607EB0C024EEA000001291870E9
:10A81000D26803F101000CD90239C9B28D1C1D4464
:10A82000034603F8012BAB424FEA1222F9D1013162
:10A830000844BC4422F060030AF1010A9CF811208C
:10A840005FFA8AFA1343BAF1080F037000F10103AB
:10A8500040D04FEA0A1C07EB0C01384A087C354906
:10A8600001449A1A91F8241055180EF1100E132D68
:10A870005FFA8EFEC6DD049D0298DFF8CCE0D2B20E
:10A88000931DDBB243F04001C17103F1010CCBB168
:10A890000532D3B20833C31804930EF1010000232C
:10A8A00010F8011B59408B0083EA4103CA084B4052
:10A8B000234902F0180241FA02F25340049A8242FC
:10A8C000DBB2EDD103980CF80E3087F875A02AF0B2
:10A8D0007BF86EE6194A049D9A1ACDE79846994688
:10A8E0001846049305939E460393FDF7BFBE154B90
:10A8F0009046B3F900A06420FDF7C0BD9846994684
:10A90000184604930393FDF7B1BE4FF0FF33EEE614
:10A910000393FDF7ABBE98460393FDF7A7BE984699
:10A9200099460393FDF7A2BE9846994618460393AD
:10A93000FDF79CBE84AC0308409200204D9200209D
:10A940000007090E646C002046920020002870B5B4
:10A950001EDB0928044620DD012303EB83035B0093
:10A96000B0FBF3F2092AF8D87BB10E4EB4FBF3F03A
:10A970000928CCBF57223022A6FB03E5024403FB83
:10A980001044EB0801F8012BF0D100230B7070BDCF
:10A990002D230B7040420131DBE7303001F8010B11
:10A9A000F3E700BFCDCCCCCC884230B44FF00104EB
:10A9B0002ED301FB04F4B0FBF4F58D42F9D284B13F
:10A9C000AAB901E0B0FBF4F5092DCCBF5722302223
:10A9D0002A4404FB150003F8012BB4FBF1F4002C0E
:10A9E000F0D100221A7030BC7047B0FBF4F5092D8D
:10A9F000CCBF372230222A4404FB150003F8012B78
:10AA0000B4FBF1F4002CF0D100221A7030BC704776
:10AA10000546002AEBD1D7E703685A1C026019707B
:10AA2000704700BF2DE9F047089C2578002B804631
:10AA300089460CBF4FF0200A4FF0300A661C35B330
:10AA4000002A29DD334601E0024698B113F8011BC4
:10AA5000501E0029F8D1971E60B13D46013D514678
:10AA60004046C8476B1C002BF8DC257827EAE770C6
:10AA7000013055B1041B29464046C847301916F825
:10AA8000015B002DF7D1BDE8F087BDE8F087002A13
:10AA900004DC2846BDE8F0870020EBE7571EDCE722
:10AAA00083684268D0ED037A00EB8301013393425F
:10AAB00081ED040A836004BF0023836000EB8303FD
:10AAC00093ED047A036870EE277A9A42C0ED037A18
:10AAD00077EEC77AC0ED037A0CDA013307EE103A4D
:10AAE000F8EEC76AB7EE007A87EEA60A036030EE8A
:10AAF000070A704707EE102AB8EEC77A87EE870A72
:10AB0000704700BF90ED057A90ED004AD0ED066ADF
:10AB1000D0ED014AD0ED047A90ED035AD0ED025AFF
:10AB2000A4EE007AB0EE406AB0EE470AB0EE667A64
:10AB3000A6EE247A67EEC07AA0EE457AE6EE257A94
:10AB400080ED057AC0ED067A704700BFD0ED057A3A
:10AB500090ED013AD0ED003AD0ED064A90ED024A70
:10AB600090ED077A90ED035A90ED086AD0ED045A03
:10AB7000C0ED067AF0EE406A27EE830AC0ED056A62
:10AB8000A3EEA60A80ED087AA4EE240AA5EE470AF1
:10AB9000A5EEC60A80ED070A704700BFD0ED007A27
:10ABA00090ED017A30EE670AE7EE007AB0EE670AC0
:10ABB000C0ED007A704700BF704700BF0A44914261
:10ABC00014D030B40139551E41F2210211F8014F61
:10ABD000082380EA042004044CBF82EA40004000BD
:10ABE000013B80B2F7D18D42F0D130BC704700BF3D
:10ABF0004FF40063838270474FF400638382704791
:10AC00004FF40063838270474FF480538382704710
:10AC1000BFF34F8F0549064BCA6802F4E062134345
:10AC2000CB60BFF34F8F00BFFDE700BF00ED00E03A
:10AC30000400FA0570B4037B04681F2B08D9203B7D
:10AC40002021626801FA03F31A421CD170BC7047DC
:10AC50002021226801FA03F31A42F7D0426914490D
:10AC6000582000FB021251685689CD68086829688F
:10AC700021F001012960828992B222EA06028281D2
:10AC8000A36070BC704742690949582000FB02125A
:10AC900051685689CD680868296821F0010129604A
:10ACA000828992B222EA06028281E36070BC704718
:10ACB0000067002030B4094B1C786CB1084A0025AD
:10ACC00002EBC404116893884D62888908320343FB
:10ACD0009BB2A2428B81F5D130BC7047C069002085
:10ACE000C469002010B4037B01681F2B09D9203BE5
:10ACF00020224C6802FA03F31C4214D15DF8044B85
:10AD0000704720220C6802FA03F31C42F6D00C4A6A
:10AD100040680024147002685DF8044B22F00102C0
:10AD200002608B607047064A406800241470026815
:10AD30005DF8044B22F001020260CB60704700BF57
:10AD40007F60002070B5044682B01430E56D0623A4
:10AD50006A464321A847B0B19DF804009DF8006001
:10AD60009DF801109DF802509DF803209DF80530D4
:10AD700041EA062143EA002342EA0522A187E2874D
:10AD8000A4F84030012002B070BD00BF70B5044689
:10AD900082B00830656A06236A463B21A847A8B1FD
:10ADA0009DF804009DF800609DF801109DF8025088
:10ADB0009DF803209DF8053041EA062143EA00236F
:10ADC00042EA0522E18222836383012002B070BD42
:10ADD00050F8043C012280F84520103803B1184790
:10ADE0007047F8B50468C4F30D0405460E4604B375
:10ADF0002F6826F021FD092840F08880454C236902
:10AE000023F440732361236943F4007323612369AE
:10AE100043F0010323613E6026F00EFD23690928FB
:10AE200023F00103236171D12B6804332B600020D0
:10AE3000F8BD394B394A93422BD902F580429342EF
:10AE400026D902F5804293422AD902F580429342E4
:10AE500028D902F58032934226D902F50032934276
:10AE600024D902F50032934222D902F500329342EE
:10AE700020D902F5003293421ED902F58022934276
:10AE80001CD9B3F1016F1BD305200CF0B7FFFBE712
:10AE9000082426F0D1FC092814D04FF0FF30F8BD6B
:10AEA0001024F6E71824F4E72024F2E72824F0E73A
:10AEB0003024EEE73824ECE74024EAE74824E8E7CA
:10AEC0005824E6E7134F3B6923F440733B613B6929
:10AED00043F400733B613B6923F0F8033B613B693A
:10AEE00043F002031C433C613B6943F480333B6104
:10AEF00026F0A2FC3B6923F002033B613B69092871
:10AF000023F0F8033B613FF473AFC6E76FF0010035
:10AF1000F8BD00BF003C024000400008FF3F0008B1
:10AF2000F8B504460D468E180027B54201D12069B8
:10AF3000F8BDE368591CE160234415F8012B1A722F
:10AF40000429F2D1206918B9A1682046FFF749FF0A
:10AF50002061E760E9E700BF014B18680BF0D0B94A
:10AF6000DC96002038B5054600BF084C2368986879
:10AF70000BF0B6FD2368294658680BF013FF2368D1
:10AF800098680BF0B3FD00BF38BD00BF5C97002090
:10AF9000F8B5057B466903681F2D29D9A5F1200462
:10AFA0005F682021A1400F422A4613D01022A24000
:10AFB000D960DA605A68E240D10703D5012202FA6B
:10AFC00004F4DC60044630460BF026F9227B23684B
:10AFD0001F2A20D9A2F1200008215A68814011427D
:10AFE00000D0D9600422596882400A4221D1F8BDBC
:10AFF00020211C68A9400C422A460CD01022AA40ED
:10B0000099609A601A68EA40D207DBD5012202FAF9
:10B0100005F59D60D6E7082118689140014200D0EF
:10B0200099600421186801FA02F2024203D09A6082
:10B03000F8BDDA60F8BDF8BD70B582B00446694667
:10B04000143028F03DFBB0B19DF805009DF801607B
:10B050009DF802109DF803509DF804209DF80630DD
:10B0600041EA062143EA002342EA0522A187E2875A
:10B07000A4F84030012002B070BD00BF38B590F890
:10B08000593003B938BD044618460BF0DFFA0546BF
:10B090000BF054FD01460028F4D1D5B12023E8710E
:10B0A000AB7128460BF064FC2146104B41F8103F71
:10B0B000284628F099FAAB88B3FA83F3C3F11F034B
:10B0C000012212FA03F3DDD009490A6813430B6029
:10B0D00038BD29460BF04CFC2146044B41F8103F8B
:10B0E0002846BDE8384028F07FBA00BFD1AD00083F
:10B0F000003C014038B5044600F11405FFF7BEFFDF
:10B10000236E80226B212846984764200DF02CFB8B
:10B11000236E072268212846984764200DF024FBFF
:10B12000236E00226B212846984764200DF01CFBFB
:10B13000236E01226B21284698470F200DF014FB47
:10B1400094F85320236E032A8CBF1A2218221B2145
:10B15000284698470F200DF007FB236E18221C216C
:10B16000284698470F200DF0FFFA236E94F85220DE
:10B170001A21284698470F200DF0F6FA236E94F80E
:10B18000542019212846984764200DF0EDFA236ECB
:10B1900010223721284698470F200DF0E5FA28465F
:10B1A000236E0122382198470F20BDE838400DF06A
:10B1B000DBBA00BF10B58021044680690BF024FE85
:10B1C00001200DF077FA2046FFF794FF10226A2144
:10B1D00004F114000AF010FE64200DF0C5FAA06915
:10B1E00004210BF011FE0120BDE810400DF062BA01
:10B1F00038B5044600F11405FFF740FFA0694FF48D
:10B2000080710BF001FE236E80226B212846984747
:10B2100064200DF0A9FA236E03226821284698477E
:10B2200064200DF0A1FA236E01226B212846984775
:10B230000F200DF099FA94F85320236E032A8CBF47
:10B240001A2218221B21284698470F200DF08CFA4D
:10B25000236E18221C21284698470F200DF084FAEF
:10B26000236E94F852201A21284698470F200DF09B
:10B270007BFA236E94F854201921284698476420BD
:10B280000DF072FA236E10223721284698470F20BE
:10B290000DF06AFA2846236E382101229847A069EA
:10B2A0000821BDE838400BF0AFBD00BFF8B5464EF1
:10B2B0000446FFF7E3FE3778DFB104F114054FF4DD
:10B2C0008071A0690BF0A0FD94F852201A21284645
:10B2D0000AF092FD01200DF0EDF90421A0690BF0B8
:10B2E00093FD2046FFF72EFD94F93E30013362D0E6
:10B2F000F8BD04F114054FF48071A0690BF084FDD2
:10B3000080226B2128460AF077FD96200DF02CFA5A
:10B310000322682128460AF06FFD96200DF024FADA
:10B3200003226B2128460AF067FD0F200DF0C2F9B9
:10B3300010226A2128460AF05FFD0F200DF0BAF9AD
:10B340003A466C2128460AF057FD0F200DF0B2F95D
:10B3500094F85420192128460AF04EFD0F200DF0D4
:10B36000A9F918221B2128460AF046FD0F200DF0EE
:10B37000A1F910221C2128460AF03EFD0F200DF0F5
:10B3800099F91022372128460AF036FD0F200DF0DA
:10B3900091F90122382128460AF02EFD0F200DF0E8
:10B3A00089F90421A0690BF02FFD01200DF082F92D
:10B3B0000123337083E794F93C30013398D10620A0
:10B3C000BDE8F8400CF01ABD7C210020F8B5654CB2
:10B3D0000601A7190546387A28F0E4F83B7A03F00D
:10B3E0001F015B090122032B02FA01F26DD0042B2D
:10B3F00066D0022B5CD0A319013518790BF026F921
:10B40000EDB2074610B11223C5718371A3195879A3
:10B410000BF01CF910B11323C5718371A31998792E
:10B420000BF014F910B11423C5718371A5190A2109
:10B43000EA7938460BF0D0F968790BF007F9EA7928
:10B440000A210BF0C9F9A8790BF000F9EA790A2171
:10B450000BF0C2F9A359444A934247D0434A93425E
:10B4600050D0434A934259D0424A934262D0424A12
:10B4700093426BD0414A93422CD03444227BE2B9B0
:10B4800001200222198801F4415141F445710A4317
:10B4900002431A809A8B22F400621204120C0721D4
:10B4A0009A8319821A8892B242F040021A80F8BD3B
:10B4B000334B596A0A435A629DE700200246E1E78E
:10B4C0002F4B19690A431A6195E72D4B196A0A43F4
:10B4D0001A6290E702F564424FF40010536A43F495
:10B4E0000013536226F0A2F8A359C6E702F584328E
:10B4F0004FF48050536A43F48053536226F096F819
:10B50000A359BAE702F500324FF48040136A43F4BE
:10B510008043136226F092F8A359AEE702F5FE329B
:10B520004FF40040136A43F40043136226F086F898
:10B53000A359A2E702F582324FF40050536A43F454
:10B540000053536226F072F8A35996E702F5684259
:10B550004FF48010536A43F48013536226F066F868
:10B56000A3598AE7286F00200030014000380040CE
:10B57000003C0040003401400050014000540140B4
:10B5800000380240427A02B9704710B50446036899
:10B59000406804F10A0198470023637210BD00BFA0
:10B5A000437A5A1C0344D2B242729972037A93428C
:10B5B00000D802B9704710B504460368406804F12A
:10B5C0000A0198470023637210BD00BF302827D0BE
:10B5D000312827D0322827D0332827D0342827D025
:10B5E000352827D0202827D0212827D0102827D059
:10B5F000112827D0122827D0132827D0142827D085
:10B60000152827D0162805D0172808BF0F2202D0EA
:10B61000002070470E22104B03EB4203587870470E
:10B620000022F8E70122F6E70222F4E70322F2E71C
:10B630000422F0E70522EEE70622ECE70722EAE71C
:10B640000822E8E70922E6E70A22E4E70B22E2E71C
:10B650000C22E0E70D22DEE7D8AC030870B5448881
:10B6600006460D46C4F30B042246002128462FF05F
:10B6700054FA3369094A934209D3094A934206D2DC
:10B68000224628461946BDE870402CF0C7BF23B1BA
:10B6900021462846BDE87040184770BDD405000813
:10B6A000D4060008064B07498B4202D300231846F4
:10B6B00070471A88C2F30B029042F8D01433F3E7B4
:10B6C00088010008D4050008024A136823EA000034
:10B6D00010607047945D0020F8B5174D2B78A32BB0
:10B6E00028D16B78BE2B25D1022229464FF6FF7058
:10B6F000FFF764FA114FAC1C22884AB1A618BE426B
:10B7000018D2052A16D92146FFF758FA3446F3E72E
:10B7100021460222FFF752FA0222A118FFF74EFA41
:10B720000634074B641B1C8041F60F53C31A584262
:10B730005841F8BD0020F8BD004000080080000816
:10B74000F83300202DE9F04FDFF84C914D4F8BB0CE
:10B750000326A7EB09071822002104A82FF0DDF922
:10B76000494BCDF8109005971A69002A04DA474A28
:10B770005A6002F188325A6001228DF82420F322A7
:10B78000DA60434B434C1B88ADF800300222694617
:10B7900004A8FFF7C5FB022269464FF6FF70FFF7CA
:10B7A0000DFADFF8F8A080464FF0000B544539D36E
:10B7B0000AAC002524F8245D0222214604A8FFF7E4
:10B7C000AFFB022221464046FFF7F8F940BAC043DA
:10B7D000ADF80800022202A904A8FFF7A1FB079810
:10B7E00078B106ABC0F10402294618442FF095F950
:10B7F000089818B9069904A8FFF7F3FA00230890EF
:10B8000007939DF82430089A23B11F490B6943F030
:10B8100000430B61013E2DD0002A9CD1FFF75CFF55
:10B8200050B32CE065888DF80DB0C5F30B05AB1D4A
:10B83000ADF808302388C3F30B02ADF80A201B0BC8
:10B84000062202A904A88DF80C30FFF769FB062236
:10B8500002A94046FFF7B2F9616880462A4604A86B
:10B86000FFF75EFB616840462A46FFF7A7F91434EC
:10B8700080469BE7002AD1D005200CF0BFFA0BB020
:10B88000BDE8F08F00800008003C024023016745BE
:10B89000F8AC03088801000800400008D40500083F
:10B8A0000378202B024600F10100F9D0092BF7D0D4
:10B8B0002D2B2CD02B2B03BF5378B7EE000A02465A
:10B8C000B7EE000AA3F13001C8B209289FED467A0D
:10B8D00010D8F2EE046A07EE901AF8EEE77A12F842
:10B8E000013FE7EE267AA3F13001C8B20928B0EE95
:10B8F000677AF0D92E2B4CD003F0DF03452B0BD009
:10B90000F7EE007A67EE276A20EE260A7047537832
:10B91000BFEE000A0246D5E710B451782D2959D060
:10B920002B290ABF9178501C901C0024A1F13003F0
:10B93000092B53D8002303EB830301EB430310F8D7
:10B94000011FA1F13002092AA3F13003F3D9B3F5A5
:10B950009A7F28BF4FF49A73072B42D9DFED236AF1
:10B960001A46F7EE007A083A072A67EEA67AFAD85E
:10B9700003F007032BB1F2EE046A013B67EEA67AEF
:10B98000FBD124B3C7EE276A5DF8044B20EE260AEC
:10B9900070475378A3F13001C8B2092802F10102BF
:10B9A000AAD8F2EE046AF0EE665A07EE901AF8EEA4
:10B9B000E77A12F8013F87EEA66AA3F13001C8B218
:10B9C000092866EEA56A37EE067AEED994E767EEA7
:10B9D000276AD9E7901C91780124A7E7F7EE007A4F
:10B9E000CFE7F7EE007AC5E70000000020BCBE4CB0
:10B9F000B5EEC00ADFED317AF1EE10FACCBF30EED1
:10BA0000270A30EE670ADFED2E7A20EE270A30B5DE
:10BA1000FDEEC07A87B017EE904A054684EAE470DE
:10BA2000002303A9A0EBE47001930093029328F094
:10BA30002DFB002CACBF20232D2303A88DF8003054
:10BA40002BF0CEFE012803A924D002282DD00328F4
:10BA500005BF3023684668468DF801302FF083F823
:10BA600068462BF0BDFE0338C4B22246694628461C
:10BA70002FF0D7F800232B5528462BF0B1FE2E22AD
:10BA8000431C2A540DEB0401E8182FF089F82846CE
:10BA900007B030BD302368468DF801308DF8023094
:10BAA0008DF803302FF05FF8DAE7302368468DF821
:10BAB00001308DF802302FF056F8D1E76F12033ABB
:10BAC00000007A442DE9F041064615460846B6FBCB
:10BAD000F2F43CB905FB1464124B1B5D00F8013B0A
:10BAE000BDE8F081B4FBF2F767B90E4B05FB1747D1
:10BAF00005FB1464DA5D00F8012B1B5D00F8013BC7
:10BB0000BDE8F081B7FBF2F8B8F1000F02D0404673
:10BB1000FFF7D8FF05FB1878024B13F8082000F850
:10BB2000012BE3E788DB030830B402681146531C9D
:10BB3000036011F8024B0160D31C517803609378C5
:10BB4000151D05601B0443EA0123D078234343EA13
:10BB5000006030BC704700BF0368591C1A46016082
:10BB600012F8021B0260587841EA0020704700BFBB
:10BB700003685A1C02601878704700BF38B5044645
:10BB8000006815462CF04AFD22682A44226038BD20
:10BB9000036810B40A0E5C1C04601A7003680A0C77
:10BBA0005C1C04601A7003680A0A5C1C04601A704A
:10BBB00003685A1C026019705DF8044B704700BF9F
:10BBC000036810B40A0A5C1C04601A7003685A1CEB
:10BBD000026019705DF8044B704700BF03685A1C7F
:10BBE000026010B4197003680A0A5C1C04601A70C1
:10BBF00003680A0C5C1C04601A700368090E5A1C66
:10BC0000026019705DF8044B704700BF03685A1C4E
:10BC1000026019700368090A5A1C026019707047A3
:10BC20002DE9F047002488B080460F461E46A14605
:10BC300005AD531C0393117839B3252933D1931CD7
:10BC4000CDF810900393507830284ED04FF0000A72
:10BC5000A0F13003DBB2092B42D96C2819D064283B
:10BC600000F0938024D825281CD063D9582876D09A
:10BC700063281BD131784046B847039A531C03937D
:10BC80001178043601340029D7D1204608B0BDE828
:10BC9000F087039B5A1C03921B78642B7CD02AD814
:10BCA000252B54D1252140460134B847039AC0E7DB
:10BCB000732833D044D975284FD106F1040E30686B
:10BCC0002B4600220A217646FEF76EFE049A009566
:10BCD000534639464046FEF7A5FE039A0444A8E7BA
:10BCE00004AA03A924F0E6FEB7E7D31C03939078D7
:10BCF0004FF0010AACE7732B10D05BD9752B3AD00B
:10BD0000782B96D1A3F15802B2FA82F23068520928
:10BD10002B4610210436FEF747FED7E73368049A16
:10BD20000093394600234046FEF77CFE0436044467
:10BD3000039A7EE70028B9D1204608B0BDE8F08715
:10BD40006E28B3D1039A336804361C6071E72AD990
:10BD5000582BD7D0632B8DD06BE77828A6D1A0F1D4
:10BD60005802B2FA82F2306852092B461021FEF7CF
:10BD70001BFE0436AAE706F1040E30682B460022AB
:10BD80000A217646FEF710FEA0E7331D30682946EB
:10BD90001E46FEF7DBFD99E7331D306829461E4637
:10BDA000FEF7D4FD92E7002B7FF443AF204608B0A6
:10BDB000BDE8F0876E2BC6D03BE700BF0EB400B5E0
:10BDC00084B005AB019053F8042B0649039301A8F6
:10BDD000FFF726FF019B00221A7004B05DF804EB08
:10BDE00003B0704719AA00080FB430B583B006AB92
:10BDF0000A490B4853F8042B096800680193FFF7C0
:10BE00000FFF084C054620680AF066FA0028FAD0B1
:10BE1000284603B0BDE8304004B070470833002026
:10BE20000C330020DC960020DFED2B7AB4EEE70A1D
:10BE3000F1EE10FA4ADDDFED296A9FED297A01E083
:10BE4000B0EE670AB4EEC70AF1EE10FA70EE667A49
:10BE5000F6DC9FED247AF4EEC77AF1EE10FA38D5CD
:10BE6000DFED1E6A9FED207A01E0F0EE407AF4EEFD
:10BE7000C77AF1EE10FA37EEA60AF6D4DFED1B7A98
:10BE8000B4EEE70AF1EE10FA14DDDFED137A37EEC7
:10BE9000C00A60EE006A9FED166A9FED167ADFED2C
:10BEA000167AA6EE867A20EE266AE6EE877AA6EE67
:10BEB000270A7047DFED117AB4EEE70AF1EE10FAC7
:10BEC00044BFDFED087A37EEC00AE2E7F0EE407AD1
:10BED000BFE7B0EE670AD1E7DB0F4940DB0FC9408F
:10BEE000E4CB1641DB0F49C0E4CB16C1DB0FC93FE1
:10BEF00092E741B99730083C15A82ABEDB0FC9BFAD
:10BF000009B909E0194690FBF1F301FB1303084658
:10BF1000002BF7D1084670470146FBE7F0EEC07AE8
:10BF2000B0EEE07AB4EEE77AF1EE10FAB4BFB0EE1C
:10BF3000676AB0EE476AB5EE406AF1EE10FA46D095
:10BF4000B4EEE77AF1EE10FA8CBFF0EE675AF0EE3D
:10BF5000475AC5EE866A9FED1F3A9FED1F6A9FED17
:10BF60001F4A9FED1F5ADFED1F3ADFED1F4ADFED3D
:10BF70001F5AA6EEC36AE6EEA34AA6EE864AB7EEBD
:10BF8000006AA6EE845AA6EEA46AE6EE855AC5EECD
:10BF9000866AB4EEE77AF1EE10FA48BFDFED147A64
:10BFA000F5EEC00A48BF77EEE66AF1EE10FA48BF38
:10BFB000DFED107AB5EEC00A48BF77EEE66AF1EE23
:10BFC00010FA48BFF1EE666AB0EE660A7047DFED20
:10BFD000076ADEE739094E3DE3B59E3E88FA163E14
:10BFE00045FE7F3F99FB243F69A2163EA7DFA83498
:10BFF000DB0FC93FDB0F4940DFED317A30EE277AA6
:10C00000FDEEC76A16EE903A2033402B02D99FED21
:10C010002D0A7047B4EEE70AF1EE10FA4DDD9FED00
:10C020002A6ADFED2A6A01E0B0EE677AB4EEE67ABA
:10C03000F1EE10FA77EE467AF6DC9FED257AF4EE13
:10C04000C77AF1EE10FA35D5DFED1F6A9FED217A40
:10C0500001E0F0EE407AF4EEC77AF1EE10FA37EE36
:10C06000A60AF6D4DFED167AB4EEE70AF1EE10FA7E
:10C070001BDCDFED197AB4EEE70AF1EE10FA44BFEB
:10C08000DFED137A37EEC00A60EE006A9FED136AA7
:10C090009FED137ADFED137AA6EE867A20EE266AFC
:10C0A000E6EE877AA6EE270A7047DFED0F7A37EEC5
:10C0B000C00AE9E7B0EE670AD4E7F0EE477ABCE7DA
:10C0C000DB0FC93F00000000DB0FC940E4CB164185
:10C0D000DB0F49C0E4CB16C1DB0FC9BF92E741B902
:10C0E0009730083C15A82ABEDB0F4940FDEEC07A08
:10C0F00017EE903A2033402B51D8DFED2D7AB4EE75
:10C10000E70AF1EE10FA50DDDFED2A6A9FED2A7A98
:10C1100001E0B0EE670AB4EEC70AF1EE10FA70EE75
:10C12000667AF6DC9FED257AF4EEC77AF1EE10FA26
:10C1300038D5DFED206A9FED227A01E0F0EE407AFB
:10C14000F4EEC77AF1EE10FA37EEA60AF6D4DFED78
:10C150001D7AB4EEE70AF1EE10FA1BDCDFED1A7A75
:10C16000B4EEE70AF1EE10FA44BFDFED147A37EED1
:10C17000C00A60EE006A9FED156A9FED157ADFED4B
:10C18000157AA6EE867A20EE266AE6EE877AA6EE85
:10C19000270A7047DFED067A37EEC00AE9E79FED20
:10C1A0000E0A7047B0EE670AD1E7F0EE407AB9E7C1
:10C1B000DB0F4940DB0FC940E4CB1641DB0F49C020
:10C1C000E4CB16C1DB0FC93FDB0FC9BF92E741B912
:10C1D0009730083C15A82ABE0000000010B507EEF5
:10C1E000901A2DED028BB8EE678ADFED217A28EEEA
:10C1F000008A044628EE278AB0EE480A2CF0CEFBCF
:10C20000F0EE408AB0EE480A2CF02AFBF7EE007AF6
:10C210009FED187AF0EE675AE8EE875A0023A36183
:10C22000B0EE676AC7EEA56A63612362E361A8EEB8
:10C23000C76ABDEC028B77EEC07AB6EE007AF8EEF4
:10C24000005A27EE877A20EE250A27EE267A26EE78
:10C25000266A67EEA67A20EE260A84ED046AC4ED0B
:10C26000017A84ED007A84ED027A84ED030A10BD30
:10C2700027D4D236F304353F10B44C09012250F8CC
:10C28000243001F01F0102FA01F10B4340F8243081
:10C290005DF8044B704700BF4B0901F01F0150F8D7
:10C2A0002320012303FA01F1114214BF1846002094
:10C2B000704700BF074A084B10781B78074A834233
:10C2C00096BFC31AC3F180030020126818441044BB
:10C2D000704700BFE06300205C630020E439002069
:10C2E000064A074B10781B7883428ABFC3F180034C
:10C2F000C01AC018C0F17F00704700BFE063002083
:10C300005C63002030B5144C237883B01BB9012046
:10C31000237003B030BD052200238DF800208DF876
:10C32000013000BF0D4D2B6898680AF0D9FB2B68CF
:10C3300001AA6946586827F091F82B6898680AF0B6
:10C34000D5FB00BF9DF8053003F0010383F0010029
:10C35000237003B030BD00BF6E9700205C970020B3
:10C3600070B5064C0646256803E023685B1BB342A4
:10C3700003D8FFF7C7FF0028F7D070BD8C790020E5
:10C380002DE9F04F89B0B2F1000A029004910393B5
:10C3900040F3B0800B46002201EB8A0153F8040BF6
:10C3A0008B420244FAD1039B0592002B00F09A8045
:10C3B000059B002B6AD0544B059A1B68DFF85C91F3
:10C3C00000920099DAB25118B1F5807F8CBFC2F5A6
:10C3D0008072009A01924D4A92689A426DD9190C66
:10C3E0001A0A4FF0020406208DF81F308DF81E2027
:10C3F0008DF81D108DF81C40FFF7B2FF0620FEF7E8
:10C40000B1FD434A0123137000BFD9F8003098688A
:10C410000AF066FBD9F8003007A95868002226F018
:10C42000D5FF0024049D029E019FA34629684FEA80
:10C43000840800220B46013471B1B9422AD2D9F8DE
:10C440000000316840680AF00BFD2A683368134425
:10C450003360BF1AC5F800B0A24505F1040506F126
:10C460000406E3D1D9F8003098680AF03FFB00BF1A
:10C47000254B019900981B68421A0092224A0B44EE
:10C480001360039A32B3009A002A9AD1059809B032
:10C49000BDE8F08F029CD9F8003054F808105868B5
:10C4A00000223B460AF0DCFC54F808202B683A4492
:10C4B000DF1B44F808202F60D4E70598009C15493D
:10C4C000154A001B0590059800230B70137009B0E6
:10C4D000BDE8F08F059B009A9B1A0593059809B05B
:10C4E000BDE8F08FFFF70EFF00287FF461AF039BDC
:10C4F0000593CBE7039C1CB9FFF704FF0594C5E740
:10C5000000230593C2E700BFE4390020D01C0020BF
:10C510006E970020E06300205C6300205C970020A1
:10C5200070B5104D104E2B7831788B4284B016D0F8
:10C530000E4A03921A4402928CBF0C46CA1A04A9EE
:10C540008CBFC3F180020024012341F8102D02A802
:10C5500002220194FFF714FF002333702B7004B004
:10C5600070BD00BF5C630020E063002060630020BA
:10C5700070B5194C194D23782978994284B027D089
:10C58000174A03921A44029234BF0E46CA1A04A9EB
:10C5900034BFC3F180020026002341F8102D02A809
:10C5A00002220196FFF7ECFE23781844C0B203067E
:10C5B0002B7848BF80F080008342207002D000209A
:10C5C00004B070BD002301202B70237004B070BD37
:10C5D000012004B070BD00BF5C630020E063002058
:10C5E0006063002008B545F20820FFF7B9FE062079
:10C5F000FEF7B8FC064B0122C7201A70FEF7B2FC0A
:10C6000004480549054A002303700B70136008BDF8
:10C610006E970020E06300205C630020E439002076
:10C620002DE9F04182B00346060C050A03240620DA
:10C630008DF80730884617468DF805608DF806504E
:10C640008DF80440FFF78CFEC0B100BF0D4C23688D
:10C6500098680AF045FA236801A95868002226F074
:10C66000B5FE23684246002158683B460AF0F8FBB5
:10C67000236898680AF03AFA00BF384602B0BDE86D
:10C68000F08100BF5C970020F0B5124B9D6885B02B
:10C690000DB905B0F0BDED0A14D0002704AE7C1929
:10C6A0006410E00210226946FFF7BAFF0F2809DD87
:10C6B0006B4653F8042B01320AD1B342F9D1254617
:10C6C000AF42ECDBFFF72CFF034BED021D60E0E710
:10C6D000671CF5E7D01C0020E43900200C4B984281
:10C6E00013D0A3F5806398420FD003F5804398429E
:10C6F0000BD003F58063984207D003F5806398421E
:10C7000003D0044B186840087047024B1868704704
:10C71000000401405C9E0020F0B5774B774A87B05B
:10C720001968914200AF00F0DB800023744A3B603F
:10C730007B60136843F48033136003E03B68B3F518
:10C74000A04F09D0136803F400337B603B680133CA
:10C750003B607B68002BF1D0694B1B6813F40033FE
:10C7600018BF01237B607B68012B7BD0654D644B38
:10C77000654AEA606549586F654A0860AA605E6B61
:10C78000644C654A654826F080065E635E6F46F03D
:10C7900080765E67196B0C431C63596B5963996B08
:10C7A0009963196C41F05B5141F47B1141F41F61B5
:10C7B00041F00F011964596C07F118040A4348F25B
:10C7C000FF715A6444F8101D002621460123FB73B3
:10C7D0003E737E73BE7324F007FE21464FF6FF734F
:10C7E0004F48BB6024F000FE4FF6FF7321464D48D2
:10C7F000BB6024F0F9FD21464B4824F0F5FD2146AD
:10C800004A4824F0F1FD2146494824F0EDFD214637
:10C81000484824F0E9FD2146474824F0E5FD21463B
:10C82000464824F0E1FD204624F0BEFF444B454C31
:10C830001B68BA6844484549A4FB03439B09A0FB15
:10C840000202013B920CB3F1807F0A6007D2404A9A
:10C85000F0200721536085F82300966011601C3793
:10C86000BD46F0BD264B3B4D1A6C3B4842F0805212
:10C870001A642C684268816844F440442C609C68C7
:10C880009C609C6844F400449C609C6844F4A05400
:10C890009C600068120642EA801242F48002490855
:10C8A00042F00802013942EA01425A601A6842F035
:10C8B00080721A601A689201FCD52849104A40F229
:10C8C00005700860996821F003019960996841F04A
:10C8D00002019960936803F00C03082BFAD145E735
:10C8E00000221A6062B61E4B1B6883F308881D4B3A
:10C8F0001B689847FEE700BFFCFF0120EFBEADDEDE
:10C900000038024000ED00E00005FA05BC6B002095
:10C9100000000008FF916700335F0700000002403D
:10C920000004024000080240000C024000100240D7
:10C930000014024000180240001C02400020024087
:10C940005C9E0020D34D621083DE1B439079002053
:10C9500010E000E00070004078000020003C024041
:10C960000000FF1F0400FF1F08B5054B1B6803B143
:10C970009847044B044A1A6072B6FEF749F900BFA3
:10C980004C3A0020FCFF0120EFBEADDE08B5034BA2
:10C990001B6803B1984772B6FEF73AF94C3A00208B
:10C9A000084B10B507281B68C8BF143818440C463C
:10C9B000007D09F04BFE20B12146BDE810400AF091
:10C9C0009BB810BD3479002038B50D4B07281B6883
:10C9D000CCBFA0F11404044623440546187D09F099
:10C9E00035FE58B101342722C4718271012109F04A
:10C9F000BFFF28460021BDE83840D1E738BD00BF61
:10CA00003479002070B50F4C0F4DC0EBC00004EB23
:10CA10008004286B26693043286382B09209667BC4
:10CA2000A1600025012101A863618DF804608DF8E3
:10CA300005208DF806508DF807101EF05BF802B047
:10CA400070BD00BF101B002000380240074BC0EB38
:10CA5000C00030B403EB8000054C0569236B2B4309
:10CA600023630176427630BC704700BF101B002064
:10CA7000003802402DE9F04F5B4C54F8204083B061
:10CA8000002C00F0AC80E66D002E00F0AA809046ED
:10CA9000564A35692260994604F2622204F1620323
:10CAA0006361A2614FF400737268A1600746E3609E
:10CAB00023616265A246B5B14D4B00205A6895428C
:10CAC00003F11C0376D001301028F7D100207A1C26
:10CAD000D2B20C21FFF7BAFF636DB16832692263ED
:10CAE0000433A1632365F068E8B1414B00215A6823
:10CAF000904203F11C035BD001311029F7D10025CE
:10CB00007A1CD2B20B212846FFF7A0FF2346F27F02
:10CB100038492846FFF776FF636DB168F2686263B3
:10CB20000433E163E36494F8610009F08FFD054686
:10CB300094F8600009F08AFD8346307F00284BD1CD
:10CB400019F0080F38D118F0020F09D045B10B22A7
:10CB50007B1CAA71EB712846727F222109F03CFEF2
:10CB600018F0010F15D1A36B7BB996F82020B17F87
:10CB70008DF8063001A8930901228DF805308DF853
:10CB800004108DF807201DF0B5FF504603B0BDE836
:10CB9000F08FBBF1000FE6D001370C238BF8077044
:10CBA0008BF806305846727F222109F015FEDAE72D
:10CBB000CDB2A5E7C0B28AE70137FFB215B10B23AA
:10CBC000EF71AB7119F0100F284614BF022112212A
:10CBD000727F09F001FEC6E726F0E4FCB0E7A2464A
:10CBE000D3E7B246D1E700BF14330020FCAC030802
:10CBF000101B002091AF00080348D0F8AC3113B1EE
:10CC000000F5D27018477047101B00200348D0F879
:10CC1000903113B100F5C47018477047101B002005
:10CC20000348D0F8743113B100F5B6701847704757
:10CC3000101B00200348D0F8583113B100F5A8703C
:10CC400018477047101B00200348D0F83C3113B13F
:10CC500000F59A7018477047101B00200348D0F861
:10CC6000203113B100F58C7018477047101B00205D
:10CC70000348D0F804310BB1FC301847704700BFAF
:10CC8000101B00200348D0F8E8300BB1E030184703
:10CC9000704700BF101B00200348D0F8CC300BB108
:10CCA000C4301847704700BF101B00200348D0F85D
:10CCB000B0300BB1A8301847704700BF101B0020E0
:10CCC0000348D0F894300BB18C301847704700BF40
:10CCD000101B00200248836F0BB17030184770475B
:10CCE000101B00200248C36D0BB154301847704729
:10CCF000101B00200248036C0BB1383018477047F6
:10CD0000101B00200248436A0BB11C3018477047C3
:10CD1000101B00200248836803B11847704700BF0A
:10CD2000101B00201549164B16480A6810B48C6871
:10CD30001549B2FBF4F203FB02F30360D1F888203B
:10CD4000124B134C42F47002C1F888201A6800207C
:10CD500042F001021A6098601A6822F0847222F48C
:10CD600080321A605C601A684FF0006422F48022FE
:10CD70001A60D8608C605DF8044B70477800002022
:10CD800040420F005C9E002000ED00E000380240B1
:10CD900010300024044B4FF4F0700A21022283E883
:10CDA0000700FFF7BFBF00BF780000202DE9F04F5C
:10CDB00095B0B0F908500D81EDB2442D00AF0C468E
:10CDC000904600F04584064643D9812D00F07D83CE
:10CDD00000F29880542D00F0CC8040F2D6806E2D69
:10CDE00000F00484802D40F0D380764B93F800A0AF
:10CDF0000AF1020A1AF0FF0A00F09780724BDFF87E
:10CE0000F481724EDFF8F0B19A4403F101090A256A
:10CE100016E0322D01F0C582A5F13C00C0B2132806
:10CE200041F2C98200232268511C216015702268DA
:10CE3000D14502F101012160137076D019F8015B30
:10CE40000A2DE6D1BBF80030FF2BA8BFFF23DBB2D1
:10CE5000E9E7052D00F0EA8320D8022D00F081805B
:10CE600040F21283032D00F0B783042D40F0908030
:10CE7000574920462A46FEF781FE00212046FEF74C
:10CE8000C5FE22680021531C0125236028462B463D
:10CE9000543711706381BD46BDE8F08F242D5ED0FC
:10CEA00040F2A882282D00F05983382D70D10A68ED
:10CEB000484B0125511C216015702268052150192D
:10CEC0002060117022680A215019206011702268B8
:10CED00000215019206011702268197850192060C3
:10CEE0001170226859785019206011702268997861
:10CEF000531923602B461170284654376381BD4671
:10CF0000BDE8F08FA02D18D040F29382B82D00F02C
:10CF10006183FE2D3CD1304D05F1080635F8021B2A
:10CF20002046FEF773FEB542F8D101252B46284670
:10CF300054376381BD46BDE8F08F284B0846196819
:10CF4000FEF74CFE264B20461968FEF747FE254BA0
:10CF5000196820460125FEF741FE2B46E7E7224BE4
:10CF6000F6E70422214920460125FEF707FE2B465D
:10CF7000C2E70B6800215A1C226019702268012543
:10CF8000531923602B461170B6E7522D3FF479AF49
:10CF9000214628460BF01AFD03460028C5D1742D02
:10CFA00000F08582772D29D13268716891421EBFC9
:10CFB000531C336011780E4A08BF1946204628F0EA
:10CFC0000DFEB2E7CD5A002024AD03085425002001
:10CFD000225C0020175C0020F05A0020107AFF1F0E
:10CFE000147AFF1F187AFF1F945D0020B0DB03083E
:10CFF000E14E0308676666667C250020F52D01F08A
:10D000003383762D00F02C83472D01F06A82292D81
:10D01000336801F04D82392D01F00082212D01F09D
:10D02000278271680B3DCA1AEF2D00F2458501A0D9
:10D0300050F825F017E30008B9DA0008B9DA00085B
:10D04000B9DA0008B9DA0008B9DA0008B9DA000874
:10D05000B9DA0008B9DA0008B9DA0008B9DA000864
:10D06000B9DA0008B9DA0008B9DA0008B9DA000854
:10D07000B9DA0008B9DA0008B9DA0008B9DA000844
:10D08000B9DA0008B9DA0008B9DA0008B9DA000834
:10D09000B9DA00084FE30008B9DA0008F5E2000841
:10D0A000B9DA0008CBE20008B9DA0008B9DA0008FA
:10D0B000B9DA0008A3E20008B9DA00082DE2000896
:10D0C000B9DA0008FBE10008B9DA0008D5E1000888
:10D0D000B9DA0008C3E10008B9DA00086BE100081A
:10D0E000B9DA000819E10008B9DA0008B9DA00086D
:10D0F000B9DA0008B9DA00082BCF0008B9DA00085D
:10D10000CBE00008B9DA0008B9DA0008B1E000089D
:10D11000B9DA000801D70008B9DA0008B9DA00085E
:10D12000B9DA0008B9DA0008A5E00008B9DA0008A1
:10D13000B9DA0008B9DA000865E00008B9DA0008D1
:10D14000D9DF0008B9DA0008B9DA000827E00008DA
:10D15000B9DA0008B9DA0008B9DA0008B9DA000863
:10D16000B9DA0008B9DA0008B9DA000805DF000802
:10D17000B9DA000883DE0008B9DA0008C9DD000862
:10D18000B9DA0008CDDC0008B9DA0008A5DC00082F
:10D1900087DC0008B9DA0008B9DA0008B9DA000853
:10D1A000B9DA0008B9DA0008B9DA0008B9DA000813
:10D1B000B9DA0008B9DA0008B9DA0008B9DA000803
:10D1C000B9DA0008B9DA0008B9DA0008B9DA0008F3
:10D1D000B9DA0008B9DA0008B9DA0008B9DA0008E3
:10D1E000B9DA0008B9DA0008B9DA0008B9DA0008D3
:10D1F000B9DA0008B9DA0008B9DA0008B9DA0008C3
:10D20000B9DA0008B9DA0008B9DA0008B9DA0008B2
:10D21000B9DA0008B9DA0008B9DA0008B9DA0008A2
:10D22000B9DA0008B9DA0008B9DA0008B9DA000892
:10D23000B9DA0008B9DA0008B9DA0008B9DA000882
:10D24000B9DA0008B9DA0008B9DA0008B9DA000872
:10D25000B9DA0008B9DA0008B9DA0008B9DA000862
:10D26000B9DA0008B9DA0008B9DA0008B9DA000852
:10D27000B9DA0008B9DA0008B9DA0008B9DA000842
:10D28000B9DA0008B9DA0008B9DA0008B9DA000832
:10D29000B9DA0008B9DA0008B9DA0008B9DA000822
:10D2A000B9DA0008B9DA0008B9DA0008B9DA000812
:10D2B000B9DA0008B9DA0008B9DA0008B9DA000802
:10D2C000B9DA0008B9DA0008B9DA0008B9DA0008F2
:10D2D000B9DA0008B9DA0008B9DA0008B9DA0008E2
:10D2E000B9DA00085DDC0008B9DA000841DC0008A2
:10D2F000B9DA0008B9DA0008B9DA0008B9DA0008C2
:10D30000B9DA0008B9DA0008B9DA0008B9DA0008B1
:10D31000B9DA0008B9DA0008B9DA0008B9DA0008A1
:10D32000B9DA0008B9DA0008E3DB000849DA0008D6
:10D33000CBD90008B9DA000829D900080FD90008AC
:10D34000F3D80008B9DA0008D9D800086DD8000869
:10D3500045D8000851D700081DDB0008B9DA0008DD
:10D36000EDDA0008B9DA0008B9DA0008C3DA000813
:10D370008DDB000879DB0008BBDB00089BDA0008C6
:10D380001BD80008EFD70008B9DA0008B9DA00089E
:10D39000B9DA0008B9DA0008B9DA0008B9DA000821
:10D3A000B9DA0008B9DA0008B9DA0008B9DA000811
:10D3B000B9DA0008B9DA0008B9DA0008B9DA000801
:10D3C000B9DA0008CFD70008B9DA0008B9DA0008DE
:10D3D00075D70008B9DA0008B9DA0008B9DA000828
:10D3E000B9DA0008B9DA0008B9DA0008B9DA0008D1
:10D3F0005BD70008202D7FF4CBAD0B68AC4D591CDA
:10D400006A7821601A7023682A78591C21601A7082
:10D410002368AA78591C21601A7029892046FEF7D2
:10D42000F5FB23686A79591C21601A702268A97972
:10D4300029E5822D7FF4ACAD0B689E4A9E4D117894
:10D440009B4A581C2060197011892046FEF7DEFBAC
:10D450009A4B22681B88FF2B02F10101A8BFFF2312
:10D4600021601370A96881F3100189B22046FEF78C
:10D47000CDFB296801F30F0189B22046FEF7C6FBF8
:10D480008F4B22681978FEE4012D7FF481AD0B6883
:10D490000022591C21601A7023685A1C22601D70DA
:10D4A00022682421531C23602B46117024E5326826
:10D4B000716891421EBF531C33601178814A08BFC6
:10D4C0001946204628F08AFB2FE57F4B1E7803364D
:10D4D00016F0FF063FF429AD7C4BDFF81C821E449A
:10D4E00003F1010A4FF00A0920E0B9F1500F00F0F2
:10D4F0005F87B9F1320F00F07487A9F13C00C0B228
:10D50000132840F272870025294623685A1C22609E
:10D51000204683F80090FEF779FB29462046FEF767
:10D5200075FB56453FF401AD1AF8019BB9F10A0F9E
:10D53000DBD1674B9D68196805EB85054FF6FF73D6
:10D540006D009D42A8BF1D469942A8BF194625EA15
:10D55000E57521EAE171ADB289B2D6E70B68DFF873
:10D560009C915C4E591C022221601A7023684FF076
:10D5700006085A1C226083F8008023680A22591C7E
:10D5800021601A70236801255A1922601D70B9F8AC
:10D5900000102046FEF73AFBB9F802102046FEF7CD
:10D5A00035FB23685A19226083F8008023685022D3
:10D5B000591921601A7023680022591921601A70C4
:10D5C00031882046FEF722FB71882046FEF71EFBBD
:10D5D0002B4691E4404BBBE40B685A1C0A601D705B
:10D5E0000B680222591C21601A704AE4334B0A6806
:10D5F0001B88314DFF2BA8BFFF23511C21601370E6
:10D60000A96881F3100189B22046FEF7FFFA334B77
:10D6100020461988FEF7FAFA296801F30F0189B24A
:10D6200020460125FEF7F2FA2B4665E40B222C4931
:10D630002046FEF7A3FA08222A492046FEF79EFA62
:10D640000125072228492046FEF798FA2B4653E485
:10D65000002A3FF46AAC254B136001252B464BE4AE
:10D660003268511C31601278002A01F00581102ABD
:10D6700007BF1F4B93E842001E46314625686B1CCE
:10D68000236020462A70FEF7A9FA31462046FEF7AD
:10D69000A5FA184B20465968FEF7A0FA204600214B
:10D6A000FEF7B4FA00212046FEF7B0FAFFF7E9BB17
:10D6B000846E0020E65B0020646C0020D05B0020BC
:10D6C000D8600020895A0308CD5A002034AD0308E1
:10D6D000082500203C250020E4530020D0600020D5
:10D6E000B8DB0308C4DB0308D0DB0308657001085E
:10D6F00094240020882100204C250020A4650020CF
:10D700005A1C3260BF4A1B78DFF82C831370002349
:10D71000C8F800303046FEF707FA3368D8F8002022
:10D72000B949BA4D10435A1CC8F8000032601B7842
:10D730000B723046FEF710FA28603046FEF70CFAFE
:10D7400068603046FEF708FAA8603046FEF704FA33
:10D750003046FEF701FAFFF7E8BBAD4B1B78DB075D
:10D7600000F1AA81012509F01BFD0AF06DFC2B4692
:10D77000FFF7C2BB5A1C32601A780F2A00F29C8154
:10D78000991C3160C2EBC202A24958788854D81C57
:10D7900030600A4499785170191D3160D9789170C0
:10D7A000591D31601979D170991D31605979117104
:10D7B000D91D31609979517103F108013160DB792C
:10D7C0009371012516F002FA2B46FFF795BB304600
:10D7D000FEF7C2F9DFF86482A8F80E003046FEF7C3
:10D7E000BBF90125A8F80C002B46FFF785BB1946AD
:10D7F0005A1C3260884A11F8020B10703160597857
:10D800005170D91C316099789170191D3160DB78A5
:10D81000D37001252B46FFF76FBB3046FEF79CF90E
:10D82000DFF81C82A8F810003046FEF795F9A8F83A
:10D8300012003046FEF790F90125A8F814002B4697
:10D84000FFF75ABB5A1C32601878060601F1B18006
:10D850006F4B1B78DD073FF568AB032828BF00201E
:10D86000012509F081FC2B46FFF746BB5A1C3260AC
:10D87000304693F800A0FEF757F981463046FEF790
:10D8800053F905463046FEF74FF980463046FEF71D
:10D8900063F93046FEF760F93046FEF769F9BAF1F0
:10D8A000000F01F06F80BAF1100F7FF43EAB5B4BBD
:10D8B000C3F800905D60B8F1000F02D0584BC3F878
:10D8C00004805849584B0222081F01251A701CF089
:10D8D000BFFC2B46FFF710BB4D4B1B78D8073FF51D
:10D8E00024AB012509F03AFD0AF0AEFB2B46FFF709
:10D8F00003BB474B1B78DA073FF517AB4B4A13784E
:10D90000012543F0040313702B46FFF7F5BA404B93
:10D910001B78D9073FF509AB454B4FF4C872012579
:10D920001A802B46FFF7E8BA092A40F3C580DFF8D2
:10D9300014811A46591CD8F80050316012F8021BA5
:10D94000297032605A78AA70DA1C32609A78642A98
:10D9500003F10401A8BF64226A713160DA78642A95
:10D9600003F10501A8BF6422AA7131601A79EA7136
:10D970009A1D32605A79642A03F10701A8BF642214
:10D980002A7231609A79EA7003F108023260DB7919
:10D990002B713046FEF7E0F8726833686881D11A5F
:10D9A00000290CDD591CD8F800003160521A002AF9
:10D9B0001978417203DD9A1C32605B78437001254F
:10D9C00029F0ACFB2B46FFF797BA1A4A1068DA1C0D
:10D9D00001462133951E356012F8035C0D70551E0B
:10D9E000356012F8025C4D70326012F8015C8D7087
:10D9F0000332934201F10301ECD118F05DFEFFF711
:10DA000094BA00BFE8390020906B00203C3300201E
:10DA10005C5B0020744000204C57002094240020C0
:10DA20008821002098240020605900209C6E00204E
:10DA3000B69E0020305C0020945D0020B46500207C
:10DA4000D8660020989E00205A1C32601A78CB4974
:10DA5000002A00F080870A7842F00202981C0A70BF
:10DA6000C74D30605B782B753046FEF75DF8286057
:10DA70003046FEF759F868603046FEF76DF82881A9
:10DA80003046FEF769F8BF4AE8811378012543F074
:10DA9000020313702B46FFF72FBA1A46591C316048
:10DAA00012F8020B3260DA1C597832609A7820F052
:10DAB00085FA00287FF439AA4FF0FF352B46FFF78F
:10DAC0001BBA3046FEF748F8DFF8C882A8F8000015
:10DAD0003046FEF741F8A8F802003046FEF73CF861
:10DAE0000125A8F804002B46FFF706BADFF8C89214
:10DAF00099F80030002B3FF418AADFF8C082002507
:10DB00003046FEF729F818F00BFF99F80030A8EC22
:10DB1000010A01359D42F3DBFFF707BA0D2ACBD18D
:10DB20005A1C32601D78072DC6D8DFF89492304613
:10DB30004FF00C08FEF710F808FB05F809EB080594
:10DB4000A8803046FEF708F8E8803046FEF704F873
:10DB5000336828811A46591C316012F8021BA972D9
:10DB600032605B78EB723046FDF7DEFF012549F845
:10DB700008002B46FFF7C0B9834B844918684E2232
:10DB800001252AF04BFD2B46FFF7B6B919465A1C62
:10DB900032607F4A11F8020B107031605978517071
:10DBA000D91C31609B7893703046FDF7D5FF794BD7
:10DBB0000125D8802B46FFF79FB91A46591C3160C2
:10DBC000754912F8020B0870326074495A788A70ED
:10DBD000DA1C3260724A9B78937001252B46FFF75E
:10DBE0008BB9C2F34705122D3FF666AFC5B107F1F9
:10DBF000500307F12A0903EB450AC846AAF1260A91
:10DC00003046FDF7A9FF28F8020FC245F8D1654B51
:10DC100039F8022F23F8022FC845F9D1112D09D860
:10DC2000614A6B00023B13440021223223F8021F99
:10DC30009A42FBD15D4A01231D461370FFF75CB980
:10DC4000DFF8808100233046C8F80030FDF76CFF14
:10DC50000125C8F800002B46FFF74EB91A46591C9B
:10DC6000316012F8025B3260DA1C587832609978C1
:10DC7000002D00F0A986012D7FF457A90DF0C4FFF7
:10DC80002B46FFF739B94A4A127812F001017FF4A6
:10DC900013AF5A1C3260187801250DF0F7FE2B46A1
:10DCA000FFF72AB91A46591C31603C4912F8020B99
:10DCB000C87032603F495A784A71DA1C3260384A7B
:10DCC0009B78D37001252B46FFF716B93046FDF738
:10DCD00043FF3046FDF740FF3046FDF73DFF30463D
:10DCE000FDF746FF3368284D1946581C2A683060F6
:10DCF00011F8020B82F82C003160597882F8361046
:10DD0000D91C31609B7882F837303046FDF730FF00
:10DD10003046FDF72DFF3046FDF72AFF3046D5F897
:10DD20000080FDF719FFA8F83A003046D5F80080CA
:10DD3000FDF712FF33687268A8F83800D11A01297C
:10DD40000ADD591C2A6831601B7882F82E30304673
:10DD5000FDF70EFF33687268D31A032B0BDD3046D4
:10DD6000D5F80080FDF7F8FEA8F8320030462E689E
:10DD7000FDF7F2FEB08628683FE600BF9C6E0020EB
:10DD8000A06E00205E590020305C0020E0C903082E
:10DD9000AC65002038560020086A0020B4650020D9
:10DDA000C4650020E6350020E83500200C36002050
:10DDB0005C5B002044630020CD5A00209055002079
:10DDC000803F0020E45300205A1C3260C64DDFF82B
:10DDD00040831B7888F805303046D5F80090FDF771
:10DDE000BBFEA9F820003046D5F80090FDF7B4FE40
:10DDF00072683368A9F81E00D11A072919DD304668
:10DE0000FDF7AAFEA8F80A003046FDF7A5FEA8F81F
:10DE10000C003046D5F80090FDF79EFEA9F82200D0
:10DE20003046D5F80090FDF797FE33687268A9F880
:10DE30002400D11A03290BDD3046FDF78DFEA8F82A
:10DE40000E003046FDF788FE33687268A8F81000AF
:10DE5000D21A002A05DD591C2A6831601B7882F825
:10DE6000263009F0A7F921F0F9FEA04B1B68002B22
:10DE700000F076852868012515F03CFF2B46FFF75A
:10DE80003BB81A46591C3160DFF8848212F8021B35
:10DE900088F80210326096495A780A70DA1C3260AB
:10DEA000944D9A782A711A1D3260DB78092BA8BF2D
:10DEB00009233046AB70FDF74FFE33687268288047
:10DEC000D11A012905DD3046FDF746FE3368726838
:10DED000E8819A4207D05A1C32601B78003318BF81
:10DEE000012388F8073009F065F9336872689A42AF
:10DEF0003FF41BA85A1C32601B78EB7001252B469F
:10DF0000FEF7FABF3046FDF727FE05461CF096FAED
:10DF1000FF283FF40AA83F2D00F2E78407F15008DC
:10DF2000002308F8243D4FEAD509414607F12B00AC
:10DF300087F82B3009F101091CF060FA97F82B30B3
:10DF40005FFA89F905F007054B4505F1010503D195
:10DF500097F82C30AB4203D0294648461CF05AFAB9
:10DF600033687268D21A012A7EF7DFAF5A1C07F1B4
:10DF70005000326000221D7800F8252D1CF032FA86
:10DF800097F82B30AB420AD05B4B1B683BB19A79B8
:10DF9000AA4204D31B681B690BB128469847336813
:10DFA0005A1C3260404600221D7887F82C201CF055
:10DFB0000DFA97F82C30AB423EF4B7AF4E4B1B68CE
:10DFC000002B3EF4B2AF1B685B69002B3EF4ADAF93
:10DFD00028469847FEF7A9BF5A1C326093F8008084
:10DFE000B8F1110F3FF668AD9A1C3260434D5B7873
:10DFF00005F818303046FDF7AFFD40F6CA039842E9
:10E00000A8BF184640F2EE23984205EB4801B8BF7E
:10E0100018460125A0F2EE222B46192092FBF0F2C1
:10E020004A70FEF769BF364A1278012A3EF67DAF84
:10E0300018465A1C3260DFF8DC8010F8022B88F892
:10E040000220DA1C891A306001295878326040F3C6
:10E05000CF843046FDF780FD0125A8F800002B464F
:10E06000FEF74ABF1A46591C264D316012F8021BB2
:10E07000297132605B786B713046FDF76DFD336856
:10E0800028805A1C32601B78AB713046FDF764FD66
:10E09000336868805A1C32601B78EB7101252B466F
:10E0A000FEF72ABF0125FEF79DFA2B46FEF724BF97
:10E0B000154A03F108010133336013F8010C02F82B
:10E0C000010F8B42F7D1FEF730BF591C1A46316061
:10E0D0000E4912F8020B887032605B784B70012594
:10E0E0002B46FEF709BF00BF305C0020E03900205E
:10E0F000A8650020D8660020745A00203C38002013
:10E100007B5D0020505600208F6B0020D0650020E2
:10E11000086A00207E5D00200721B2FBF1F1C1EB0F
:10E12000C105521B7FF4C8ACC9B201F1FF395FFAD7
:10E1300089F900293EF4F9AEDFF808A309F10109D5
:10E1400015465A1C326093F90010BE4B4FF0000880
:10E1500093F902208A4203F1080300F0688308F172
:10E160000108B8F1040FF3D1A6E45A1C32601A7802
:10E170000E2A3FF6A1AC991C31605D78032D3FF665
:10E180009BACB148062101FB02F1421803F1030EDA
:10E190005571C6F800E09D784554191D3160D97855
:10E1A0005170591D316019799170991D31605979FB
:10E1B000D170D91D31609B79137101252B46FEF773
:10E1C0009BBE5A1C3260A14A1B78537501252B4611
:10E1D000FEF792BE591C31601D781F2D3FF66CACC6
:10E1E000052A7FF469AC3046FDF79EFC984B43F856
:10E1F00025001BF09FF9FEF798BE954D05F14008EC
:10E200003046FDF7A9FC3368A5F88000591C1A4672
:10E21000316012F8021B85F8821032605B7885F855
:10E2200083300435A845EBD1FEF77FBE5A1C32601F
:10E23000864D1B782B723046FDF78EFCA883304646
:10E24000FDF78AFC28833046FDF786FC3268688338
:10E25000531C33601278EA747268D31A032B00F3EC
:10E260005B833368D11A05290EDD5A1C32601B7896
:10E27000EB723046FDF758FC3368E8605A1C326098
:10E280001B782B7433687268D21A002A7EF74DAE61
:10E290005A1C32601B7885F8213001252B46FEF789
:10E2A0002BBE581C30606B4A1D781570091A002966
:10E2B0007EF73BAE991C31605B78003318BF0123B9
:10E2C000012553702B46FEF717BE3046FDF744FC80
:10E2D000DFF89481C8F800003046FDF73DFCC8F82F
:10E2E00004003046FDF738FC0125C8F808002B462D
:10E2F000FEF702BEDFF874810023C8F80030304614
:10E30000FDF712FCD8F8003001250343C8F80030AF
:10E310002B46FEF7F1BD5049102A13464FF000027C
:10E3200028BF10230A604A608A60CA600A74002B02
:10E330003EF4FBAD3268013913440132326012F809
:10E34000010C01F8010F9A42F7D1FEF7EEBD5A1CFD
:10E3500032601D78132D3FF6AFAB9A1C32605878AF
:10E360007B6227F075FC00283FF4A6AB7B6A3B4A32
:10E37000017802F82510D91C316002EB85029978EA
:10E380005170191D3160D8789070581D3060344933
:10E390001B79D3700868012528F04EFE2B46FEF746
:10E3A000ABBD3388FF2BA8BFFF23DBB2FEF73BBD1D
:10E3B0002C4BFFF7BFB81DF021F900283EF432AD19
:10E3C00003780A2B28D8B0F9023088FB0312DB1738
:10E3D000C3EBA2039BB2FF2BA8BFFF23DBB2FEF768
:10E3E00022BD98E82200FFF7A7B81DF007F9002822
:10E3F0003FF489A803780A2B3FF685A8B0F90430CA
:10E40000B0F9061003EB830383F3500521EAE171B1
:10E41000ADB289B2FFF779B80023DFE75A1C32604A
:10E420001A780A2A00F0E9813046FDF7A1FB304650
:10E43000FDF79EFB01253046FDF79AFB2B46FEF7C4
:10E440005BBD00BF689D0020F0530020906B002052
:10E450007C5F0020E839002090650020EC39002026
:10E46000305C0020402500203C330020945D0020DB
:10E470001A46591C3160BE4D12F8021B6970326099
:10E480005A782A70DA1C32609B78AB703046FDF700
:10E4900063FB33682881591C1A46316012F8021B4D
:10E4A000697132605B78AB7101252B46FEF724BDA4
:10E4B0005A1C32601B780A2B00F09981502B7FF494
:10E4C00044A93046FDF748FBDFF8BC82A8F80000FD
:10E4D0003046FDF741FB0125A8F802002B46FEF768
:10E4E0000BBD726835687B623046551BFDF71CFB1F
:10E4F000052D38627B6A00F26E818026B3460125C5
:10E5000094E80600521A103AB242B8BF1FFA82FBD2
:10E51000984A396A92683A61521A9345396A7B621D
:10E520002046FA6088BF1FFA82FBFDF757FB7B6A23
:10E53000002B00F02F81002D40F0F3802368C7F8F6
:10E5400000D05D71C0B00533C7F808D0FB61BBF1E6
:10E55000000F00F013823B6A3A69934280F00B820D
:10E56000AA463E6A7D627C6080255446FB681C1B7F
:10E57000804BB4F5807F28BF4FF480749B683219BC
:10E580009A4288BF9C1BFDF7CBFF2246BC683046F1
:10E590002146FEF745F8F969B86104EB000C0B78E9
:10E5A0007B6164452ED2DFF8E4910CF1FF3C04F16D
:10E5B000FF3E1EF8013F09EB830219F823405688FD
:10E5C000ECB100234FF4004204F1FF3816424FEA49
:10E5D000520202D00878284308706D0806D10AF16B
:10E5E000010A4D701FFA8AFA01318025D34503D8FC
:10E5F000F44533D8984531DC01339C42E6D1E645F9
:10E60000D7D1F9617B6ABA6913449BB2D3457B6267
:10E6100006D97B6A3A6A1C46D6183B699E42A5D346
:10E620007C68802D1CBF0AF101031FFA83FA0AF1EE
:10E63000020189B22046FDF7E9FA2368796A0125CB
:10E640005A19226020461D70FDF7E0FA23685344F2
:10E6500023602B46D7F800D0FEF74EBCFB697C68E0
:10E660001A463B7D1370DCE7336872689A4240F0CB
:10E670000881414BFF221A704FF0000A3F4D19F0FC
:10E68000C1FE514620223E4885F800A02CF045FAF4
:10E6900087F82CA097F82C30072B00F22481DFF8A4
:10E6A000F090374E524697F82C3003EB430309EBBA
:10E6B000C3035B7CE3B197F82C3003EB430309EB16
:10E6C000C30320215B699BB197F82C3003EB430314
:10E6D00009EBC303586946F8220008F049F92B7882
:10E6E00056F8230008F002FA2A780132D2B22A70D2
:10E6F00097F82C300133DBB287F82C3097F82C30A8
:10E70000072BD0D92368591C21601A70B8F1000F6B
:10E710003EF40BAC1B4BC8F8003001252B46FEF72E
:10E72000EBBB144B3A6A9B68D4F800905A449A4267
:10E7300072D93A6AA3EB0208FDF7F2FE4246494657
:10E74000386AFDF76DFF236803442360002D3EF413
:10E75000ECABB042BEF6E9AB002100E0236801302B
:10E760005A1CB04222601970F8D1FEF7DEBB00BF20
:10E77000846E0020D01C0020882100205B3E0020F9
:10E7800068370020012E02083C25002044AD030814
:10E7900018660020002DC4D159462046FDF736FAF0
:10E7A00023685A1C22601D70984B26689D683B6A3E
:10E7B0000BEB0302AA4200F20D81FDF7B1FE5A46AF
:10E7C0003146386AFDF72CFF236801250344236096
:10E7D0002B46FEF791BB3046FDF7BEF932687168F3
:10E7E0007B6A9142834675D106461D4688E63046CF
:10E7F000FDF7B2F9DFF8488268E69A1C3260844A75
:10E8000059781170D91C316099785170191D316097
:10E81000DB789370FEF789BBFDF782FE5A464946C6
:10E82000386AFDF7FDFE23680344236091E70AEB95
:10E83000C80B30468BF80210FDF78EF932682AF8C3
:10E8400038001346511C316013F8021B8BF803107B
:10E85000336053788BF80430D31C336093788BF893
:10E860000630131D33600135D2788BF80520A94599
:10E870007FF467ACFEF759BB664B93E84200FEF7A6
:10E88000FDBE5A1C19463260634811F8022B027013
:10E8900031605B784370042A03D9FF2A7EF4F1AA21
:10E8A000EAE65E490978994205D8022A7EF4E9AA87
:10E8B000FF2B7EF4E6AA236801255A1922601D70F9
:10E8C000B8F1000F3EF431AB554BC8F800302B4681
:10E8D000FEF712BB511C316012781D46131C064610
:10E8E00018BF01230CE652460CE707F12C084046FE
:10E8F0001BF060FDBB8DAB423FF432AB494B1B6854
:10E90000002B3FF42DAB1B689B69002B3FF428AB19
:10E9100028469847FFF724BB3046FDF71DF9A88429
:10E920003046FDF719F933687268E884D11A032973
:10E930007FF798AC1A46591C316012F8021BA97770
:10E9400032605B7885F820303046FDF705F9336892
:10E950007268688486E40A7802F0FD02FFF77EB8E8
:10E9600031483249324A334B036001250B60136052
:10E970002B46FEF7C1BA7D62AA4658E6DA46C7F8CA
:10E9800024B054E6234B1020C3F800905D600CF0D7
:10E9900085FB294A137843F001031370B8F1000F87
:10E9A0003EF4C3AA1C4B0125C3F804802B46FEF796
:10E9B000A3BA00F07F00032828BF002001250DF036
:10E9C0003FF92B46FEF798BA012515F05BFB2B4665
:10E9D000FEF792BA3B6AED1AFDF7A2FD2A463146D0
:10E9E000386AFDF71DFE236803442360FEF79DBAD5
:10E9F000124A99781288012512FB00F22B4692FBED
:10EA0000F1F2A8F80020FEF777BA00BFD01C002072
:10EA1000175C00205459002088210020CD5A002086
:10EA200071700108745A0020EC4000204041002021
:10EA300040450020B9AB00089C6E0020F463002024
:10EA4000A46500202DE9F04F2DED0A8B444B1B7877
:10EA500095B0012B089001F0F585424C94F8002107
:10EA6000002A41F02D80072B3F4D01F0E685002361
:10EA700004936B683C489847002800F0CE80B5F8B6
:10EA8000B430002185F85510002B41F02682EB6C44
:10EA9000B5F94070B5F93CE0686AB5F93E60A96A1D
:10EAA000DFF8D0B0A7EB030C8CEAEC72A2EBEC72AF
:10EAB000B2F5804FEA6AD8BFEF64AEEB0000D8BF72
:10EAC0003B46711A9B1A28636963284895F85610CB
:10EAD000AB6313F0F9FDDBF80030990040F10B87D0
:10EAE000D5ED0D5AD5ED0C7A214A94ED676AD4ED37
:10EAF000686A94ED697AD4F8A8311268B8EEE58AAC
:10EB0000D5ED0E5AF8EEE77AF8EEE58A013377EEA6
:10EB1000867A38EE268A78EE878A9342C4ED677A41
:10EB200084ED688AC4ED698AC4F8A83102F0D78000
:10EB30000B4B93F80080B8F1140F03F0BF81002352
:10EB4000D4F8B0710593062F00F2C886DFE817F0FD
:10EB5000DE14C81465148B1630061A16A11500BFF2
:10EB6000EC5A002090210020586F0020886F002070
:10EB7000503A00202C6A0020D34EDFF8BC93DFF817
:10EB8000BCA306F2DC680027D04BD5ED087A1B78D1
:10EB9000172B01F09E8096ED007AB8EEC78A082BFD
:10EBA00028EE278A07D1B0EE480A059329F0AAFE7D
:10EBB000059B2AF81700DBF8002092000BD5002FE8
:10EBC00004F0E185B0EE480AD5F8783708F1700016
:10EBD0009847B0EE408AB0EE480AD5F89836A8F1CA
:10EBE00070009847D5F8083740469847B74B1B78D0
:10EBF000032BB0EE408A01F07980D6F85C06D5F898
:10EC0000B830B0EE480A98470137032F08F12408BE
:10EC1000A9EC010A06F10406B6D1AC4B1F78072F08
:10EC200001F0188294F8C031002B40F09286A84B76
:10EC30005B79002B40F0A4850123A44A84F8C031FD
:10EC40001278072A02F0368000230B93A14B94ED33
:10EC5000729A93ED007AA04BDFF8E482D3F800A01B
:10EC60009E4B0593F7EE007A37EEC9BA9C4B07939B
:10EC70002BEE07BA9B4B09939B4B0693B4EEE7BA76
:10EC800008F168030025F1EE10FA0A93D4ED71BA89
:10EC9000964BDFF8B0B2DFED968A9FED96AADFEDD6
:10ECA00096AADFED969ADFF8A092954F049388BF5D
:10ECB000B0EE67BA2E46934B98ED008A2B44D3ED05
:10ECC000007AF5EE407AF1EE10FA17D08E4B2B4415
:10ECD000D3ED006A38EE667AB0EEC76AF4EEC67A13
:10ECE000F1EE10FA08D5B5EEC07AF1EE10FACCBF0D
:10ECF00037EEA68A36EEE78A83ED008A059B1A88EE
:10ED000093073FD0022E3DD0804B9AF82E1033F956
:10ED1000163007EE103A0A9B07EE901A2B44F8EED5
:10ED2000E76AB8EEC77AD3ED007A4B42A6EEA77A2F
:10ED3000700007EE903AF8EEE77AB4EEE77AF1EE7B
:10ED400010FA0AD407EE901AF8EE677AF4EEC77A52
:10ED5000F1EE10FA88BFF0EE477A6D4B6D4903442F
:10ED6000085EB3F90C30C01A07EE100AB8EEC77A85
:10ED7000D007E7EE687A40F1F485674B93ED008A9F
:10ED800027EE888A069B94F8D8212B44D3ED01CA3C
:10ED900038EE6CCA002A3DD0604BD4F8DC210899CB
:10EDA0001B688A1A9A4235DD9AF84830022B02F025
:10EDB0009280022E04F07584594B1B68990740F12C
:10EDC0006F87534B5349DFF850E131F916C09EED80
:10EDD000008ADFF878E1C7ED00AA03EB460028EED1
:10EDE000288AB0F90C00A0EB0C0007EE900AF8EEB0
:10EDF000E77ADEF8000027EE888A904238EE6CCA87
:10EE0000C1F23E82F7EE007AB4EEE79AF1EE10FA24
:10EE100001F10D82434B2B4493ED000A049B2BEE32
:10EE2000800A022E20EE0C0AA3EC010A049304F0DF
:10EE30005284079B9BED007AD3ED007A3A4BD7EDD5
:10EE4000006A93ED006A394B67EE277A2B4427EE70
:10EE50008B7AD3ED007A67EE277AF0EE665AE7EE0A
:10EE60008C5AB1EE467AB4EEE57AF1EE10FA08DC8F
:10EE7000F4EEC65AF1EE10FA8CBFB0EE467AB0EE60
:10EE8000657A94ED726AF7EE007AB4EEE76AF1EE15
:10EE900010FAACBF0123002343B1F0EEE66AF0EEB6
:10EEA000C77AF4EEE67AF1EE10FA01D587ED007A32
:10EEB000022E04F0DB831E4A1E4B52F826001B680C
:10EEC000B0EE6C0A44E000BF886F0020EC5A0020CE
:10EED000086A00205C550020305C0020D2600020D1
:10EEE000940000205C5B00201C6A00208839002010
:10EEF000CDCCCC3DAE47813F000000000000C842B1
:10EF000094390020505500205C230020202300204D
:10EF1000B46500207C6E0020385500206455002028
:10EF2000986E00200C5500208055002018550020B8
:10EF3000F0400020EC400020206A0020F05A002021
:10EF400094220020E8400020A039002060550020D5
:10EF50009847CB4ACB4B52F826001B6898479AF843
:10EF6000373023B1059B1B88002B00F06485B0EE81
:10EF70006A8AC54B9BED007A38EE400A2B4493ED2C
:10EF8000008A83ED000A9AF8483030EE480AC0EE55
:10EF9000077A2BB3099B1B78DB0721D5B7EE007AE4
:10EFA000B4EEC79AF1EE10FA04DB94F8D831002BD6
:10EFB00000F04A87D4F8DC31089AD31AB34A1268B1
:10EFC0009A420DDDB24B93ED007AB0EECCCAB4EEAE
:10EFD000C7CAF1EE10FA41F16F81002384F8D831ED
:10EFE000AC4B94F8E8212B4493ED007A2BEE877A12
:10EFF00067EE277AC9ED007A32B9049BC7ED00AA03
:10F0000043ED01AAC9ED00AA0136032E08F1040858
:10F0100009F1040907F1040705F104057FF44BAE7B
:10F020009D4B1B78072B01F05C83012B01F0478679
:10F03000002794F8F031002B40F0FC85974A984B5C
:10F0400010681B6810F4805A93F82C3040F05486F6
:10F05000944A954992ED006A498B944A84ED806AFE
:10F0600092ED007A924A84ED817A07EE901AF8EEDA
:10F07000E76AD2ED037A8F4A84ED7E6A37EE467AEC
:10F0800077EEE67AD2ED006A84ED7D7A012284F88B
:10F090000822C7EEA65A8849884A91ED005A884945
:10F0A0009FED886A91ED004A8749DFED886AD1EDCE
:10F0B000004A92ED007A35EE045AF7EE007AF4EE4B
:10F0C000E75A35EE245AF1EE10FA88BFF0EE675A8F
:10F0D00025EE065AF4EEE65AB1EE476AF1EE10FA62
:10F0E000B4EEC65AB8BFF0EE665AF1EE10FAC4EDAF
:10F0F000835A01F1F080B4EEC75AF1EE10FA88BFDE
:10F10000B0EE475A6C4ADFED6F6AD2ED017A6C4A75
:10F1100092ED014A6C4A77EE847AD2ED014A77EE9D
:10F12000A47A67EEA67AB4EEE76AF1EE10FA08DC8C
:10F13000B4EEE77AF1EE10FA8CBFB0EE676AB0EE8B
:10F14000476A5D4ADFED5F6AD2ED027A5C4AD2ED32
:10F15000024A5F4A77EEA47A92ED007A67EEA67AC9
:10F16000B1EE473AF4EEC37AF1EE10FA08D4F4EEB9
:10F17000C77AF1EE10FA8CBFB0EE473AB0EE673ABC
:10F18000544A52780AB9B1EE433A002B41F0C88391
:10F19000F7EE003A504D2A78002A02F044864F4B91
:10F1A000DFED4A7AD3ED024AD3ED016A93ED037A9B
:10F1B00066EE244AE5EE264AE3EE074A63EEA44AE9
:10F1C000F4EEE74AF1EE10FAB4BFB0EE674AB0EEE3
:10F1D000644A98BFF0EE647A012ACDED0C4A02F041
:10F1E000838693ED067AD3ED052AD3ED076A26EEE2
:10F1F000077AA5EE227AA3EE267A23EE877AB4EE7A
:10F20000E77AF1EE10FAB4EEC47A8CBFF0EE676ADA
:10F21000F0EE476AF1EE10FA88BFF0EE676AB4BF0D
:10F22000F0EE447AF0EE477A022A8DED0D7A00F086
:10F230000F8193ED0A7AD3ED092A93ED0B4A26EE5E
:10F24000077AA5EE227AA3EE047A23EE877AB4EE4B
:10F25000E67AF1EE10FAB4EEE77A8CBFB0EE664AC9
:10F26000B0EE474AF1EE10FA98BFF0EE446AA8BF3C
:10F27000F0EE477A032A8DED0E7A00F0E9802FE058
:10F2800044410020404100207023002064550020AC
:10F290007055002024550020EC5A00202C6A0020D4
:10F2A000305C002010640020906B002084650020FA
:10F2B000E85B00204056002088390020845500205B
:10F2C000943900206F12833AA0390020000000001A
:10F2D00088550020E8390020CD5A0020B055002084
:10F2E00093ED0E7AD3ED0D2A93ED0F4A26EE077AB1
:10F2F000A5EE227AA3EE047A23EE877AB4EEE67ABC
:10F30000F1EE10FAB4EEE77A8CBFB0EE664AB0EEDA
:10F31000474AF1EE10FA98BFF0EE446AA8BFF0EE4B
:10F32000477A042A8DED0F7A00F0928093ED124A0D
:10F33000D3ED112A93ED137A26EE044AA5EE224A64
:10F34000A3EE074A23EE844AB4EEE64AF1EE10FA41
:10F35000B4EEE74A8CBFB0EE667AB0EE447AF1EED6
:10F3600010FA98BFF0EE476AA8BFF0EE447A052A7B
:10F370008DED104A6CD093ED164AD3ED152A93ED1E
:10F38000177A26EE044AA5EE224AA3EE074A23EE98
:10F39000844AB4EEE64AF1EE10FAB4EEE74A8CBFC6
:10F3A000B0EE667AB0EE447AF1EE10FA98BFF0EE65
:10F3B000476AA8BFF0EE447A062A8DED114A47D07D
:10F3C00093ED1A4AD3ED192A93ED1B7A26EE044ADF
:10F3D000A5EE224AA3EE074A23EE844AB4EEE64A9B
:10F3E000F1EE10FAB4EEE74A8CBFB0EE667AB0EEFA
:10F3F000447AF1EE10FA98BFF0EE476AA8BFF0EE3B
:10F40000447A072A8DED124A22D093ED1E7AD3ED6D
:10F410001D2A93ED1F4A26EE077AA5EE227AA4EE66
:10F42000037A27EE237AB4EEE67AF1EE10FAB4EE20
:10F43000E77A8CBFB0EE666AB0EE476AF1EE10FA7A
:10F440008DED137A98BFF0EE466AA8BFF0EE477ACA
:10F4500077EEE67AF7EE006AF4EEE67AF1EE10FA6D
:10F46000C4ED727A43F3298686EEA77A022ADDED8F
:10F470000D7A67EE244A67EE877ACDED0C4ACDED22
:10F480000D7A2DD0DDED0E7A67EE877A032ACDED69
:10F490000E7A25D0DDED0F7A67EE877A042ACDED5E
:10F4A0000F7A1DD0DDED107A67EE877A052ACDED53
:10F4B000107A15D0DDED117A67EE877A062ACDED48
:10F4C000117A0DD0DDED127A67EE877A072ACDED3D
:10F4D000127A05D0DDED137A27EE877A8DED137A57
:10F4E000AA4B1E6816F0805601F0C280F6EE005A54
:10F4F000C4ED835A002A02F08B84A54BD4ED814AD7
:10F5000093F8038094F908320999D4ED806A91F850
:10F5100000E0DFF88CC29F49DFF88892B1F906104D
:10F520009CED007A049106EE103AFDEEE44A9A4B07
:10F5300099F80090B3F81AB094ED7D5AD4ED7E7A24
:10F5400014EE903AFDEEE64A00F0100C00F4800054
:10F550000EF0010EB8EEC66A14EE901A0590B8F1DE
:10F56000000F41F01F82DFF84082BCF1000F41F034
:10F57000CB8098ED007ADDED0C6ADFF830C225EE25
:10F58000877AA6EE267AF0EE676AE5EE076ABDEEA8
:10F59000E67A17EE106A17EE100A9E42A8BF1846C8
:10F5A000B142C8BF084607EE100AB8EEC77A012A72
:10F5B0008CED007A00F0DC8098ED047ADDED0D6AC8
:10F5C00025EE877AA6EE267AF0EE676AE5EE076A00
:10F5D000BDEEE67A17EE106A17EE100A9E42A8BF3B
:10F5E0001846B142C8BF084607EE100AB8EEC77AFF
:10F5F000022A8CED017A00F0BB8098ED087ADDEDEF
:10F600000E6A25EE877AA6EE267AF0EE676AE5EEB8
:10F61000076ABDEEE67A17EE106A17EE100A9E42F0
:10F62000A8BF1846B142C8BF084607EE100AB8EE98
:10F63000C77A032A8CED027A00F09A8098ED0C7A52
:10F64000DDED0F6A25EE877AA6EE267AF0EE676A80
:10F65000E5EE076ABDEEE67A17EE106A17EE100ABD
:10F660009E42A8BF1846B142C8BF084607EE100A1E
:10F67000B8EEC77A042A8CED037A79D098ED107A27
:10F68000DDED106A25EE877AA6EE267AF0EE676A3F
:10F69000E5EE076ABDEEE67A17EE106A17EE100A7D
:10F6A0009E42A8BF1846B142C8BF084607EE100ADE
:10F6B000B8EEC77A052A8CED047A59D098ED147A01
:10F6C000DDED116A25EE877AA6EE267AF0EE676AFE
:10F6D000E7EE056ABDEEE67A17EE106A17EE100A3D
:10F6E0009E42A8BF1846B142C8BF084607EE100A9E
:10F6F000B8EEC77A062A8CED057A39D098ED187ADB
:10F70000DDED126A25EE877AA6EE867AF0EE676A5C
:10F71000E7EE056ABDEEE67A17EE106A17EE100AFC
:10F720009E42A8BF1846B142C8BF084607EE100A5D
:10F73000B8EEC77A072A8CED067A19D098ED1C7AB4
:10F74000DDED136A65EE875AE6EE265AE5EE257A78
:10F75000FDEEE77A17EE900A8342A8BF0346814286
:10F76000C8BF0B4607EE903AF8EEE77ACCED077A81
:10F77000BEF1000F40F06B82002A40F0638266E227
:10F78000064B1B78013BDBB2FFF757BA68650020D8
:10F79000DC600020A8600020906B0020A86500209D
:10F7A0008C550020FC660020B0550020BC3900209C
:10F7B000AE4B1A78D4F8B4E1AD4E9FEDAE7A4FEA75
:10F7C000CE00331883ED007A002A7CD0AA49B0EE2F
:10F7D000476AF0EE476A0023F1EC017A013367EEE5
:10F7E000A77A05EE903AB4EEE77AF1EE10FAF8EE69
:10F7F000E55AB8BFB0EE677A934276EEA76AA7EEF5
:10F80000A56AE9D1F5EEC06A3318F1EE10FA83ED7E
:10F81000007A58DDC6EE265A984B994A1288B7EE00
:10F82000000AD3ED007A75EEC05A65EEA77AFDEEB8
:10F83000E77A17EE903A812B42F376849342A8BF81
:10F84000134607EE903AF8EEE77A8E4B00EB0E0186
:10F8500003EB810393ED057AD3ED003A93ED066A4D
:10F8600093ED014AD3ED046AD3ED034A93ED025AB6
:10F87000A3EEA77AA4EE276A66EEC76AA7EE646ACB
:10F88000BDEEC77AE5EE276A17EE101A812983EDDF
:10F89000056AC3ED066A42F34B848A42A8BF0A4652
:10F8A00007EE902AF8EEE77AFCEEE77ACDED067ADD
:10F8B000BDF8183032189380BEF1000F03D1B8F1B3
:10F8C000130F03F00284B8F1150F41F0FB853044AB
:10F8D0006D4E838826F81E30D4F8B0716B4B01371B
:10F8E00083FB0723DA19FB17C3EBA203C3EBC303A4
:10F8F000FF1AC4F8B071664B1B78002B7FF43CA94B
:10F90000644FDFF8B89107F24C7607F5F768F7EC2B
:10F91000017A95ED080AD5F87837F8EEE77A30469F
:10F9200027EE800A9847A6F1E000D5F89836984768
:10F93000A6F17000D5F808379847D7F85806D5F8DB
:10F94000B83098472436B045A9EC010ADFD1FFF75B
:10F9500064B9013B84F8C03115B0BDEC0A8BBDE839
:10F96000F08F94ED5E7AB1F90000D4ED5F6AB1F9E1
:10F9700002E0494AF4EEC76A80EAE0738EEAEE716B
:10F98000A3EBE073F1EE10FAA1EBEE71B4BFB0EEB1
:10F99000476AB0EE666A8B42B8BF0B4607EE103A74
:10F9A0001378B8EEC77A27EE287A002B40F0E7816B
:10F9B0003A4BD3ED005AF4EECA5AF1EE10FA41F187
:10F9C0000D81B7EE005A75EE654ADFED356A9FEDA1
:10F9D000355A354B36EEC77A24EE855AD3ED006A98
:10F9E000E7EE055A65EEA65AF5EEC05AF1EE10FAAA
:10F9F00040F23A86C9EEA56AB7EE007AF0EE475AB1
:10FA0000E6EE665AF0EE656AF4EEC76AF1EE10FAB9
:10FA100088BFF0EE476AF5EEC06AF1EE10FAB8BFA3
:10FA2000F0EE6A6A214B93ED007A67EE877AA7EED3
:10FA3000A68AFFF7A7B91E4B1E4A2B4493ED007A06
:10FA4000D2ED007A1C4B67EE277AF7EE006AF4EEEF
:10FA5000E67AF1EE10FA93ED007A88BFF0EE667A5E
:10FA600067EE877A27EE888AFFF783BA563A002036
:10FA7000743C00200000000090210020583A002033
:10FA8000543A00208C3C0020F05A002093244992E4
:10FA9000493A0020886F0020445500204C55002032
:10FAA00000003443610BB63B405500203C5500201C
:10FAB000082300203455002030550020206A002003
:10FAC000072B02F00C820027DFF874B3C34DDBF87C
:10FAD00000305E0501F1E480C14B1B78002B40F043
:10FAE000DE81DFF83C9394F8126126B1BD4B1B8890
:10FAF000980742F0508194F81821002A41F0738051
:10FB000099F81E30002B00F0FF83022B01F07C8758
:10FB1000032B01F05583B44B598899F81F300233F9
:10FB2000DBB2002A01F06187002901F05E87AF484F
:10FB30000068B1FBF0F10FFA81F8A4F84881002BBE
:10FB400003F0CF8207EE908AF8EEE77AF7EE006ACC
:10FB500086EEA77AA649012BD4ED576AD1ED007A3B
:10FB600077EEE67A67EE877AC4ED537A21D0D1ED4D
:10FB7000017AD4ED586A77EEE67A022B67EE877A3F
:10FB8000C4ED547A15D0D1ED027AD4ED596A77EEEE
:10FB9000E67A032B67EE877AC4ED557A09D0D1ED6A
:10FBA000037AD4ED5A6A77EEE67A67EE877AC4ED87
:10FBB000567A90480078092803F0C382B8F1000F04
:10FBC00040F3A98393B394ED577AD4ED537A77EE4B
:10FBD000877A012BC4ED577AC1ED007A21D094EDDC
:10FBE000587AD4ED547A77EE877A022BC4ED587A9E
:10FBF000C1ED017A15D094ED597AD4ED557A77EEAE
:10FC0000877A032BC4ED597AC1ED027A09D0D4ED7D
:10FC10005A7A94ED567A77EE877AC4ED5A7AC1ED26
:10FC2000037A013B022BB8BF0223DBB2002A18BFC4
:10FC3000022371E3099B704D1B78DE0700F12882D7
:10FC40002A7822B192006D496D4828F0E7FC6D4B8F
:10FC50001B68002B40F043836B4B1B789BB12878CB
:10FC600070B1DFF89C81DFF8DC910026F0B2D9F8A2
:10FC70000030B8EC010A9847287801368642F5DB57
:10FC8000624B1B6898475B4B1B78072B00F0228563
:10FC9000012384F8003115B0BDEC0A8BBDE8F08F6C
:10FCA0005B4BC7ED00AA1B689342BFF6ABA8594B4C
:10FCB0001A88002384F8D831002A41F07D86564AFC
:10FCC000564B1178186881F0010106F015FFFFF717
:10FCD000A1B896ED007A05EB4702B8EEC78A928F7D
:10FCE0002AF8172028EE278AFEF765BF28F00AFEBB
:10FCF0002AF81700FEF781BF099A1278D50703D4B6
:10FD0000474A128BA4F8FC21464A3949128891EDE2
:10FD1000037A07EE902AF8EEE77AB4EEE77AF1EE8E
:10FD200010FA41F265814049098807EE901AF8EE11
:10FD3000E77AB4EEE77AF1EE10FAC1F2A3803B491C
:10FD40003B4AD1ED006A92ED006A3A49C4ED806AFF
:10FD5000BCEEC75A76EE665A15EE102AC4ED7E6ADE
:10FD6000C4ED7D5A84ED816AA4F8FC210122D1ED15
:10FD7000006A84F8082277EE677AFFF78AB92E4B7B
:10FD800093ED005AB5EEC05AF1EE10FA40F36C84D0
:10FD90002A4BD3ED006AF5EEC06AF1EE10FA40F39B
:10FDA000638436EEC77A66EE695A87EE266AC5EE38
:10FDB000856AB7EE007AB4EEC76AF1EE10FA88BF32
:10FDC000B0EE476AB5EEC06AF1EE10FA76EE876AD9
:10FDD000B8BFB0EE6A6A66EE266A15E6586F002074
:10FDE000E01C0020D2600020D8350020E03900203F
:10FDF000E85B0020EC5A0020CD5A002090550020EE
:10FE0000BC390020E4400020046A0020F86600208D
:10FE10006055002064790020667900206879002010
:10FE2000906B00204456002046560020305600209B
:10FE3000846500204C560020405500204855002085
:10FE40002C6A0020F0660020864A92ED007AF0EEDF
:10FE5000E76AF4EEC76AF1EE10FA7FF7ABA8824AC0
:10FE600092ED007AF0EECC6AF4EEC76AF1EE10FA89
:10FE70007FF7A0A87D4A98ED007AD2ED006AB0EE37
:10FE8000C77AB4EEE67AF1EE10FA7FF593A8012274
:10FE90000899C4F8DC1184F8D821FFF78FB8744BA7
:10FEA000DFF8E891B3F90620B9F81A309A423FF723
:10FEB0001AAE704B1B78012B01F08885192B01F0CD
:10FEC00085850E2B3FF40FAE082B3FF40CAE6A492C
:10FED00000238B60C4F80C3105E6684A06924FF4A3
:10FEE0007A7E1268BEFBF2F2C2EB421802EB880285
:10FEF0004FEAC2086248634E634F90F801903F7822
:10FF0000B6F906001FFA88F8434502F01481D5F8C7
:10FF100088E0B5F93CC0EA6E0EF1010107EE90CA27
:10FF200062440129C5F88810EA66F8EEE77A02F023
:10FF30000D81D5ED1E5AD5ED206A07EE101A37EE69
:10FF4000E56AB8EEC75A012B86EE057A37EE257AB8
:10FF500077EEC77A85ED1F7AE7EE866A85ED1E7A21
:10FF6000F0EE667AC5ED216AC5ED206A02F0C5861D
:10FF7000D5F89CE0B5F93EC02A6F0EF1010107EEFD
:10FF800090CA62440129C5F89C102A67F8EEE77A06
:10FF900002F0F580D5ED235AD5ED256A07EE101A4B
:10FFA00037EEE56AB8EEC75A012B86EE057A37EED2
:10FFB000257A77EEC77A85ED247AE7EE866A85EDB5
:10FFC000237AF0EE667AC5ED266AC5ED256A02F061
:10FFD000BE86D5F8B0E0B5F940C06A6F0EF10101F8
:10FFE00007EE90CA62440129C5F8B0106A67F8EEBE
:10FFF000E77A02F0DD80D5ED285AD5ED2A6A07EEC2
:020000040801F1
:10000000101A37EEE56AB8EEC75A012B86EE057A6C
:1000100037EE257A77EEC77A85ED297AE6EE276AFC
:1000200085ED287AF0EE667AC5ED2B6AC5ED2A6A71
:1000300002F05686F080B5F8B430134A013B1778C9
:10004000A5F8B43006990023072F4B608B60CB6076
:100050007EF4E8AD08F0E2FA049B0A4EC01A308044
:10006000FEF7E0BD74550020705500207855002043
:10007000A8600020E8390020E85B00201C6A00200E
:10008000086A0020F05A0020EC5A0020906B0020F3
:100090002B78002B3FF4DBADD4ED5F3A94ED5E4A54
:1000A000D4ED7E7A8F4A94ED7D7A92ED005AD4EDAC
:1000B0005C5A94ED5B6ADFF84882DFF848C2F4EEE0
:1000C000C43AF3EE046AF1EE10FA77EEA64A00F1B4
:1000D000C88798ED026A26EE656AB0EE674AA6EE1A
:1000E000074AB4EEE44A34EE666AF1EE10FA48BF0D
:1000F000B0EE456A012B8CED006A3FF4A8AD98ED97
:10010000066A26EE656AB0EE674AA6EE074AF4EE86
:10011000C44A34EE666AF1EE10FA88BFB0EE456A62
:10012000022B8CED016A3FF492AD98ED0A6A26EE3F
:10013000656AB0EE674AA6EE074AB4EEE44A34EECA
:10014000666AF1EE10FA48BFB0EE456A032B8CEDFB
:10015000026A3FF47CAD98ED0E6A26EE656AB0EE59
:10016000674AA6EE074AF4EEC44A34EE666AF1EE38
:1001700010FAC8BFB0EE456A042B8CED036A3FF459
:1001800066AD98ED126A26EE656AB0EE674AA6EE95
:10019000074AF4EEC44A34EE666AF1EE10FAC8BFBC
:1001A000B0EE456A052B8CED046A3FF450AD98ED36
:1001B000166A26EE656AB0EE674AA6EE074AB4EE06
:1001C000E44A74EE666AF1EE10FAB8BFF0EE456AE2
:1001D000062BCCED056A3FF43AADD8ED1A6A66EE0F
:1001E000E56AB0EE674AA6EE874AB3EE046AF4EE1B
:1001F000C44A74EE466AF1EE10FAC8BFF0EE456AE2
:10020000072BCCED066A3FF422ADD8ED1E6A66EEF0
:10021000E55AE5EE877AF4EEE74A77EEC67AF1EE34
:1002200010FAC8BFF0EE457ACCED077A0FE50699D3
:100230002D4BD1ED017A93ED007AF0EEE77AF4EEF2
:10024000C77AF1EE10FA7EF5E5ADD1ED027AF0EE67
:10025000E77AB4EEE77AF1EE10FA7EF7DBADD1ED96
:10026000037AF0EEE77AB4EEE77AF1EE10FA7EF771
:10027000D1AD1E4B1B689A077FF519AD1C491D4B6C
:10028000B3F90C20B1F900E01B48AEEB020E006898
:100290008EEAEE72A2EBEE728242BEF6BBADB3F90D
:1002A0000E30B1F90220D21A82EAE273A3EBE273B4
:1002B00098427EF7AFADFAE4104B98ED007AD3ED9B
:1002C000006AB0EEC77AB4EEE67AF1EE10FA7EF785
:1002D00087AEFEF782BEB0EE465AFEF713BF13F0AC
:1002E000C5F8B9E48C5500206C550020986E0020AC
:1002F0007C6E0020B46500206855002078550020F1
:10030000B0550020BC390020A4F848319846002A96
:1003100000F07281D9490223D94ADFEDDA6A106808
:10032000D94A90F802E092F800C0027807EE902ACD
:10033000F8EEE77AB0EE007A67EEA67AF4EEC77AC6
:10034000F1EE10FA40F31D8337EEC77ADFEDCF6A86
:10035000B0EE676AA7EE266AB0EE467A9FEDCC6AE9
:10036000D1ED006A66EE866AB0EEE66AC4ED5B6ABD
:1003700084ED5E6ABEF1000F13D005EE90EAB8EE90
:10038000E55ADFEDC05A66EEA64A25EE255AF7EE8D
:10039000005A75EEC55A64EE864AE4EE855A66EE5A
:1003A000A56ADFEDBC5A427927EE257A27EE267A38
:1003B000CAB1DFEDB46ADFEDB85A26EE266A06EE62
:1003C000902AF8EEE66A26EE266AB4EEE56AF1EEC9
:1003D00010FA00F33486F7EE005A35EEC66AC5EE21
:1003E000866A27EE267ABCF10C0F9FEDAC8ADFED12
:1003F000AC6A00F0D985B4EEC87AF1EE10FA98BF75
:10040000B0EE478AB4EEE68AF1EE10FAB8BFB0EE6D
:10041000668A84ED418A002B00F0E280B0EE007A1B
:10042000F4EEC77AF1EE10FA05DD37EEC77ADFEDAC
:10043000976AE7EE267A91ED017ADFED956A27EE6D
:10044000267AB0EEC76A84ED5C7A84ED5F6ABEF10D
:10045000000F13D006EE90EADFED8A5AF8EEE66A56
:1004600027EE075A66EEA56AF7EE005A75EEE65AD1
:1004700025EE065AE5EE265A27EE257ADFED856A47
:10048000827967EEA67A67EE877AAAB107EE102A1C
:10049000B8EEC77ADFED7B5ADFED7F6A27EE067A8A
:1004A00027EE257AB4EEE67AF1EE10FA40F3CB852A
:1004B000DFED7C6A67EEA67ABCF10C0F00F02485B4
:1004C000DFED766A9FED767AF4EEE67AF1EE10FAD9
:1004D00088BFF0EE667AF4EEC77AF1EE10FAB8BF94
:1004E000F0EE477A012BC4ED427A79DD4378DFEDF7
:1004F000656A07EE903AF8EEE77AB0EE007A67EEBA
:10050000A67A437AF4EEC77AF1EE10FA05DD37EEFB
:10051000C77ADFED5E6AE7EE267A91ED027ADFEDCB
:100520005C6A27EE267AB0EEC76A84ED5D7A84EDC8
:10053000606A9BB106EE903ADFED525AF8EEE66A39
:1005400027EE075A66EEA56AF7EE005A75EEE65AF0
:1005500025EE065AE6EE855A27EE257ADFED4D6A3E
:10056000C37967EEA67A67EE877A0BB307EE103A87
:10057000B8EEC77ADFED435ADFED476A27EE067A19
:1005800027EE257AB4EEE67AF1EE10FA0CDCB5EE41
:10059000C07AF1EE10FA01F12482B7EE006A36EE6D
:1005A000477AC6EE076A01E0DFED3E6A67EEA67A9B
:1005B000BCF10C0F00F0A084DFED386A9FED387AB3
:1005C000F4EEE67AF1EE10FA88BFF0EE667AF4EE19
:1005D000C77AF1EE10FAB8BFF0EE477AC4ED437A6D
:1005E000BCF1090F00F06D8499F82160002E40F0F5
:1005F0000384002384F818312B4B1B68990609D516
:100600002A4B1B8803F0300323B1294B1B78DA07F0
:1006100002F13F80274B1B7823B9274EB378002B7C
:1006200041F0F981184B1B78072B00F0D884002289
:10063000072B84F800217EF41AAA07F0EFFF04903C
:10064000FEF717BA1D4B1E4C1A681E4B1E4E94F82F
:100650000001D2691B883280738000287FF433AA9E
:1006600004901A4DFEF705BADFED196AFFF7DAB903
:1006700041023EF53BAFFEF73DBF00BFE85B002007
:10068000989E00200AD7233CEC5A0020D7A368414B
:100690006F12033B00004843A4707D3F00C0F94443
:1006A00000C0F9C40000C842986E0020D26000204B
:1006B0009C6E00204F5900207E5D00205863002072
:1006C00090210020FA330020F05A0020586F0020BB
:1006D0000000000007F0A2FFAB4BC01BD880FFF763
:1006E000D7BA07F09BFFA94B0B9A1B78A64E801A2E
:1006F000012B708000F0E482072B7EF499AC07F0A8
:100700008DFF0746FEF795BCBEF1000F41F0FE835A
:1007100098ED007ADDED0C6ADFF884C225EE877A69
:10072000A6EE867AF0EE676AE7EE056ABDEEE67A37
:1007300017EE106A17EE100A9E42A8BF1846B14283
:10074000C8BF084607EE100AB8EEC77A012A8CED3A
:10075000007A3FF477AA98ED047ADDED0D6A25EE74
:10076000877AA6EE867AF0EE676AE7EE056ABDEE56
:10077000E67A17EE106A17EE100A9E42A8BF1846D6
:10078000B142C8BF084607EE100AB8EEC77A022A7F
:100790008CED017A3FF456AA98ED087ADDED0E6AE9
:1007A00025EE877AA6EE867AF0EE676AE7EE056AAE
:1007B000BDEEE67A17EE106A17EE100A9E42A8BF49
:1007C0001846B142C8BF084607EE100AB8EEC77A0D
:1007D000032A8CED027A3FF435AA98ED0C7ADDED10
:1007E0000F6A25EE877AA6EE867AF0EE676AE7EE64
:1007F000056ABDEEE67A17EE106A17EE100A9E4201
:10080000A8BF1846B142C8BF084607EE100AB8EEA6
:10081000C77A042A8CED037A3FF414AA98ED107A73
:10082000DDED106A25EE877AA6EE867AF0EE676A2D
:10083000E7EE056ABDEEE67A17EE106A17EE100ACB
:100840009E42A8BF1846B142C8BF084607EE100A2C
:10085000B8EEC77A052A8CED047A3FF4F3A998ED37
:10086000147ADDED116A25EE877AA6EE867AF0EE2F
:10087000676AE7EE056ABDEEE67A17EE106A17EED4
:10088000100A9E42A8BF1846B142C8BF084607EEEC
:10089000100AB8EEC77A062A8CED057A3FF4D2A981
:1008A00098ED187ADDED126A25EE877AA6EE867A43
:1008B000F0EE676AE7EE056ABDEEE67A17EE106ABB
:1008C00017EE100A9E42A8BF1846B142C8BF08469C
:1008D00007EE100AB8EEC77A072A8CED067A3FF4C5
:1008E000B1A998ED1C7ADDED136A65EE875AE6EE44
:1008F000265AE5EE257AFDEEE77A17EE900A834256
:10090000A8BF03468142C8BF0B4607EE903AF8EEF7
:10091000E77ACCED077A002A7FF494A9FFF797B91C
:100920001B4B5A79002A3EF433AC1A4A1278002A3B
:100930003EF42EAC1B78DFED184A07EE903A174BC9
:10094000B8EE677A1B8807EE902A06EE903AF8EE2A
:10095000E77AF8EE666A67EE277AB7EE007AC7EEB6
:10096000A63AF4EEE43AF1EE10FA88BFF0EE643AFB
:10097000F4EEC73AF1EE10FAB8BFF0EE473AFEF7E0
:1009800009BCB0EE677AE9E4F05A0020EC5A002086
:10099000846E0020E65B0020713DAA3FD05B002002
:1009A000BC390020BCF1000F00F02284BEF1000F22
:1009B00042F05F80DFF8E485B9F1000F41F0008775
:1009C000D8ED006ADDED0C4ADFF8D4C565EEA66A05
:1009D000BDEEC77A17EE101AB0EE667AA4EE867AEC
:1009E000F0EE676AE7EE056ABDEEE67A17EE106A8A
:1009F00017EE100A9E42A8BF1846B142C8BF08466B
:100A000007EE100AB8EEC77A012A8CED007A3FF49F
:100A100019A998ED047ADDED0D6A25EE877AA6EE28
:100A2000867AF0EE676AE7EE056ABDEEE67A17EEC3
:100A3000106A17EE100A9E42A8BF18468E42B8BF31
:100A4000084607EE100AB8EEC77A022A8CED017A42
:100A50003FF4F8A898ED087ADDED0E6A25EE877A66
:100A6000A6EE867AF0EE676AE7EE056ABDEEE67AF4
:100A700017EE106A17EE100A9E42A8BF18468E4263
:100A8000B8BF084607EE100AB8EEC77A032A8CED05
:100A9000027A3FF4D7A898ED0C7ADDED0F6A25EEC7
:100AA000877AA6EE867AF0EE676AE7EE056ABDEE13
:100AB000E67A17EE106A17EE100A9E42A8BF184693
:100AC0008E42B8BF084607EE100AB8EEC77A042A6D
:100AD0008CED037A3FF4B6A898ED107ADDED106A3C
:100AE00025EE877AA6EE867AF0EE676AE7EE056A6B
:100AF000BDEEE67A17EE106A17EE100A9E42A8BF06
:100B000018468E42B8BF084607EE100AB8EEC77AFC
:100B1000052A8CED047A3FF495A898ED147ADDED62
:100B2000116A25EE877AA6EE867AF0EE676AE7EE1E
:100B3000056ABDEEE67A17EE106A17EE100A9E42BD
:100B4000A8BF18468E42B8BF084607EE100AB8EE96
:100B5000C77A062A8CED057A3FF474A898ED187AC6
:100B6000DDED126A25EE877AA6EE867AF0EE676AE8
:100B7000E7EE056ABDEEE67A17EE106A17EE100A88
:100B80009E42A8BF18468E42B8BF084607EE100A1C
:100B9000B8EEC77A072A8CED067A3FF453A898ED91
:100BA0001C7ADDED136A65EE875AE6EE265AE5EE0D
:100BB000257AFDEEE77A17EE900A8342A8BF034636
:100BC0008142D8BF194607EE901AF8EEE77ACCEDCD
:100BD000077A002A7FF436A8FFF739B8DA4BD3ED4D
:100BE000005AFEF701BFD94BD949D3F8EC30096858
:100BF00044F620608342A8BF0346B3F57A7FB8BFAE
:100C00004FF47A7398B2C906A4F81A01DBF80030E1
:100C100041F18582DB0400F19286CE4BD3F800E0EF
:100C2000BEF93260CC49DFF87CC3D1ED037AD4F849
:100C30001C31ACFB00108009642191FBF0F11429F8
:100C4000BDEEE77A04EB430CA8BF142101338B42BD
:100C5000C4F81C3117EE108AA4BF0023C4F81C315D
:100C600004EB4303ACF82081B3F9203107EE103ACE
:100C7000B8EEC77A77EEC77AFDEEE77ACDED047A63
:100C8000BDF9101081EAE173A3EBE173B34202F303
:100C90000582B24B19464FF07E530B60FEF730BF12
:100CA000AB68002B3EF418AF05F150012846984779
:100CB000FEF712BF07F0B2FC0B90FDF7C7BFA84EBE
:100CC00007F0ACFCA74AD4F8EC311268C4F8EC0188
:100CD000C31A9A1A0746B380F280FEF7AAB907EE44
:100CE000103AA14B9E4E1B78B6F9040095ED080A08
:100CF000B4F8AC81B8EEC77AF7EE006A0022132B85
:100D000086EE879AC4F8A82101F0F983974B984A98
:100D100002EB88070021C4F89C11C4F8A01167EE0B
:100D2000897A93ED001A93ED053A93ED122A93ED2B
:100D3000176AD3ED091A93ED0E4AD3ED015AD3ED9C
:100D4000063A93ED0A7A93ED0F5AD3ED132AD3EDB9
:100D5000186AD3ED044AD3ED030A69EE288A29EE16
:100D6000088AA1EE273AA2EE286AA1EE884AE5EEAB
:100D7000A73AA7EE085A93ED167AD3ED0D5A93EDE4
:100D8000021AD3ED0C1A87ED003AE2EEA86A64EE7F
:100D9000C34A27EE467A93ED0B2AD3ED152A87ED49
:100DA000204AE0EEC33A65EEC45A93ED143AC3ED1F
:100DB000053AE1EE274AF0EE477AA1EEC45AE2EE98
:100DC000085AE2EEC66AE3EE287AC3ED064A83EDDE
:100DD0000E5AC3ED0F5A87ED406AC3ED176AC3ED93
:100DE000187AC4F8A41108F1010303F01F03A4F852
:100DF000AC31B080FDF79CBE1E215548FBF74CFA84
:100E000000283FF4F6AB5B4B1B8858063FF5F1AB6F
:100E100094F88431B34242F0F981504BD4ED627AB8
:100E2000D3ED016A94ED435ADFED535A9FED536AB7
:100E300027EEC57A68EE277AA8EE267AE5EE267ABE
:100E4000B4EEE57AF1EE10FA88BFB0EE657AB4EE52
:100E5000C67AF1EE10FAF4EEE57AB8BFB0EE467A53
:100E6000F1EE10FA88BFF0EE657AF4EEC67AF1EE94
:100E700010FAB8BFF0EE467A84ED417AC4ED437AB9
:100E8000FFF7B7BBB4F8FC11914240F264853C49CE
:100E90003C4AD1ED007A92ED007A3B49C4ED807A6C
:100EA00077EE676AC4ED7E7A0122C4ED7D6A84ED37
:100EB000817AD1ED006ADFED357A84F80822FEF7F9
:100EC000E8B8FDEEC87A264E17EE903AA6F80480F0
:100ED000F380FFF789BB2E4B1B88002B40F05A850F
:100EE0002C4A2D4B1178186805F006FED4F8DC2149
:100EF000089B9A1AFDF75DBFBDEEE77A184E17EE14
:100F0000103AB380FFF758BB9FED1B7ADFED1B6AE9
:100F1000134EF4EEC77AF1EE10FA98BFB0EE677A8E
:100F2000FDEEE77AB4EEE67AF1EE10FA17EE902ACB
:100F3000B8BFB0EE667A012B84ED427A72803FF73B
:100F4000D5AAFFF751BB00BF4055002080160020F6
:100F500068650020305C0020E85B002094000020E1
:100F6000F05A0020E0390020EC5A0020F83C002024
:100F7000743A0020D260002000C0F94400C0F9C4D7
:100F800030560020846500204C56002000000000F0
:100F9000647900206679002068790020B05500202F
:100FA000BC390020D34D6210B4EEC87AF1EE10FACD
:100FB00098BFB0EE478ABDEEC77AB4EEE68A854E9A
:100FC000F1EE10FA17EE102AB8BFB0EE668A84ED83
:100FD000418A3280002B7FF421AAFFF705BB07F07E
:100FE0001DFB7C4E7C4BC01B1B78B080FFF71FBBEA
:100FF0007A4A7B49D2ED006A7A4A91ED006A12780A
:10100000C4ED806A84ED816A002A40F0A08476EE07
:10101000C65AF0EE466ABCEEC76A7349C4ED7D5A03
:1010200016EE102AC4ED7E6AA4F8FC21FF22D1ED51
:10103000006A84F8082277EEC77AFEF72AB8DFED57
:101040006B6AFFF7CEB9B5EEC07AF1EE10FA00F197
:10105000C484B7EE006A36EE477AC6EE076AFFF739
:1010600029BAD8ED015A65EEC65AB0EE674AA5EE28
:10107000874AF4EEC44A74EE665AF1EE10FAC8BF1D
:10108000F0EE455A012BCCED005A3EF4E0ADD8ED20
:10109000055A65EEC65AB0EE674AA5EE874AF4EEE9
:1010A000C44A74EE665AF1EE10FAC8BFF0EE455A23
:1010B000022BCCED015A3EF4CAADD8ED095A65EECB
:1010C000C65AB0EE674AA5EE874AF4EEC44A74EEFB
:1010D000665AF1EE10FAC8BFF0EE455A032BCCED7C
:1010E000025A3EF4B4ADD8ED0D5A65EEC65AB0EED4
:1010F000674AA5EE874AF4EEC44A74EE665AF1EEEA
:1011000010FAC8BFF0EE455A042BCCED035A3EF45A
:101110009EADD8ED115A65EEC65AB0EE674AA5EEFF
:10112000874AF4EEC44A74EE665AF1EE10FAC8BF6C
:10113000F0EE455A052BCCED045A3EF488ADD8EDBF
:10114000155A65EEC65AB0EE674AA5EE874AF4EE28
:10115000C44A74EE666AF1EE10FAC8BFF0EE456A52
:10116000062BCCED056A3EF472ADD8ED196A66EE39
:10117000C66AB0EE674AA6EE874AF3EE045AF4EE6A
:10118000C44A74EE656AF1EE10FAC8BFF0EE456A23
:10119000072BCCED066A3EF45AADD8ED1D6A26EE5B
:1011A000C66AE6EE077AF4EEE47A77EEE57AF1EED7
:1011B00010FAB8BFF0EE457ACCED077AFEF747BDDE
:1011C00099F82030C3EB431103EB8101C90089B2C8
:1011D000FEF7A3BCF05A0020EC5A00201064002057
:1011E00034560020FC660020485600200000C8420B
:1011F000DFF88485B9F1000F41F04280D8ED006A34
:10120000DDED0C4ADFF874C565EEA66ABDEEC77A5F
:1012100017EE101AB0EE667AA4EE867AF0EE676AE0
:10122000E7EE056ABDEEE67A17EE106A17EE100AD1
:101230009E42A8BF1846B142C8BF084607EE100A32
:10124000B8EEC77A012A8CED007A3EF491AA98EDA7
:10125000047ADDED0D6A25EE877AA6EE867AF0EE49
:10126000676AE7EE056ABDEEE67A17EE106A17EEDA
:10127000100A9E42A8BF18468E42B8BF084607EE25
:10128000100AB8EEC77A022A8CED017A3EF470AAF1
:1012900098ED087ADDED0E6A25EE877AA6EE867A5D
:1012A000F0EE676AE7EE056ABDEEE67A17EE106AC1
:1012B00017EE100A9E42A8BF18468E42B8BF0846D5
:1012C00007EE100AB8EEC77A032A8CED027A3EF4D4
:1012D0004FAA98ED0C7ADDED0F6A25EE877AA6EE1F
:1012E000867AF0EE676AE7EE056ABDEEE67A17EEFB
:1012F000106A17EE100A9E42A8BF18468E42B8BF69
:10130000084607EE100AB8EEC77A042A8CED037A75
:101310003EF42EAA98ED107ADDED106A25EE877A5C
:10132000A6EE867AF0EE676AE7EE056ABDEEE67A2B
:1013300017EE106A17EE100A9E42A8BF18468E429A
:10134000B8BF084607EE100AB8EEC77A052A8CED3A
:10135000047A3EF40DAA98ED147ADDED116A25EEBB
:10136000877AA6EE867AF0EE676AE7EE056ABDEE4A
:10137000E67A17EE106A17EE100A9E42A8BF1846CA
:101380008E42B8BF084607EE100AB8EEC77A062AA2
:101390008CED057A3EF4ECA998ED187ADDED126A31
:1013A00025EE877AA6EE867AF0EE676AE7EE056AA2
:1013B000BDEEE67A17EE106A17EE100A9E42A8BF3D
:1013C00018468E42B8BF084607EE100AB8EEC77A34
:1013D000072A8CED067A3EF4CBA998ED1C7ADDED58
:1013E000136A65EE875AE6EE265AE5EE257AFDEE9B
:1013F000E77A17EE900A8342A8BF03468142D8BF1E
:10140000194607EE901AF8EEE77ACCED077ABEF1AE
:10141000000F7EF41CACFEF7AFB9DFF86493D4ED97
:10142000017A94ED006AB9F80000D9F8143077EE2B
:10143000A77AF0EE006AB0EE677AA6EE267A013857
:1014400004EBC002D6EE267A083A1033F6EE003AE4
:1014500027EE237A67EEA37A84ED207AC4ED217A11
:10146000BE4C264604F1800192ED027A92ED036AA9
:10147000D6ED036AD6ED027A53ED014A13ED025A16
:1014800037EE674A76EEC65A77EE277AE4EE845A4C
:101490000138A2F10802E5EE047A06F1080603F12C
:1014A000080336EE267A01F10801E4EE877AE5EECC
:1014B000475A67EEA37A25EEA37AC1ED007A81ED53
:1014C000017AD1D1B8F1140F7EF408AA07F0A6F87A
:1014D000059BA34EC01A7080D4F8B071FEF7FEB918
:1014E000DFF89C929D48D9F80820B9F80C1026F036
:1014F00017F99C4B93F80080B8F1140F01F06F8638
:10150000D4F8B0710137C4F8B07188E7DFF8709291
:10151000B9F80070D9F804E04FEA570C4FEA8C0292
:1015200004EB8708FF0804EB020300F09F801032F1
:1015300001378D4803EB0717424410330EF11006B4
:1015400008F1100151ED032A51ED043A10ED043A6F
:1015500010ED032A51ED026A11ED016A10ED020A45
:1015600010ED018A12ED044A12ED035A53ED044ABC
:1015700053ED035A13ED027A53ED017A52ED020A4C
:1015800012ED011A73EE238A72EE221A40ED048ADC
:1015900040ED031A70EE268A78EE061A40ED028AB4
:1015A00040ED011A74EE848A75EE851A43ED048AC3
:1015B00043ED031A77EE208A77EE811A43ED028A13
:1015C00043ED011A73EE633A75EE655A16ED035A50
:1015D00032EE623A74EE644A65EE631A16ED044A1E
:1015E00023EE052A64EE652AE3EE041A10339F42C7
:1015F00024EE843AA3EE842A00F1100006F11006CE
:10160000A5EE853A01F1100102F11002E4EE852AFF
:1016100041ED071A01ED082A02ED073A42ED082ACA
:1016200056ED055A16ED065A70EE666A38EE466AB1
:1016300030EEC77A71EE677A26EE253A65EEE63A25
:1016400025EE674A67EE054AE6EE053AA6EE853ACC
:10165000A7EE254AE7EEA54A01ED063A41ED053A27
:1016600002ED064A42ED054A7FF46CAF1FFA8CF694
:1016700072463146394824F0B3FC3146D9F804208B
:10168000404624F0ADFC374B1B78142B7FF424AF7D
:101690001CE7D4F8B4C1B4F8ACA1344BCAF12009AA
:1016A0005FFA89F90AEB4C165FEA990003EB8606AC
:1016B00001F01A85013000012D492B4A06EB000E7E
:1016C00006F1100313ED024A13ED035A13ED016AFC
:1016D00013ED047A51ED024A51ED035A51ED016ABE
:1016E00051ED047A64EE244A65EE255A66EE266AC8
:1016F00067EE277A10339E4542ED024A42ED035AC7
:1017000042ED016A42ED047A01F1100102F110028A
:10171000D8D1184A103806441118204419F0030390
:1017200009D0B6EC017AF1EC017A67EE277A013B39
:10173000E0EC017AF5D1BAF1000F40F05587B8F12D
:10174000140F7EF4CBA806F069FF059B044ED4F875
:10175000B071C01A7080FEF7C1B800BF90210020A0
:10176000F05A0020EC5A0020A0210020743A0020FA
:10177000043C0020F43B0020B0550020BC39002080
:101780005C3A0020D4F8B491D24BD34ADFEDD37A3F
:10179000D2ED008AD24E4FEAC9010B44F8EE688AB6
:1017A0009B8809EE103A643BC82BA8BFC82368EE9B
:1017B000A78AF8EE497A782BB8BF782368EEA78A13
:1017C00007EE903A4944B0EE680A06EB8106B8EE9F
:1017D000E78A27F0E3F8B8EEC99AF0EE409AB0EE47
:1017E000680A27F03DF838EE097A79EE487A28EE53
:1017F000098A67EE877AB7EE006A88EE277AB8F131
:10180000140FF8EE007A77EE076A60EE277A89EE19
:10181000A67A77EE065A36EE477AC6EE256A67EE66
:10182000A67A27EE267AC6ED006A86ED047AC6ED22
:10183000026AC6ED017AC6ED037A01F0DB84A94B9A
:10184000A94A09F1010983FB093CACEBE97C0CEBEB
:101850004C0C0137A9EB0C0C92F80080C4F8B07165
:10186000C4F8B4C117E7DFF8BC9299F800209008DB
:1018700001F0A485DFF8B0E200F1010C4FEA4C1C46
:101880000EEB0C060EF12003AEF1700113ED076AAA
:1018900053ED056A13ED037A53ED017A53ED025AC5
:1018A00013ED084A53ED064A13ED045A26EE066A74
:1018B00066EEA66A27EE077A67EEA77AA4EE046AB8
:1018C00020339E42E4EEA46A01F11001A5EE057AF0
:1018D000E5EEA57AF1EEC65AB1EEE66AF1EEC76A18
:1018E000B1EEE77A41ED085A01ED076A41ED066A6B
:1018F00001ED057ACAD1ACF1200CE64404EB0010EE
:1019000012F0030318BF0EF1080E0FD05EED017A3E
:101910001EED027A67EEA77A013BE7EE077A0EF139
:10192000080EB1EEE77AA0EC017AEFD1B8F1140F0E
:1019300001F046840137C4F8B071FDF73BBF6B4B33
:10194000D3F800E0BEF832607608FFF76BB976EEA8
:10195000665AFFF760BB664A6649D2ED007A664A6E
:1019600091ED007A1278C4ED807A84ED817A002AB4
:1019700001F08E8377EE676A6049C4ED7E7AC4ED2C
:101980007D6AFF22D1ED006ADFED5D7A84F80822DE
:10199000FDF77FBB5B494B69002B3DF40AAA5A480F
:1019A0005A4B008893FBF0F00B684FF0010E186063
:1019B00081F811E0FDF7FDB952494A69002A3DF46A
:1019C00029AA0A6813604B74FDF724BA504B9B7B1D
:1019D000002B3EF47CAAFEF786B8F7EE006AFEF70D
:1019E00069BDF7EE006AFEF7E1BDB4F8488108F181
:1019F000FF380FFA88F8B8F1000FA4F848817EF795
:101A000086AC4449FEF7DEB8B4F81A1101F57A71D4
:101A100089B2FEF782B8DFF8148198F80020013A05
:101A20000D2A18D8DFE812F09C01AB0158013601ED
:101A30001D010001EA00E100BC00A5009000840047
:101A400092010E001F20049325F0F0FA049B10B9B8
:101A5000012288F80020012B00F0F587F278002A97
:101A60003EF4E0AD2C4A1278D00706D4049315F06A
:101A7000FDFB049B002841F07E84284ED4F8981189
:101A80003268914201F27E8498F80030012B3EF4D6
:101A9000C9AD94F89421002A3EF4C4AD0B2B0DD8A7
:101AA00001229A4040F6030112EA01090CD112F416
:101AB000C06F03D0093B012B41F28A86184B326874
:101AC0005A600B2388F80030002384F89431FEF725
:101AD000A9BD00BF743C00201C6A002027D4D23668
:101AE000D476002056555555EC5A0020305C002025
:101AF0001064002034560020FC6600204856002068
:101B0000000000006C7900208479002020A10700EB
:101B10008C9D0020E85B00205C5B00208C7900201D
:101B200088650020563A0020102200207B5D0020AE
:101B3000012B01D1FAF756FD0D23132088F8003050
:101B400009F07CF9B37886E7C74AC8495268096842
:101B5000C8328A4205D326F027FDB37800283FF427
:101B60007AAF032B01F0F385012388F80030B378B6
:101B700071E7BF4B1B78002B01F06F841A2025F012
:101B800055FA002841F0698494F89431002B41F013
:101B90006484092388F800301CF0B6FFB3785AE754
:101BA0001A2025F043FA0028F6D0B24B1B88002BF0
:101BB000F2D1B14B4520D3F800901CF0FBFA0E2077
:101BC0001CF0F8FA48461CF0EBFBDDF82090484684
:101BD0001CF0E6FBA94AAA4B12681A6048460A2381
:101BE00088F800301CF070FCD6E71AF07FFF1CF07C
:101BF000C1FF002841F02785B3782CE71AF076FF63
:101C0000A04B002105208DE80300A3F108020291FA
:101C1000532010F023F80028EED1934AB3781060D7
:101C2000082288F8002016E71AF060FF964A029210
:101C3000A2F10C034FF007090193CDF80090A2F137
:101C400008030021143A472010F008F80028D3D1E7
:101C5000854B88F800904FF0FF3283E80500B37899
:101C6000F9E61AF043FF894B002102208DE80300BA
:101C7000A3F10802029148200FF0F0FF0028BBD129
:101C8000794AB37810604FF0FF315160062288F82E
:101C90000020E0E61AF02AFF7D4A0292A2F10C032E
:101CA000252101930091A2F10A035021163A4920FF
:101CB0000FF0D4FF00289FD1DBF8002012F0800243
:101CC00001F0DB84684AB37810604FF0FF31516057
:101CD000052288F80020BEE6DFF88C911AF006FF96
:101CE000624AD9F8043012686433934284D24020A7
:101CF0001AF0D4FE00287FF47FAFD9F80030DFF867
:101D0000B8A164494FF0400B0FE004911CF052FA67
:101D10000499D9F800300A680133013ABBF1010B8C
:101D20000A60C9F8003001F087851AF803301846B8
:101D3000002BEAD100234FF0FF32C9F80030042312
:101D400088F80030C9F80420B37884E6012B01F04C
:101D500069840E23132088F8003009F06FF84BE7F0
:101D60004D4B1B78DB0701F164841F2025F05EF9E1
:101D700000283FF441AF0C2388F800303CE73B4A91
:101D8000394912684A60434800220A600321026010
:101D900088F800105FE6414BDFED417A93ED080AC9
:101DA000B4EEE70AF1EE10FA40F2498626F040FE62
:101DB000D4ED457A20EE270A26F0A4FDB0F5617F28
:101DC00000F3EF8707EE900AF8EEE76ADFED357A69
:101DD00066EEA76A07EE906AB8EEE77AFDEEE67A5D
:101DE00017EE903A2033402B41F2F3829FED2E0AFA
:101DF00026F088FD00B207EE900AB8EEE77A2B498C
:101E0000D1ED037A77EE877AC1ED037AFDF773BEE1
:101E1000099B93F800E00EF0010EBEF1000F7DF477
:101E200016AFFDF7A9BC224BDFED227A1E68C4ED88
:101E3000727A16F0805640F0A38410F4800600F009
:101E400015820026B6EE007A67EE877AF4EEE75A3E
:101E5000F1EE10FA48BFF0EE675A40F19184C4EDFC
:101E6000835AFDF747BB00BF886500208C790020AE
:101E70003C3A0020E8630020E4630020F86300207F
:101E8000F0630020C0B3030878B303085CB3030811
:101E9000AEB103083C5E00205C5B00207053002064
:101EA0008FC2753CD06D393A00000000E85B00201D
:101EB000686500200000008048B1030806F0AEFB12
:101EC000E14B059093F80080B8F1140F05BFDF4E89
:101ED000D4F8B071D4F8B0713780FCF734BE06F096
:101EE0009DFB0746FDF7F0BD74EE677AB7EE007A0A
:101EF000F4EEC77AF1EE10FAC4ED727A41F3DD80A8
:101F000084EEA77A8DED0C7AFDF7EABABAF1000FEC
:101F100000F0A88798ED007ADDED0C6ADFF848C381
:101F200025EE877AA6EE867AF0EE676AE7EE056A16
:101F3000BDEEE67A17EE106A17EE100A9E42A8BFB1
:101F40001846B142C8BF084607EE100AB8EEC77A75
:101F5000012A8CED007A3DF47AAE98ED047ADDED3D
:101F60000D6A25EE877AA6EE867AF0EE676AE7EECE
:101F7000056ABDEEE67A17EE106A17EE100A9E4269
:101F8000A8BF1846B142C8BF084607EE100AB8EE0F
:101F9000C77A022A8CED017A3DF459AE98ED087AA1
:101FA000DDED0E6A25EE877AA6EE867AF0EE676A98
:101FB000E7EE056ABDEEE67A17EE106A17EE100A34
:101FC0009E42A8BF1846B142C8BF084607EE100A95
:101FD000B8EEC77A032A8CED027A3DF438AE98ED5C
:101FE0000C7ADDED0F6A25EE877AA6EE867AF0EEA2
:101FF000676AE7EE056ABDEEE67A17EE106A17EE3D
:10200000100A9E42A8BF1846B142C8BF084607EE54
:10201000100AB8EEC77A042A8CED037A3DF417AEA5
:1020200098ED107ADDED106A25EE877AA6EE867AB5
:10203000F0EE676AE7EE056ABDEEE67A17EE106A23
:1020400017EE100A9E42A8BF1846B142C8BF084604
:1020500007EE100AB8EEC77A052A8CED047A3DF433
:10206000F6AD98ED147ADDED116A25EE877AA6EECD
:10207000867AF0EE676AE7EE056ABDEEE67A17EE5D
:10208000106A17EE100A9E42A8BF1846B142C8BF98
:10209000084607EE100AB8EEC77A062A8CED057AD4
:1020A0003DF4D5AD98ED187ADDED126A25EE877A0C
:1020B000A6EE867AF0EE676AE7EE056ABDEEE67A8E
:1020C00017EE106A17EE100A9E42A8BF1846B142DA
:1020D000C8BF084607EE100AB8EEC77A072A8CED8B
:1020E000067A3DF4B4AD98ED1C7ADDED136A65EE29
:1020F000875AE6EE265AE5EE257AFDEEE77A17EEE8
:10210000902A9342A8BF13468A42A8BF194607EEF9
:10211000901AF8EEE77ACCED077AFDF798BDDE006D
:102120003EF578ADFDF7ECBCDFED497AFDF78DBBF0
:102130008223FDF7BFBBB5F93C20696207EE902A08
:102140000121F8EEE77AEA66C5F888100022012B33
:10215000C5ED1F7AC5ED1E7AC5F8802001F03381E8
:1021600043457DF405AFB5F93E202A6707EE902A76
:1021700000210122F8EEE77AA962C5F89C2000222E
:10218000012BC5ED247AC5ED237AC5F8942001F022
:102190001D8143457DF41DAFB5F940206A6707EE08
:1021A000902A00210122F8EEE77AE962C5F8B02012
:1021B0000022012BC5ED297AC5ED287AC5F8A820A3
:1021C0007DF438AF9FED238A032F36D0B9F1000F8D
:1021D00009D007EE909AF8EEE77AF4EEC87AF1EEBD
:1021E00010FA01F10E821C4A6B6F1268F08094F8AD
:1021F000B801002103EB580393FBF8F3EB62916203
:102200001163D16230B1154B1B8823F40063002B9E
:102210007DF411AF124B1B6813F4003341F0C680FC
:1022200010481A46C15C012903F10C0300F0028634
:102230000132152AF6D1FDF7FEBEB0EE480A26F0AF
:1022400061FB00B2C2E700BFEC5A0020F05A002048
:1022500000000243000000005863002000610020DD
:10226000E453002098CD0308BC390020B6EE007A74
:10227000F4EEC75AF1EE10FA3FF7E4ADFDF73AB9C4
:10228000D8ED004A9DED0C4ADFF830C565EEA44A52
:10229000FDEEC73AE4EE064AB0EE674AA4EE854A80
:1022A00013EE901AF4EEC46AF1EE10FAF0EE444A1E
:1022B00088BFF0EE474AFDEEE44A14EE900A14EEB1
:1022C000906A9842A8BF1E468142C8BF0E4604EEDF
:1022D000906AF8EEE44A012ACCED004A3DF448AA9F
:1022E000D8ED044A9DED0D4A65EEA44AE4EE064A97
:1022F000B0EE674AA4EE854AF4EEC46AF1EE10FA35
:10230000F0EE444A88BFF0EE474AFDEEE44A14EE90
:10231000900A14EE906A9842A8BF1E468842B8BF41
:102320000E4604EE906AF8EEE44A022ACCED014A29
:102330003DF41EAAD8ED084A9DED0E4A65EEA44A6A
:10234000E4EE064AB0EE674AA4EE854AF4EEC46AAB
:10235000F1EE10FAF0EE444A88BFF0EE474AFDEE87
:10236000E44A14EE900A14EE906A9842A8BF1E4602
:102370008842B8BF0E4604EE906AF8EEE44A032A9B
:10238000CCED024A3DF4F4A9D8ED0C4A9DED0F4A7C
:1023900065EEA44AE4EE064AB0EE674AA4EE854A2A
:1023A000F4EEC46AF1EE10FAF0EE444A88BFF0EEA3
:1023B000474AFDEEE44A14EE900A14EE906A984201
:1023C000A8BF1E468842B8BF0E4604EE906AF8EEDB
:1023D000E44A042ACCED034A3DF4CAA9D8ED104AD8
:1023E0009DED104A65EEA44AE4EE064AB0EE674A57
:1023F000A4EE854AF4EEC46AF1EE10FAF0EE444A17
:1024000088BFF0EE474AFDEEE44A14EE900A14EE5F
:10241000906A9842A8BF1E468842B8BF0E4604EE96
:10242000906AF8EEE44A052ACCED044A3DF4A0A9EE
:10243000D8ED144A9DED114A65EEA44AE4EE064A31
:10244000B0EE674AA4EE854AF4EEC46AF1EE10FAE3
:10245000F0EE444A88BFF0EE474AFDEEE44A14EE3F
:10246000900A14EE906A9842A8BF1E468842B8BFF0
:102470000E4604EE906AF8EEE44A062ACCED054AD0
:102480003DF476A9D8ED184A9DED124A65EEA44AAE
:10249000E4EE064AB0EE674AA4EE854AF4EEC46A5A
:1024A000F1EE10FAF0EE444A88BFF0EE474AFDEE36
:1024B000E44A14EE900A14EE906A9842A8BF1E46B1
:1024C0008842B8BF0E4604EE906AF8EEE44A072A46
:1024D000CCED064A3DF44CA9D8ED1C4A9DED134ABB
:1024E00065EEA45AE6EE045AE5EE257AF4EEE76AC4
:1024F000F1EE10FAC8BFF0EE477AFEF778BFA74FAB
:10250000DFF89C9297ED004A97ED057AD7ED014AE6
:1025100097ED066AD7ED046A97ED035AD7ED025A94
:1025200067EE897A09EB8803A4EE277AA4EEA76AFE
:1025300066EEC76AA5EE476AE5EEA76A20EE070ACF
:1025400087ED056AC7ED066A83ED007A29EE088AF1
:1025500026F0D8F969EE288AD7ED0E5AD7ED176A1A
:1025600097ED091AD7ED121A97ED0F5A97ED187AD1
:1025700097ED0A2AD7ED132A97ED0D6AD7ED167A53
:1025800097ED0C3AD7ED0B3A97ED154AD7ED144A73
:10259000E1EE085A002209EB8803E8EEA16A00B2D6
:1025A000C4F89C21A2EE085AC4F8A021C4F8A421C2
:1025B000A8EEA27A26EE656A67EEE67AA3EE655A81
:1025C000A3EE886AA6EEC47AE8EEA47A87ED0E5AE6
:1025D000C3ED205A87ED0F6AC3ED406A87ED177A85
:1025E000C7ED187AFEF7FFBB6D4B4FEA890603EB88
:1025F000CC1C5FEA9A0302EB060E264400F07B87B0
:1026000001334FEA03190CEB09000CF110030EF132
:10261000100106F1100213ED024A13ED035A13EDF7
:10262000016A13ED047A51ED024A51ED035A51ED5E
:10263000016A51ED047A64EE244A65EE255A66EE8D
:10264000266A67EE277A1033984242ED024A42ED3D
:10265000035A42ED016A42ED047A01F1100102F1E0
:102660001002D8D1A9F110039C440EEB03021E44C2
:102670001AF0030A3FF463A8BCEC017AF2EC017A89
:1026800067EE277ABAF1010AE6EC017AF4D1FFF796
:1026900056B8444B444AB3F90430DFED447A82FB28
:1026A0000312DB17C3EBA2031BB208EE103AB8EE1D
:1026B000C88A28EE278AB0EE480AF9F717FDF0EE2F
:1026C000408AB0EE480AF9F797FC394BD8780028D1
:1026D00000F094833749B4F98E31B1F9022044F205
:1026E0005066D21AB24240F30F85A2F50C42A03ACE
:1026F0004642964200F3FD848242A8BF0246B1F9E9
:102700000010B4F98CE11344A1EB0E0244F25061C5
:102710001BB28A42A4F88E3140F3EE84A2F50C423B
:10272000A03A964203DC9042A8BF104606460EEB44
:10273000060212B207EE902A07EE103AF8EEE77A98
:10274000F8EEC76A27EEE87A60EE277AA0EE267ADE
:10275000A4F88C21E8EEA67ADFED176A27EE267A38
:1027600067EEA67ABDEEC77AFDEEE77A17EE102A7D
:1027700017EE903AA4F89021A4F89231FDF74ABFE1
:10278000B7EE007A77EE677AF4EEE75AF1EE10FAD8
:1027900088BFF0EE675AFFF762BB00BFF83C00202D
:1027A000743A00207C6E00206766666635FA8E3CBF
:1027B000F4590020505A0020CDCCCC3DBC3900202B
:1027C000D8ED004A9DED0C4ADFF828C665EEA44A14
:1027D000FDEEC73AE4EE064AB0EE674AA4EE854A3B
:1027E00013EE901AF4EEC46AF1EE10FAF0EE444AD9
:1027F00088BFF0EE474AFDEEE44A14EE900A14EE6C
:10280000906A9842A8BF1E468142C8BF0E4604EE99
:10281000906AF8EEE44A012ACCED004A3DF412AA8F
:10282000D8ED044A9DED0D4A65EEA44AE4EE064A51
:10283000B0EE674AA4EE854AF4EEC46AF1EE10FAEF
:10284000F0EE444A88BFF0EE474AFDEEE44A14EE4B
:10285000900A14EE906A9842A8BF1E468842B8BFFC
:102860000E4604EE906AF8EEE44A022ACCED014AE4
:102870003DF4E8A9D8ED084A9DED0E4A65EEA44A5C
:10288000E4EE064AB0EE674AA4EE854AF4EEC46A66
:10289000F1EE10FAF0EE444A88BFF0EE474AFDEE42
:1028A000E44A14EE900A14EE906A9842A8BF1E46BD
:1028B0008842B8BF0E4604EE906AF8EEE44A032A56
:1028C000CCED024A3DF4BEA9D8ED0C4A9DED0F4A6D
:1028D00065EEA44AE4EE064AB0EE674AA4EE854AE5
:1028E000F4EEC46AF1EE10FAF0EE444A88BFF0EE5E
:1028F000474AFDEEE44A14EE900A14EE906A9842BC
:10290000A8BF1E468842B8BF0E4604EE906AF8EE95
:10291000E44A042ACCED034A3DF494A9D8ED104AC8
:102920009DED104A65EEA44AE4EE064AB0EE674A11
:10293000A4EE854AF4EEC46AF1EE10FAF0EE444AD1
:1029400088BFF0EE474AFDEEE44A14EE900A14EE1A
:10295000906A9842A8BF1E468842B8BF0E4604EE51
:10296000906AF8EEE44A052ACCED044A3DF46AA9DF
:10297000D8ED144A9DED114A65EEA44AE4EE064AEC
:10298000B0EE674AA4EE854AF4EEC46AF1EE10FA9E
:10299000F0EE444A88BFF0EE474AFDEEE44A14EEFA
:1029A000900A14EE906A9842A8BF1E468842B8BFAB
:1029B0000E4604EE906AF8EEE44A062ACCED054A8B
:1029C0003DF440A9D8ED184A9DED124A65EEA44A9F
:1029D000E4EE064AB0EE674AA4EE854AF4EEC46A15
:1029E000F1EE10FAF0EE444A88BFF0EE474AFDEEF1
:1029F000E44A14EE900A14EE906A9842A8BF1E466C
:102A00008842B8BF0E4604EE906AF8EEE44A072A00
:102A1000CCED064A3DF416A9D8ED1C4A9DED134AAB
:102A200065EEA45AE6EE045AE5EE257AF4EEE76A7E
:102A3000F1EE10FAC8BFF0EE477AFEF7BAB89FED94
:102A4000E67AFFF7DCB9E549E54A89681268914200
:102A50003FF604A898F800200C3A022A7DF6E2AD71
:102A600094F8942188F80030002A3DF4DBADFFF79C
:102A70002BB8BAF1000F00F03884DFF87C839DEDAD
:102A80000C4AD8ED004A65EEA44AE4EE064AB0EEE0
:102A9000674AA4EE854AF0EE444AB9F1000F06D029
:102AA000F4EE446AF1EE10FAC8BFF0EE474ABDEE0C
:102AB000C77A17EE101ABDEEE47A04EE901A17EEFC
:102AC000100A814200F38D859842A8BF184607EE90
:102AD000100AB8EEC77ADFF81CC3012A8CED007A21
:102AE0003DF4B5A898ED047A9DED0D4A25EE877A60
:102AF000A4EE067AB0EE674AA7EE054AB0EE447A35
:102B0000B9F1000F00F0EC84F4EEC46AF1EE10FAB3
:102B100040F3E68408469842A8BF184607EE100A1C
:102B2000B8EEC77A022A8CED017A3DF490A898EDB0
:102B3000087A9DED0E4A25EE877AA4EE067AB0EE6D
:102B4000674AA7EE054AB0EE447AB9F1000F00F0EB
:102B5000BC84F4EEC46AF1EE10FA40F3B684084681
:102B60009842A8BF184607EE100AB8EEC77A032AA3
:102B70008CED027A3DF46BA898ED0C7A9DED0F4A2E
:102B800025EE877AA4EE067AB0EE674AA7EE054AEC
:102B9000B0EE447AB9F1000F00F08C84F4EEC46A10
:102BA000F1EE10FA40F3868408469842A8BF184612
:102BB00007EE100AB8EEC77A042A8CED037A3DF4CA
:102BC00046A898ED107A9DED104A25EE877AA4EE7E
:102BD000067AB0EE674AA7EE054AB0EE447AB9F13C
:102BE000000F00F05C84F4EEC46AF1EE10FA40F3DA
:102BF000568408469842A8BF184607EE100AB8EE59
:102C0000C77A052A8CED047A3DF421A898ED147A50
:102C10009DED114A25EE877AA4EE067AB0EE674A5A
:102C2000A7EE054AB0EE447AB9F1000F00F02C840B
:102C3000F4EEC46AF1EE10FA40F326840846984296
:102C4000A8BF184607EE100AB8EEC77A062A8CED20
:102C5000057A3CF4FCAF98ED187A9DED124A25EE0A
:102C6000877AA4EE067AB0EE674AA7EE054AB0EE80
:102C7000447AB9F1000F00F0FD83F4EEC46AF1EE7E
:102C800010FA40F3F78308469842A8BF184607EEAB
:102C9000100AB8EEC77A072A8CED067A3CF4D7AF53
:102CA00098ED1C7A9DED134A65EE875AE4EE065ABC
:102CB000E5EE857AB9F1000F00F0D483F4EEE67A00
:102CC000F1EE10FA40F1CE830A469A42A8BF1A46A6
:102CD00004EE902AF8EEE44ACCED074AFCF7B7BFC1
:102CE00001297FF76FAA07EE10EAB8EEC77AC7EEA0
:102CF000876AB1EEE68AFFF767BA012940F363837A
:102D000007EE10EAB8EEC77AC7EE876AB1EEE68A38
:102D1000032F14D0B9F1000F09D007EE909AF8EE06
:102D2000E77AF4EEC87AF1EE10FA00F16A84EA6EFE
:102D300002EB580292FBF8F26A62FFF711BAB0EEAA
:102D4000480A059325F0DEFD059B00B2E2E7012964
:102D500040F33C8307EE10EAB8EEC77AC7EE876A05
:102D6000B1EEE68A032F14D0B9F1000F09D007EEB7
:102D7000909AF8EEE77AF4EEC87AF1EE10FA00F1E4
:102D800040842A6F02EB580292FBF8F2AA62FFF726
:102D900000BAB0EE480A059325F0B4FD059B00B2D9
:102DA000E2E707EE906ADFED0F6AB8EEE77A66EECB
:102DB000A65A9FED0D5A9FED0D6ADFED0D7AA5EE37
:102DC000856A26EEA55AE5EE867AE5EE276A26EEB6
:102DD000870AFFF70DB800BF00000000D01C0020DC
:102DE000E439002084F9223F92E741B99730083C4A
:102DF00015A82ABEBC390020B0550020E24B9FED3B
:102E0000E36AB3F90020B3F9023007EE902A06EE28
:102E1000903AF8EEE77AF8EEE66A27EEE87A60EEA6
:102E2000277AA0EE267AE8EEA67A27EE067A67EEF3
:102E3000867A97E4D4F8BC6153003EB1991800EB50
:102E4000810176784978B142BDF4F5A8134400EBCE
:102E500083030022C4F8BC31A4F81022C4F8142261
:102E6000FDF7E9B8D8ED006ADDED0C4A65EEA66A1B
:102E7000E4EE866AF0EE674AE6EE854AFDEEE46A25
:102E800016EE90EA714500F34A819E45A8BF9E4622
:102E900006EE90EAF8EEE66A002E00F0EA84DFF82B
:102EA00014C3012ACCED006A3CF4D1AED8ED046A1B
:102EB000DDED0D4A65EEA66AE4EE866AF0EE674A3D
:102EC000E6EE854AFDEEE46A16EE90EA714500F3FF
:102ED00023819E45A8BF9E4606EE90EAF8EEE66A7C
:102EE000002E00F09E84022ACCED016A3CF4AFAEC5
:102EF000D8ED086ADDED0E4A65EEA66AE4EE866A54
:102F0000F0EE674AE6EE854AFDEEE46A16EE90EAD8
:102F1000714500F310819E45A8BF9E4606EE90EADB
:102F2000F8EEE66A002E00F06184032ACCED026A16
:102F30003CF48DAED8ED0C6ADDED0F4A65EEA66A65
:102F4000E4EE866AF0EE674AE6EE854AFDEEE46A54
:102F500016EE90EA714500F3EB809E45A8BF9E46B1
:102F600006EE90EAF8EEE66A002E00F07784042A76
:102F7000CCED036A3CF46BAED8ED106ADDED104A7F
:102F800065EEA66AE4EE866AF0EE674AE6EE854AEA
:102F9000FDEEE46A16EE90EA714500F3C6809E45A8
:102FA000A8BF9E4606EE90EAF8EEE66A002E00F014
:102FB0004A84052ACCED046A3CF449AED8ED146A83
:102FC000DDED114A65EEA66AE4EE866AF0EE674A28
:102FD000E6EE854AFDEEE46A16EE90EA714500F3EE
:102FE000A1809E45A8BF9E4606EE90EAF8EEE66AEE
:102FF000002E00F04984062ACCED056A3CF427AE89
:10300000D8ED186ADDED124A65EEA66AE4EE866A2E
:10301000F0EE674AE6EE854AFDEEE46A16EE90EAC7
:10302000714500F38B809E45A8BF9E4606EE90EA50
:10303000F8EEE66A002E00F0E483072ACCED066A7B
:103040003CF405AED8ED1C6ADDED134A65EEA65AD8
:10305000E4EE865AE5EE857AFDEEE77A17EE902AE1
:10306000914203DC9A42A8BF1A46114607EE901A15
:10307000F8EEE77A002E7FF44EA8059B002B7FF434
:103080004AA8049B5B45B8BFF0EE477AFFF743B808
:1030900077EEC76AF0EE477AFEF76EBCBEF83430C2
:1030A0009FED3B7A07EE903AF8EEE77A394B67EE00
:1030B000877AC3ED007AFCF723BD374B1E6816F004
:1030C00080567EF4BFAEFEF7B8BE9FED340A344E94
:1030D00025EE800A25F016FCD4F8B071F080FCF7DC
:1030E000FDBB3049FCF765BD2F4A30481146FEF75D
:1030F00015BB3246FFF703BB2D498A42BCBF02F520
:103100000C42A032FFF70DBB294EB242BCBF02F504
:103110000C42A032FFF7ECBA06EE901ADEE606EE9D
:10312000901AB7E606EE901A60E706EE901A3BE7B3
:1031300006EE901A16E706EE901AF1E606EE901AE1
:1031400076E791ED000A06930592049125F0DAFBEB
:10315000DFF864E0DFF864C0DEF8ECE0104E8CFBD2
:103160000E3C4FEAEE7ECEEBAC1E07EE90EAF8EE98
:10317000E77A3080FDEEE77A04A917EE900A0EC9CF
:103180007080FCF71BBD00BF505A0020CDCCCC3D59
:103190006F12833A94000020686500200000C84246
:1031A000F05A0020E85B0020F43B00209021002032
:1031B000B0B9FFFFBC39002080160020D34D62104B
:1031C00005F02CFADF4BE04E93F80080059B99F850
:1031D0000020D4F8B071C01AB080FEF7ABBB05F088
:1031E0001DFAD84BD84E93F80080059BC01A70800A
:1031F000FEF786B905F012FA059BD34ED4F8B491C8
:10320000D4F8B071C01A7080FEF719BB07EE906A4F
:103210009FEDCE7ADFEDD86A84F88461F8EEE77A24
:1032200067EE877A37EEA67ABDEEC76A16EE103AD9
:103230002033402B40F26581DFEDC56AC54BBDEE02
:10324000E77AC3ED016A17EE103A2033402B00F203
:1032500055819FEDCA7AF4EEC77AF1EE10FA40F389
:103260001782DFEDBD5A9FEDBD6A01E0F0EE477AAF
:10327000F4EEC67AF1EE10FA37EEE57AF6DCDFED21
:10328000C47AB4EEE77AF1EE10FA40F15D82DFED38
:10329000B25A9FEDB36A01E0B0EE677AB4EEC67A37
:1032A000F1EE10FA77EE257AF6D49FEDB37AF4EECC
:1032B000C77AF1EE10FA40F398819FEDB07A77EE7D
:1032C000677A67EEA75A9FEDAE5A9FEDAE6A9FED03
:1032D000AE7AA5EE856A27EEA55AA5EE867AE5EECA
:1032E000077AC4ED627AFDF79DBDFDEEC74A0DF188
:1032F000300E9A46DFF878C2DFF8788214EE901A22
:103300000EEB82024B4606E07245E8EC014A0CF1F6
:10331000100C3CF49CACDCED004ABEEC014A65EEBE
:10332000A44AE6EE044AB0EE674AA5EE244AF0EE5F
:10333000444A33B1F4EE446AF1EE10FAC8BFF0EE3D
:10334000474AFDEEE44A14EE909A494504EE901A7D
:1033500004DCD145A8BFD14604EE909AF8EEE44AC9
:10336000002ED1D105980028CED104985845B8BF79
:10337000F0EE474AC8E77B4A126802F59C520832D1
:10338000C4F8982198F80020012A7DF44BA994F8FC
:103390009421002A7DF446A9032B00F0ED8124F04E
:1033A00079FF012384F89431FDF73CB96E4B1B780B
:1033B000032B00F057810023FEF732BF6B4800F16A
:1033C000800EFEF79DBA9FED628AA1E49FED608AB0
:1033D000C8E4DFED6A7AF4EEE76AF1EE10FA40F342
:1033E0001D82DFED5D5A9FED5D6A01E0F0EE676AD8
:1033F000F4EEC66AF1EE10FA76EEE57AF6DCDFED71
:10340000646AF4EEE67AF1EE10FA40F10482DFED40
:10341000525A9FED536A01E0F0EE667AF4EEC67AF6
:10342000F1EE10FA77EEA56AF6D4DFED537AF4EEFA
:10343000E76AF1EE10FA04DDDFED507A77EEE66A26
:10344000B5E4DFED527AF4EEE76AF1EE10FA44BF2C
:10345000DFED4F7A77EEE66AA9E408981BF034F8BE
:10346000FEF79ABBFDEEE77A17EE902A8A42FFF646
:1034700031AC2AE4BDEEC77A17EE100A8842BFF6D7
:1034800003AC07EE101A04E4BDEEC77A17EE100A7B
:103490008842BFF6D4AB07EE101AFFF7D5BBBDEEDE
:1034A000C77A17EE100A8842BFF6A4AB07EE101ACF
:1034B000FFF7A5BBBDEEC77A17EE100A8842BFF62C
:1034C00074AB07EE101AFFF775BBBDEEC77A17EEA7
:1034D000100A8842BFF644AB07EE101AFFF745BB4F
:1034E000BDEEC77A17EE100A8842BFF614AB07EE9E
:1034F000101AFFF715BB7246FFF7BAB8DFED147A62
:10350000EFE6F4EEE67AF1EE10FA40F3C780DFED75
:10351000125A9FED126A01E0B0EE667AB4EEC67AF6
:10352000F1EE10FA77EE656AF6DC9FED197AF4EEAB
:10353000C76AF1EE10FA40F1AE80DFED075A9FED59
:10354000086A29E0EC5A0020F05A002035FA8E3C37
:103550000000000094000020DB0FC940E4CB1641BE
:10356000E4CB16C18C790020D86000209021002087
:10357000B0550020BC390020DB0FC93FDB0F4940AC
:1035800092E741B99730083C15A82ABEDB0FC9BFA6
:10359000DB0F49C0F0EE476AF4EEC66AF1EE10FAAE
:1035A00036EEA57AF6D45FED0C6AB4EEE67AF1EE6B
:1035B00010FA2BDD5FED0F6A36EEC77A67EE075A19
:1035C0001FED115A1FED116A5FED116AA5EE856AB4
:1035D00027EE255AE5EE866AA5EE267AF0EE476AD2
:1035E0002CE607EE101AFFF774BA1FED187AF4EE06
:1035F000C77AF1EE10FA44BF1FED1B7A77EE677AB7
:103600005FE6F080A5F8B480FCF71CBD5FED216A91
:10361000B4EEE67AF1EE10FA44BF5FED236A36EEBF
:10362000C77ACBE7F8F76EFE00283EF4E5AAFEF76E
:1036300090BB802020F0ECFF08B106F0A5FC24F040
:1036400029FEFEF792BB24F0AFFF00283EF4D4AA77
:10365000934A944B12681A600A2388F80030B378B2
:10366000FEF7F9B907F0CEFBFCF7E5BC94F8E831BA
:10367000002B7BF4D5ACFBF7C0BC8B49B3780A6058
:103680004FF0FF324A60072288F80020FEF7E3B9C6
:10369000B0EE677AF3E5B0EE667A84E7F0EE476A5B
:1036A00043E7824BD3ED007AB1EE677AB4EEC7CA36
:1036B000F1EE10FA5DD4B4EEE7CAF1EE10FA88BF6D
:1036C000B0EE67CA7A4BC7ED00AA1B689342BBF6FF
:1036D00099ABFCF7CEBD774A774B10681B689847CB
:1036E000079BDBED007A93ED007A744BD7ED006A0F
:1036F00093ED006A724B83ED020A724B67EE277AF4
:103700002B4427EE8B7AD3ED007A67EE277AF0EE22
:10371000665AECEE275AB1EE467AB4EEE57AF1EE4F
:1037200010FA4BDD684B1B78012B02D0192B7BF470
:10373000A8ABDFED667AB4EEE7CAF1EE10FACCBFC3
:1037400001230023FBF7A8BBF0EE477AADE5DFF8D5
:103750009091D9F8000006F0F5FB5D4B1B78002234
:10376000022BC9F800207EF4FFA907F07FFAFEF7CC
:10377000FBB9B0EE47CAA5E7802020F049FF00283A
:103780007CF450AF0BE6132B05D1B0EE480A25F0C0
:10379000B9F8AAF80000B0EE480AD5F878374D48D5
:1037A00098474D4B1B78132BB0EE408A7BF413AA3D
:1037B00025F0A8F8AAF80200FBF70DBAB4EEE56A06
:1037C000F1EE10FA8CBFB0EE657AB0EE467AA9E75A
:1037D00045201AF0EFFCFF201AF0ECFC3F481AF0ED
:1037E0005FFC48461AF0E6FCFEF768B90598002829
:1037F0007FF49BAB04985845B8BFF0EE476AFFF7DB
:1038000094BB059800287FF418AC04985845B8BFBD
:10381000F0EE476A11E4F0EE676A06E6F0EE667ACB
:10382000EDE5059800287FF45EAB04985845B8BFD5
:10383000F0EE476AFFF757BB1AF80330002B7EF40F
:10384000DBA9FEF777BA059800287FF4B2AB04989D
:103850005845B8BFF0EE476AFFF7ABBB05980028A4
:103860007FF485AB04985845B8BFF0EE476AFFF780
:103870007EBB059800287FF412AB04985845B8BF6A
:10388000F0EE476AFFF70BBB059800287FF4B3AB57
:1038900004985845B8BFF0EE476AFFF7ACBB00BFCD
:1038A000F8630020F0630020886500207C5500202C
:1038B000605500202C450020404500208055002008
:1038C00088390020185500207C3F002000009642D7
:1038D000DC390020D4760020EC5A0020DCDB030821
:1038E000405E00202DE9F04F2DED028B984B994A58
:1038F0001C7893B000F59C412031814607911160FE
:10390000002C00F0C386944A1268904240F28A80EC
:10391000924A93491768934DDFF888B20592013CAB
:1039200003911C7007F48057002F40F08880039BA0
:103930005B7D002B40F02986059B1B681E0401F16E
:103940004B81894B99459BF8023000F2FB84002B98
:1039500040F0FC84854B0693059B1F6817F4805943
:1039600040F0B785039BB5F906605B8B9E42B4BF00
:10397000002601267E4B1B6813F0805369D0069AFF
:10398000127812F001026AD003987A49408C91EDC6
:10399000037A049107EE900AF8EEE77AB4EEE77A3C
:1039A000F1EE10FA81F2DF81002E60D1724C94F8B2
:1039B000A01000295BD171487149006890F82D0072
:1039C00000240C604C608C606E49002850D1087057
:1039D000002A51D0F8064FD56B4A1278D1064BD445
:1039E000B9F1000F48D1002B46D17A0244D4674B7D
:1039F0001B78002B02F00380654B9B78002E42F071
:103A0000CF803BB1634A644B12681B689B1A002B42
:103A1000C2F2AB801020584C07F010FA012384F852
:103A2000A13029E04D4B4E4A1F68059307F480579B
:103A300003924C4DDFF86CB1002F3FF478AF0021BA
:103A40004B48F8F729FC00287FF471AF14F074FE9E
:103A50006DE77C0293D4069A127802F00102464C7C
:103A6000002184F8A01043490491002EA3D04549B9
:103A700001200870002AADD1484B1A78002A50D195
:103A80000399B5F900E0488B898BB5F90240704580
:103A9000B4BF8027002747F040037145D8BF3B469D
:103AA0009B0843F08007A042B8BF3B4643F0400765
:103AB000A142C8BF3B469B08B5F90440B5F9067062
:103AC00043F0800EA042B8BF734643F0400EA142BF
:103AD000C8BF73469B0843F0800E274C8742C8BF7F
:103AE000734643F0400E94F8A2C08F42B8BF7346AD
:103AF0009C4501F02283A4F8A42084F8A620234941
:103B000084F8A2300F78002F01F083825F2B01F040
:103B1000EE826F2B01F08381069B1B78DE0741F15B
:103B20004781059B1B6803F00403002B40F0C5860A
:103B30000DF140081A4C0022C8F8042004F1500985
:103B4000109240F6330A192740F283362FE000BF67
:103B50009C370020E4350020983700202C6A002094
:103B6000906B0020A8600020404B4C005C5B002064
:103B700068650020E85B0020AC230020305C00205A
:103B800094390020782300209C6E0020E01C002047
:103B9000D06500208C7900203C570020085E002072
:103BA000EC390020DC60002004344C4520D0A278A1
:103BB000E3789A4217FB0261F6D26278043217FB6F
:103BC000036335F912205245A8BF5246B2F5617F12
:103BD000B8BF4FF461728A42E6DD9A42E4DC217894
:103BE0002429E1D840460434F8F746FB4C45DED1A1
:103BF000644A654B177898E8030083E80300002FB8
:103C000000F0E485614B08935F480121F8F744FB1D
:103C1000002840F0A7829BF80330002B40F0A282DE
:103C20005B4B07935B4E33881CB224F00104A7B2B0
:103C3000BB42378001F02F80574C4FF002080E2016
:103C40004FF014094FF0FF0A84F8008084F80190C7
:103C500084F802A007F0F2F841464B483788F8F79D
:103C60001BFB002841F00F8227F002039BB2BB42EE
:103C700033800AD0484B1421FF2202240E201C70EE
:103C800059709A7007F0DAF83788444B444A19782B
:103C900050680A93BC0708BF81F00201C1F34001DC
:103CA000099202F029FF24213748F8F7F5FA30B9D4
:103CB000069A1378590744BF23F004031370079B37
:103CC0001B6813F00A0F1DD005212F48F8F7E4FAFE
:103CD000002801F015803488630741F140812A48AB
:103CE0000621F8F7D9FA002800F0F787670641F1B6
:103CF0002E8107212448F8F7CFFA002840F0668487
:103D0000079B1B68980600F1718437881E480C21B8
:103D1000F8F7C2FA002800F0688247F48073BB42CB
:103D2000338009D01C4B02201421FF2218700E2072
:103D300059709A7007F082F81A4B1B78082B00F024
:103D400060820E2B00F05D82059B1B6858055CD5D8
:103D5000154B1B79002B00F0208114210A48F8F73D
:103D60009BFA002840F01E8119F0C6FD012006F0E4
:103D700053FF002849D0DFF8349000244FF0CC0ADC
:103D800019E000BF4F59002068650020989E002070
:103D9000986E0020D26000205856002056790020EE
:103DA00058790020E8390020D85B00206892002074
:103DB000DCB2022C29D80AFB04F8631C59F80870FD
:103DC000002FF5D1C378D04A90F9020052F8233081
:103DD00001970322009201213A4606F0EDF80346CE
:103DE00004EB440000EB0010079353B1394609EB94
:103DF0008000CC2226F091FE079B49F80830013460
:103E0000E4B222F0A3FC0028D3D1069B1C7814F066
:103E1000010400F02682BD4B01221A70089BB5F9FF
:103E200006101B68BA485A8901279142077080F230
:103E3000FE81B84B4FF07E521A60B74A039BB5F92A
:103E400000E01F8B92F90430107892F801C0002B2B
:103E5000AEEB070314BF01224FF0FF32002BB8BFB7
:103E60005B42B3F5FA7FA8BF4FF4FA73984280F231
:103E7000DB811B1A07EE903AF8EEE77A049BBE4509
:103E8000C3ED007A03DAF1EE677AC3ED007AB5F993
:103E900002E0AEEB0703002BB8BF5B42B3F5FA7F3D
:103EA000A8BF4FF4FA73984280F29C811B1A07EE68
:103EB000903AF8EEE77A049B7745C3ED017A03DD8B
:103EC000F1EE677AC3ED017AB5F90400C31B002B4C
:103ED000B8BF5B42B3F5FA7FA8BF4FF4FA736345EE
:103EE000CCBFA3EB0C03002302FB03F307EE903AD5
:103EF000049A059BF8EEE77AB842C2ED027ABCBF9D
:103F0000F1EE677AC2ED027A1A6812F4805200F07C
:103F10004681B1F5FA6F814BA8BF4FF4FA61B1F554
:103F20007A7F1878B8BF4FF47A71A1F57A710028BA
:103F300040F04E817A4D7B4885FB013ECB17C3EBA9
:103F40006E1303F1010E6FF0630C30F91EE030F9CF
:103F500013000CFB0313AEEB000103FB01F385FB25
:103F60000315DB17C3EB651303441BB207EE903A4E
:103F7000049BB8EEE78A83ED038A002A40F0C883E9
:103F800033885A0624D4002C40F0B08023F0A7FADE
:103F900013B0BDEC028BBDE8F08F069B1B78D907F0
:103FA0007FF5E2AE3C2020F033FB00283FF42DAF3C
:103FB00005F0EAFF3C2020F093FA00283FF425AFFB
:103FC00005F0E2FF3C2020F08BFA0028F0D11CE73E
:103FD000554B564AB3F904305549DFED566A098806
:103FE0009FED557A82FB0302DB17C3EBA2035B1A3A
:103FF0001BB207EE903AF8EEE77A67EEA67A77EE14
:10400000876ABDEEE66A16EE103A2033402B40F286
:10401000AE87BDEEE77ADFED496A17EE103A20333E
:10402000402B00F2F2879FED467AF4EEC77AF1EE6C
:1040300010FA41F35483DFED435A9FED436A01E0E8
:10404000F0EE477AF4EEC67AF1EE10FA37EEE57A42
:10405000F6DCDFED3E7AB4EEE77AF1EE10FA41F1EC
:104060003A83DFED385A9FED3A6A01E0B0EE677AA5
:10407000B4EEC67AF1EE10FA77EE257AF6D49FED1B
:104080002E7AF4EEC77AF1EE10FA00F384869FEDF3
:10409000317AF4EEC77AF1EE10FA44BF9FED2B7A35
:1040A00077EE677A67EEA75A9FED2B5A9FED2B6A42
:1040B0009FED2B7AA5EE856A27EEA55AA5EE867AA6
:1040C000E5EE077A049A92ED016AD2ED005A27EEE6
:1040D000C67A65EEA77AA5EEA67AE6EE267A82ED96
:1040E000007AC2ED017A002C3FF450AF0A9B197898
:1040F000099B01F00101186802F0FEFC13B0BDEC51
:10410000028BBDE8F08F00BFBCD103085D5B0020CF
:10411000A822002054230020AC650020AC250020FC
:104120001F85EB519C9E00207C6E002067666666B2
:104130003857002035FA8E3CDB0FC93F00000000E5
:10414000DB0F4940DB0FC940E4CB1641DB0F49C010
:10415000E4CB16C1DB0FC9BF92E741B99730083CE9
:1041600015A82ABEB54B07931B6899077FF55AAD72
:10417000B34E3788FA073FF577AD47F001039F420A
:1041800033803FF471ADAF4B022214211A700E2020
:10419000FF2259709A7006F051FE378864E5039B40
:1041A000588B8142C0F28A84B1F5FA6FD4BFC0EB5C
:1041B0000101C0F5FA614FF47A7303FB01F1A24BE0
:1041C0001D78C0F5FA60B1FBF0F1002D3FF4B2AEFE
:1041D0005B789E4801FB03F380FB0301DB17C3EB15
:1041E0006111A7E6DFED9A7A65E627F480739BB24A
:1041F000BB4233807FF496AD964B1B78082B7FF43F
:10420000A0AD328822F040039BB29A4233803FF443
:104210009BAD8C4B02201421FF2218700E20597088
:104220009A7006F00BFE8FE5DFED897A26E6B1F590
:10423000FA6F80F24684187A8B1A03FB00F3C2F5FA
:10424000FA6293FBF2F3C3F1640307EE903AF8EEDF
:10425000E77A9FED817A814B67EE877AC3ED007A2A
:10426000EBE57F4B1B780793002B7FF4D7ADDFF88E
:1042700020A2DFF820921AF8030C99F8008051462A
:10428000AAF1030722F0A8FE002800F04B84079B48
:10429000B8F1000F53D107F10801787922F09CFEA4
:1042A000002841F091826F49B87A22F095FE0028EB
:1042B00000F04C84B8F1020F41F089826A49F87B22
:1042C00022F08AFE002841F085826849387D22F07C
:1042D00083FE002800F04C84B8F1040F41F07D8289
:1042E0006349787E22F078FE002841F079826149A6
:1042F000B87F22F071FE002800F04C84B8F1060F60
:1043000041F05F825C4997F8230022F065FE0028A7
:1043100040F0F887594997F8280022F05DFE002800
:1043200000F04C84B8F1080F40F0FD87544997F82D
:104330002D0022F051FE00283FF470AD09231A46EB
:1043400000F0E2BF13B901238BF802304D4B069306
:104350001B201F789BF8216022F068FE012E07F0D9
:104360000109824600F0BF8607F0020304939BF820
:104370002030DFF82481444C052B00F29D80DFE8DB
:1043800013F08D0050000600DE000201C000012E77
:1043900004BF05238BF82030B9F1000F00F06181D4
:1043A000039B3A4FB3F91810B8F80030002261F3BC
:1043B0000F0263F31F42002361F30F0361F31F43F6
:1043C0006A603968DBF814202B608A42C0F0B2843E
:1043D000012E41F0DA8303229BF820300492CBE7D0
:1043E00022F050FE012808D1284FB8F802303A6870
:1043F000642101FB0323CBF81030BAF1000F04D085
:1044000098F80630002B40F09180012E54D01F4FB9
:10441000DBF810203B689A42C0F0058701238BF837
:104420002030012E6DD098F80730012B00F0238149
:1044300012F094FF9BF820309EE700BF986E00209A
:10444000D260002058560020AC2500201F85EB517B
:1044500000000000E83900200AD7233C5423002044
:104460005D5B0020E4540020E9540020EE5400205D
:10447000F3540020F8540020FD5400200255002081
:10448000075500205C5B0020006100208C79002033
:10449000DA5400209C00002050560020B9F1000F93
:1044A0009ED14FF48060BAF1000F00F0128406F044
:1044B0000DFE0023CBF81030049B002B3FF44CAAD8
:1044C000049806F0BBFC059B1F6817F480593FF465
:1044D00049AA1D21A548F7F7DFFE00287FF442AA6C
:1044E000A34A039BD2881B8BB5F90660991A8E42AA
:1044F00040F3968613449E42B4BF00260126FFF780
:1045000039BA9C4F3A68B8F80230642101FB0323A2
:104510004FF480600022CBF810308BF820208BF80D
:10452000032006F0BBFD9BF8203025E712F016FFB4
:1045300003224FF47A738BF82020CBF81C308D4F78
:10454000238843F00203238014F0F6F83A68DBF87E
:104550001C3013440422CBF818308BF82020012E95
:1045600040F06C863B68DBF818209A42A4D2824B5C
:10457000187818B922F05AFD00289DD1238823F01D
:1045800002032380BEE77B4FE9E7039A013BD27D1C
:1045900035F91330002A40F0C883A3F57A73B3F5D8
:1045A0007A7FA8BF4FF47A7323EAE37307EE903A59
:1045B0009FED727AF8EEE77A67EE877A704AFCEE42
:1045C000E77A17EE903A1380FFF7BBB96D4B6E494F
:1045D000B3F90420079B6D481B6881FB0241D21789
:1045E000C2EBA102028098067FF58FAB684B1B7867
:1045F000990706D5DFF8C48198F81430042B00F22F
:104600002586378817F0300F3FF480AB102006F076
:1046100045FD202006F042FD5E4B378800221A70CF
:104620005D495E4A5E4C5F4800230B605E49236033
:104630004FF0000E036053609361C2F800E0C2F8CF
:1046400008E0C2F814E0C2F81CE0C1F800E04B60DA
:10465000C1F808E0C1F814E08B61C1F81CE0FFF775
:1046600055BB444F3B6847F230520323CBF81C2024
:104670008BF8203064E712F071FE032240F6B83365
:104680008BF82020CBF81C303A4F59E7474F3B7846
:10469000002B01F04C80464BDFF82481DFF824B179
:1046A000DFF824A1039345465E46049099460EE048
:1046B00019F804109847032C28DC88B93B782AF8AD
:1046C000020F01349C4205F1040580F21A81072C87
:1046D000E1B23046DBF80430EADD984700B2EDE79E
:1046E00038F824206B88801A4FF47A719B1A01FBEA
:1046F00000F040F6CA0290FBF3F00844904240F20A
:10470000EE23A8BF10469842B8BF184600B2D5E7BE
:104710001D211648F7F7C0FD00283FF431AC9BF887
:104720000330002B7FF42CACDFED227A224938EEE7
:10473000678AC7F5FA63FDEEC87A1BB2CDED037A3E
:10474000BDF90C20120381FB0201D217C2EBA112AA
:1047500003FB02F343F30F333B4407EE903A049B11
:10476000F8EEE77AC3ED037A0AE400BF686500203B
:10477000385600208C790020E01C0020AAF1823FEE
:10478000D06000207C6E0020676666663857002087
:104790009C6E002060590020505A0020005A0020D2
:1047A000202300201C230020285A0020F03700205E
:1047B000906B002000007A44D34D6210A06E002060
:1047C00008380020D8350020AA230020DFF844A3B1
:1047D000DFF84483BE4C0AF15A064FF001095146F6
:1047E0001AF8010C22F0F8FBF8B19AF804009AF8D4
:1047F00002309AF803E000EB400104EB8101013B39
:10480000D1F8B42003EB4303434493420DD094F812
:10481000E02081F8B0E009FA00F022EA0000C1F8D7
:10482000B430C1F8B87084F8E0000AF1060A5645C1
:10483000D5D1A84B08931946A74AA84BA84C09689C
:104840001B78D2F8009009910793A4F1B00A0026D2
:1048500063685BB31F784FB3A268A9EB0202002A1A
:104860000ADB9AF8E0200121B14022EA010209F5B1
:10487000FA718AF8E020A160079ABAB122785978D3
:104880000432D2B2002940F07482039935F9122023
:10489000098B01F1C800824240F394849AF8E01039
:1048A0009A7841FA06F3DB0740F127850136042E9A
:1048B00004F10C04CCD1FFF7A7B9854C94F8AA30C9
:1048C00053B1069B1B78DA0706D5039BB5F9062082
:1048D0005B8B9A4200F3E68411218248F7F7DCFCF7
:1048E000002800F02E8294F8AE302BB994F8A8304E
:1048F00013B93223A4F8AC30012384F8AE30FFF7AB
:1049000017B9DDF81090784A05921146774A096880
:1049100042F2010AA2FB092B11EA0A0A4FEA9B1B89
:1049200000F00B82724D73486C4C734A95F800E0AE
:10493000007884F800E01070BEF1000F04D06E4AD9
:1049400092F800E08EF0010E614C0F2084F82400F4
:10495000002B00F06B83694B0C931B780B931E4666
:104960003B78039F664AB7F824C0DFF8B0810A900D
:104970003D46FF8C09973746A2FB0662520802EBC0
:1049800042022D8B0E95BA1A94F825500495D2B296
:1049900001F4805108925B4DCDF834900BF596727E
:1049A000DDF810900F91CDF810E004F128060020FA
:1049B00006926746A646049A002A00F06B823EF9EA
:1049C00010101FFA81FCBC454FEA400203D3099C3A
:1049D000A44540F2A38258F820108B4580F06382F2
:1049E000A95EBAF1000F40F0788201309842A952D6
:1049F00006F10606DFDB0A98434A8EF82400494692
:104A00000F288EF825100CBF01210021DDF834900D
:104A1000117000F01183DFF808B13C4E2E4F34883E
:104A20003868DBF80810DBF80420CBF80C0044F001
:104A30000404401A90422F4F34802F4C4FF0010154
:104A400088BF00223970217088BF8BF82120002B8D
:104A500000F00783059A039917682D4EB1F824C01A
:104A6000B1F818E0274817F48057344640F01D830A
:104A700039460EE0627802EB820202EB820202F219
:104A8000EE2292B201318B4220F8022B04F1020493
:104A90000ED016F81120002A00F04482022AE9D034
:104AA0000131028820F8022B8B4204F10204F0D17C
:104AB0000C9A137801331370FEF736BF1146FFF7D7
:104AC0007EBB1B7AC3F1640307EE903AFFF7BFBBCE
:104AD000AC230020989E00208C7900207960002073
:104AE0005C240020686500202C6A0020D34D6210F1
:104AF000B435002040010020410100209D370020F6
:104B0000ABAAAAAAA8600020483A002000610020B1
:104B10003C380020F1530020E0B30308A037002008
:104B2000DC6000200AF10501787922F055FA0028AE
:104B30003FF4B9ABB8F1010F40F0468607F10D0123
:104B4000B87A22F049FA002840F04186C049F87B43
:104B500022F042FA00283FF4B8ABB8F1030F40F05E
:104B60003986BC49387D22F037FA002840F0358676
:104B7000B949787E22F030FA00283FF4B8ABB8F19A
:104B8000050F40F02D86B549B87F22F025FA0028A0
:104B900040F01786B24997F8230022F01DFA00284A
:104BA0003FF4B8ABB8F1070F40F0AC83AD4997F8CC
:104BB000280022F011FA002840F0B583AA4997F89E
:104BC0002D0022F009FA00283FF428A9B8F1090FB6
:104BD0003FF424A9FFF7B2BBA44CD4F88830A9EB6A
:104BE0000303002BFEF6ADAEA14A94F88C30517C45
:104BF000079AC4F8882001339E4A039E32F8112098
:104C0000B17D03F00F0384F88C30234492B292FB01
:104C1000F1F283F8902094F8901094F8912094F891
:104C2000923094F89C000A4494F89310134494F83A
:104C30009420194494F895300A4494F8961013443B
:104C400094F89720194494F898300A4494F89910ED
:104C5000134494F89A20194494F89B300A4413445E
:104C600094F89D1094F89F20184494F89E300144C5
:104C70000B441A4442F30B12642AF17DA8BF64224C
:104C800013B209B1C2F1640307EE903A9FED7A7A4C
:104C9000F8EEE77A90E402217848F7F7FDFA002869
:104CA0003EF4E2AF3480BB073EF5EFAF47F00203BE
:104CB000BB4233803EF4E9AF714B022214211A70DB
:104CC0000E20FF2259709A7006F0B8F83788FEF768
:104CD000DCBF06F0E3F9FFF7ECBB24F040039BB226
:104CE000A34233803FF405A8654B022214211A70B9
:104CF0000E20FF2259709A7006F0A0F8FEF7F9BF57
:104D0000338823F00404A4B2A34234803EF4E7AF16
:104D10005B4B022214211A700E20FF2259709A70E8
:104D200006F08CF83488FEF7DABFC3F53B6308332E
:104D30001BB232E40323049395E4524A92F800E054
:104D4000FAE594F8A830002B3EF4F2AE069B1B78EF
:104D500013F001037EF4ECAE012284F8A83084F84D
:104D6000A920FEF7E5BE414C012184F8A010FEF712
:104D70007EBE012900F072849AF8E0200123B3403E
:104D800001361343042E8AF8E03004F10C047FF45A
:104D90005FADFEF739BF9FED3C7A77EE677AFFF79C
:104DA00081B9069B394A1B781060DB0700F18882C5
:104DB00094F8A60000287EF4B4AEB4F9A430322BE7
:104DC0007EF7AFAE94F8A2200121572A84F8A610EE
:104DD00000F00985059B1B6813F0040302D05A2AD2
:104DE00000F04E865D2A00F02B855B2A00F080855E
:104DF0005E2A00F0E785562A00F0F285972A00F037
:104E0000E585A72A40F02B852149059B0A781B6878
:104E100042F004020A7003F00403FEF786BEB2F506
:104E2000FA7FFEF67EAE94F8A620002A7EF479AED4
:104E3000069B1B780121DF0784F8A61000F1F88497
:104E400012F0E0FD059B1B6803F00403FEF76DBE46
:104E5000E9540020EE540020F3540020F8540020C0
:104E6000FD5400200255002007550020AC230020EF
:104E7000107900202C79002014AE234168650020B1
:104E80005856002079600020DB0F49404057002031
:104E90009C6E0020002F3FD058F820108B454FEA21
:104EA0004002FFF49DADB149B04C895C04EB020CAB
:104EB000002900F0DB80022947D19CF8011001EBAA
:104EC000810101EB810101F2EE2189B2032833DD7A
:104ED00009B2BAF1000F3FF488AD089C26F814100F
:104EE000B9F1000F03D10B9C022C7FF67EADB6F812
:104EF00000907188B6F804C049448C449C490FFA6C
:104F00008CFC81FB0C419B4CA1EBEC7124F802C0A2
:104F100009B24FF0010968E539464200069C48F89D
:104F200020405EE5CAB2022A04D9032A7FF4B8AD54
:104F30006246A7E57246A5E5012404FA00FC0A9C36
:104F400024EA0C0409B20A944BE5A95ABEE744F0DE
:104F50004003A34233807FF4C7AEFEF7CABE44F0DD
:104F600004039C4233807FF4D3AEFEF7B8BEF4EE68
:104F7000C77AF1EE10FA40F3D783DFED7F5A9FED49
:104F80007F6A01E0F0EE476AF4EEC66AF1EE10FACD
:104F900036EEE57AF6DCDFED7A6AB4EEE67AF1EE2B
:104FA00010FA40F1C883DFED745A9FED766A01E094
:104FB000B0EE667AB4EEC67AF1EE10FA77EE256AB4
:104FC000F6D49FED717AF4EEC76AF1EE10FA40F371
:104FD000A8809FED6E7A77EE666A66EEA65A9FED20
:104FE0006C5A9FED6C6A9FED6C7AA5EE856A26EE91
:104FF000A55AA5EE867AE5EE076ABDEEE77A17EECA
:10500000103A2033402B7FF60EA8DFED647AFFF7CD
:1050100059B839466248F7F73FF900283FF4C1AE66
:1050200084F8A77012F0EEFCFEF776BD5D495E4A8B
:105030000C915E4D012111701B2159480493F7F723
:105040002BF9049B00287FF4E6ACDFF874B1584FCD
:10505000DBF80C203B68CBF808309B1AC82B00F219
:105060006D83059B1F6807F4805721E5C1B20229B3
:1050700040F2F28203297FF468AF0E990F9C002C56
:1050800008BF394622E727F0010292B2BA423280C5
:105090003FF409AE0E2084F8008084F8019084F873
:1050A00002A005F0CBFE3788FDE500210FE0627815
:1050B00002EB820202EB820202F2EE2292B2013194
:1050C0008B4220F8022B04F102043FF4F1AC16F8F5
:1050D00011201AB1022AEAD00288F0E7CAB2032AE4
:1050E000FAD87246EBE700230493FFF740B9B2F514
:1050F000FA7FFEF616AD94F8A630002B7EF411ADC3
:10510000069B1B78012113EA010084F8A61000F029
:10511000238313F011FB059B1B6803F00403FEF7C8
:1051200004BD9FED247AF4EEC76AF1EE10FA44BF95
:105130009FED137A77EE666A4FE71F4A1F491068A2
:10514000B4F9A420C76981FB07018911FF17781AF8
:1051500000F5FF407F3082423EF7D1ACC91B0A44C4
:1051600012B2A4F8A420FEF7CABC00BF3C3800204D
:10517000565555551C240020DB0FC940E4CB164181
:10518000DB0F49C0E4CB16C1DB0FC93FDB0F494041
:1051900092E741B99730083C15A82ABE00000000EC
:1051A000686500209D370020483A0020A860002054
:1051B0008C790020DB0FC9BF58630020D34D6210EB
:1051C000DC600020C8398A425FDA9AF8E0109A78E9
:1051D00041FA06F3D8073FF569AB524201200A9223
:1051E00005F044FF7B1E0A9A162B00F21F81DFE8B0
:1051F00013F0C001E101A7010A02F7011E027A01C2
:1052000065014E01370120011D010A020D011E0238
:105210007A016501F700E100CB008F01B3009D002A
:105220000126FEF7A7BB12F099F8032240F6B83327
:105230008BF82020CBF81C30FFF782B93A68DBF8F6
:105240001C301344CBF81830FFF736B90A2021F090
:10525000EDFE37888146002800F04582FA0640F1CD
:105260003183CF4C94F8F090B9F1000F7EF44EAD3D
:105270000D2005F0E3FD012384F8F0303788B9F103
:10528000000F7FF4CDA9FEF741BD9AF8E03001226E
:10529000B24023EA020309F5FA728AF8E030A2600C
:1052A000FFF704BB0021BF48F6F7F6FF00287FF4A4
:1052B00013AB322384F8AA00A4F8AC30FFF70CBB80
:1052C000B94B1B78002B3EF42CAC9BF80330002B21
:1052D0007EF427AC94F8A7300133DBB2032B84F8BB
:1052E000A7307EF61EACB14B5B7813B9002E7EF46E
:1052F00018AC13F021FAFEF70FBC002A0CBF0120F6
:1053000002206CE707231A4602EB8202174489F851
:105310000030B978787815F07DF8069B1C7804F099
:105320000104FEF77BBD08231A46EDE7DAF8E40036
:10533000DFF87C8290F8361098F802301144642926
:10534000A8BF642121EAE17180F83610002B40F0FB
:10535000398411F0B1F90FE5DAF8E400DFF8508292
:1053600090F8371098F802301144FE29A8BFFE21AA
:1053700021EAE17180F83710002BEAD0162021F0E5
:10538000B3FEDAF8E400E4E7DAF8E400DFF82082BC
:1053900081781144C829A8BFC82121EAE171817030
:1053A00098F80230002BD4D0142021F09DFEDAF8BA
:1053B000E400CEE7DAF8E400DFF8F4814178114444
:1053C000C829A8BFC82121EAE171417098F80230CC
:1053D000002BBED0132021F087FEDAF8E400B8E7F6
:1053E000DAF8E400DFF8C88101781144C829A8BFC1
:1053F000C82121EAE171017098F80230002BA8D091
:10540000122021F071FEDAF8E400A2E7DFF8A081B3
:10541000099898F80230417911446429A8BF6421A1
:1054200021EAE1714171002B40F0B383DAF8E40026
:105430008FE7DAF8E400DFF87881017A98F8023033
:105440001144C829A8BFC82121EAE1710172002BCB
:105450003FF47FAF0B2021F047FEDAF8E40078E755
:10546000DAF8E400DFF84881C17998F80230114495
:10547000C829A8BFC82121EAE171C171002B3FF4FE
:1054800068AF0A2021F030FEDAF8E40061E7DAF8CC
:10549000E400DFF81C81817998F802301144C829B2
:1054A000A8BFC82121EAE1718171002B3FF451AFFF
:1054B000092021F019FEDAF8E4004AE7DAF8E400FE
:1054C000DFF8EC80417998F802301144C829A8BF70
:1054D000C82121EAE1714171002B40F03883112F7E
:1054E0007FF456AF35E7DAF8E400DFF8C4800179DD
:1054F00098F802301144C829A8BFC82121EAE171F7
:105500000171002B40F06283102F7FF457AF20E72A
:105510000998DFF89C8041781144B1F5967FA8BFC7
:105520004FF4967121EAE171417098F80230002B36
:105530003FF47CAF152021F0D7FDDAF8E40008E74E
:105540000999DFF86C800F791744642FA8BF64278E
:1055500027EAE7770F7121F0E1FD98F80230002B80
:105560003FF464AF0320394621F0BEFDDAF8E400D1
:10557000EFE60998DFF8388001781144FA29A8BFCE
:10558000FA2121EAE171017098F80230002B3FF412
:105590004DAF012021F0A8FDDAF8E400D9E600BF04
:1055A000AC2300206865002079600020D0650020D1
:1055B0007E5D00200998DFF8C48481781144642955
:1055C000A8BF642121EAE171817098F80230002BB4
:1055D0003FF42CAF022021F087FDDAF8E400B8E6B2
:1055E0000998DFF89884C17998F80230114481F362
:1055F0000801C171002B3FF419AF052021F074FDA3
:10560000DAF8E400A5E6099BDFF87084997998F848
:10561000020011446429A8BF642121EAE171997153
:10562000002840F09C820D2F7FF4F2AEFEE6DAF8FF
:10563000E400DFF84884C17898F802301144C829A2
:10564000A8BFC82121EAE171C170002B40F095820A
:105650000F2F7FF4C9AE7CE60E9937E435F912209E
:105660009978B2F5617F4FF4966393FBF1F352DBC7
:1056700040F633019142A8BF11460C2FA1F561718C
:1056800091FBF3F100F03881182F7FF475ABC9B2AC
:10569000C8290B46A8BFC823DAF8E400C27DDFB2F0
:1056A00097423FF469AB9A1ADFF8D083C77548BFB9
:1056B0000732D71098F802300137FFB23BB9002FFC
:1056C0003FF45AAB384605F0D1FCFFF755BB182024
:1056D00021F00AFDF3E7F0EE477AFEF7D0BCB0EE1A
:1056E000677AFEF7B6BCFB0600F153810B2021F070
:1056F0009DFC002840F01A81BC0600F15481C84C82
:1057000094F8F030002B3FF4B3ADB9F1000F7EF404
:1057100087AFFEF7FBBA0C2F00F00581182F7FF43E
:105720002BAB00210B46B7E7B0EE667A33E4BD4AF7
:105730000392FFF7E8B8F0EE476A42E4BA4A059BE5
:105740001F68138823F004031380012307F4805794
:105750008BF82130FFF7ACB9B44B1B6813F400335E
:1057600040F029811846B2490E5C0F2E00F10C0062
:105770000ED00133152BF7D1059B1B68FA3A002197
:10578000A4F8A42003F0040384F8A610FEF7CDB912
:10579000A84FD7F800E05800BEF1000F07D0C61898
:1057A00001EB86069EF801E076787645E4D218444F
:1057B000A14EA24B01EB80010020396030801860BF
:1057C000DAE706231A469FE501231A469CE50223E1
:1057D0001A4699E503231A4696E504231A4693E5EB
:1057E00005231A4690E5964B96491A684FF47A734A
:1057F000B3FBF2F3C3EB431203EB8202059B1B687E
:10580000D2001806A1F8B4207EF58DA98E4A127830
:1058100091077EF588A98D4A127D042A7EF683A918
:1058200013F0ACFF059B1B6803F00403FEF77DB982
:10583000059B87491B680A6003F00403FEF775B9EE
:10584000844B002201208449844C0B60227005F0B7
:105850000DFC059B1B6803F00403FEF766B90021ED
:10586000BB2A109100F03D81B72A00F03681BE2A94
:1058700000F03181BD2A00F017819E2A00F0588186
:105880009D2A00F04E81AE2A00F04481AD2A00F03E
:105890003A81EF2A00F0B481FD2A00F0AB81FB2AA7
:1058A00000F0A281FE2A00F09981F72A00F084819D
:1058B0007B2A7EF436A94FF4FA61022006F0E6F85E
:1058C000FEF72FB9102005F001FC202005F0E6FBC3
:1058D0006349534C081F14F0BBFC624B02221A7040
:1058E00094F8F030002B00F029813788FEF798BE3D
:1058F0005D4B01220220A6E7CFB2584B0A915B789C
:10590000BB423FF439AADFF87481384606F098F9B3
:1059100098F802300A991BB1C9B20C2021F0E4FBBF
:105920000137FFB2CBE600273946E6E74F4B049933
:105930005B8991ED007A07EE903AF8EEE77AB0EEE7
:10594000C77AB4EEE77AF1EE10FA7FF5D5AE91EDB5
:10595000017AB0EEC77AF4EEC77AF1EE10FA7FF76B
:10596000CBAEBB063FF5CBAE2D4C202005F0AEFBF9
:105970002146D8F80420D8F8003041F8EC2F04F183
:10598000E800C4F8E83014F063FC364B01221A70CA
:10599000A6E7102005F082FB324B378883F8009091
:1059A0004FF00109A2E6202005F078FB2D4B1C4C9E
:1059B00000221A7094E72E4B1B78032B00F0C28054
:1059C0000346D0E62B4B022203203CE7059B2A4AE4
:1059D0001B684FF4C871118003F00403FEF7A5B8EB
:1059E0000AF050FEF5F7AEFE0AF034FE02F02CFB92
:1059F000012005F03BFB94F8A220FFF7FFB9002E31
:105A00003EF408A8064C94F8A130002B3EF434A8CC
:105A100005F0F8F9002384F8A130FEF72DB800BF97
:105A2000AC230020906B002000610020E453002094
:105A300098CD03084C230020A0230020A42300209D
:105A40001C6A0020586F00209C6E0020A06E002071
:105A5000405700203E5C0020305C00201C5C002091
:105A600058590020605900208C5C0020F459002017
:105A7000D8600020DA5C0020B69E00207E5D002009
:105A800094F8A820002A38D194F8AA3083F00103B2
:105A900084F8AA3043BB0C2005F0D0F9059B1B68A5
:105AA00003F00403FEF741B84FF6FE73574AD0895E
:105AB0009689014433449381D1810AF0E3FDF5F7DF
:105AC00041FE0AF0C7FD02F0BFFA012005F0CEFA50
:105AD000B4F8A42050E60223E8E70B464FF6FE7127
:105AE000E4E70B460221E1E70B2005F0A7F9059B4F
:105AF0001B6803F00403FEF718B884F8A80084F8C4
:105B0000A910FEF712B8FF21002022F027FD94F81B
:105B1000A220BEE60121002022F020FD94F8A22060
:105B2000B4E60021FF2022F019FD94F8A220AAE695
:105B3000012022F013FD94F8A220A1E64FF0010904
:105B4000FFF796BB05F05EF9B4F9A42014E6112026
:105B50000A9221F0C9FADAF8E4000A9ABFE40D20AB
:105B60000A9221F0C1FA0A9A5DE5294C12F0E4FD8F
:105B7000002384F8A130FDF77FBF0F200A9221F0A7
:105B8000B3FADAF8E4000A9A62E503230493FEF715
:105B900097BC0E2021F0A8FADAF8E400FFF7D9BB91
:105BA000002B3FF42FAF1B491B4A09684FF47A7052
:105BB00000FB0313136025E70021042005F066FFB6
:105BC000FDF7AFBF172021F08FFA2FE410200A92C3
:105BD00021F08AFADAF8E4000A9A95E40021032019
:105BE00005F054FFFDF79DBF0021022005F04EFF98
:105BF000FDF797BF0021012005F048FFFDF791BF99
:105C00000021084605F042FFFDF78BBFB465002078
:105C1000AC2300208C7900203C570020436A826925
:105C2000D154436A0169426B01338B4228BF002380
:105C30004362002A2FD0EFF31182502383F312889E
:105C4000436B1968C9072CD470B45E686EB9456A95
:105C5000816A8D4217D084690C44DC600ED9691AC0
:105C600059608562002180F85810196841F00101DF
:105C7000D2B2196082F3118870BC70470469611A4E
:105C800059608662EEE7012380F85830D2B282F381
:105C9000118870BC7047426DD36843F08003D360B5
:105CA0007047D2B282F31188704700BF026B10B404
:105CB00062B1836CC2684469D11A013B615C5DF8D2
:105CC000044B08BF13468364C8B27047016A436936
:105CD000C4685B5C0131A14228BF114601625DF8D6
:105CE000044BD8B2704700BF436B13B190F8580013
:105CF0007047836A406A181AB0FA80F0400970470A
:105D0000416A836A99420AD3CB1A416B026961B135
:105D10004968501E0B4483420AD2C01A7047026978
:105D20001144CB1A416B0029F2D1501EC01A7047A2
:105D300000207047036B43B1826C5B6893422FBFB6
:105D4000981AC0689B1AC0187047C269036A9A42C1
:105D50002FBFD01AC0688018C01A70470A4B30B5E0
:105D600003F10C0493F900205D78072AC8BF143AA8
:105D7000811804338D7213F8025C855413F8012CDA
:105D80000A75A342EED130BD28B4030803682DE99B
:105D9000F041DF691FB13B46BDE8F0411847002ADA
:105DA000164611DD04460D460E4400E023689B684C
:105DB000204698470028F9D0236815F8011B1B6876
:105DC00020469847AE42F1D1BDE8F08100231F2163
:105DD0002622017042708370C370704715230370D0
:105DE0001623C370172383713A2383703B234371B7
:105DF0003C230372704700BF30B4846814B1236839
:105E0000A5885D83436840F2E93001E0002832D084
:105E10001D89013815F0020F80B2F7D089B299813F
:105E200040F2E93101E0002947D01889013910F02A
:105E3000010F89B2F7D0998940F2E93100E059B3F6
:105E40001889013910F0020F89B2F8D092B29A8104
:105E500040F2E93201E0002A3FD01989013A11F0FD
:105E6000010F92B2F7D09B8914B12368A2881A83DC
:105E7000012030BC704721498B4204D0A1F5744108
:105E80008B42D9D102201E4901EB0010418901311A
:105E900089B241814189CFE7184A934204D0A2F5E3
:105EA00074429342E0D10221154B03EB01114B895F
:105EB00001339BB24B814B89D6E71048834203D014
:105EC00010498B42B8D102210D4800EB01114889DD
:105ED000013080B248814989AEE708498B4203D03E
:105EE000084A9342C0D10222054B03EB02125389A8
:105EF00001339BB253815389B6E700BF00300140A4
:105F0000286F0020003C004030B50446406D6171B0
:105F10008389A26823F400531B041B0C838185B082
:105F2000A379009213F0040230D04FF4805213F0A2
:105F30000203ADF8042056D1ADF806304FF480636B
:105F40000022ADF8083011F00103ADF80C2028D183
:105F5000ADF80A3008238D07694648BFADF80A300E
:105F600014F000FEA279636DD10724D412F0080F5B
:105F70009A8A1BD122F008021204120C9A829A8982
:105F800092B242F400529A8105B030BD13F0020380
:105F9000ADF8042024D04FF400551346ADF8065058
:105FA000CEE70423ADF80A300C23D4E792B242F0D6
:105FB00008029A82E3E70D498B420FD0A1F54841D0
:105FC0008B4209D00A498B42D0D105200121F6F736
:105FD000E7FCA279636DC9E70220F7E70020F5E747
:105FE000ADF80630ACE74FF40053A5E700100140D0
:105FF0000014014010B50446406DA160838923F46C
:1060000000531B041B0C8381A37984B013F004029A
:10601000009135D04FF4805213F00203ADF8042004
:1060200056D1ADF806304FF480636279ADF8083090
:10603000D1074FF00003ADF80A30ADF80C3045BF82
:106040000423ADF80A3008230C236946920748BFA1
:10605000ADF80A3014F086FDA279636DD1071FD424
:1060600012F0080F9A8A16D122F008021204120CBC
:106070009A829A8992B242F400529A8104B010BD79
:1060800013F00203ADF804201FD04FF40051134663
:10609000ADF80610C9E792B242F008029A82E8E72A
:1060A0000D498B420FD0A1F548418B4209D00B49D5
:1060B0008B42D5D105200121F6F772FCA279636DE0
:1060C000CEE70220F7E70020F5E7ADF80630ACE7B1
:1060D0004FF40053A5E700BF001001400014014039
:1060E00038B5254B9C68236B73B1636D626BCAB185
:1060F000998A1A88C90592B201D5D20700D438BD51
:106100004FF6F7721A8038BD636D99891A8889062F
:1061100092B2EBD59206E9D5E26ACAB1988880B20C
:106120009047E2E799891A880D0692B2E0D51006E9
:10613000DED5A26A616A8A4219D0A1692569885CA4
:1061400098800132B2FBF5F105FB1122A262CFE784
:106150009B88E2696169DBB28B54E269E068636D38
:106160000132B2FBF0F100FB1122E261BEE7DA6816
:1061700022F08002DA60BBE71433002038B5254BEB
:106180001C68236B73B1636D626BCAB1998A1A88FC
:10619000C90592B201D5D20700D438BD4FF6F772C7
:1061A0001A8038BD636D99891A88890692B2EBD539
:1061B0009206E9D5E26ACAB1988880B29047E2E7D0
:1061C00099891A880D0692B2E0D51006DED5A26A2A
:1061D000616A8A4219D0A1692569885C9880013278
:1061E000B2FBF5F105FB1122A262CFE79B88E269C1
:1061F0006169DBB28B54E269E068636D0132B2FB26
:10620000F0F100FB1122E261BEE7DA6822F08002C1
:10621000DA60BBE71433002070B4EFF3118650232B
:1062200083F31288436B1A68D20720D45D686DB976
:10623000446A826A944217D081691144D9600ED9A8
:10624000A21A5A608462002280F858201A6842F02C
:106250000102F1B21A6081F3118870BC70470169C4
:106260008A1A5A608562EEE7012380F85830F3B24B
:1062700083F3118870BC704703685B6A03B11847E9
:10628000704700BF03681B6A03B11847704700BF1F
:1062900003682DE9F041DF691FB13B46BDE8F041DD
:1062A0001847002A164611DD04460D460E4400E04C
:1062B00023689B68204698470028F9D0236815F882
:1062C000011B1B6820469847AE42F1D1BDE8F08122
:1062D00003689B69184700BF03685B69184700BFE4
:1062E00003681B69184700BF0368DB68184700BFD5
:1062F00003689B68184700BF03685B68184700BFC6
:1063000003681B68184700BF38B50C46097849B1C7
:10631000054601342B6828461B68984714F8011B72
:106320000029F7D138BD00BF064B53F820302BB100
:106330001A689B8851690B4201D1138370475383BC
:10634000704700BF5879002003682DE9F04F03F132
:106350003F4404F57E04604EA40A0125345D04F038
:106360001F066409032C05FA06F500F0AF80042C23
:1063700000F0A780022C54D08588B5FA85F0C0F1D2
:106380001F0080B2C40803EB840400F00700266AF3
:1063900080000F27874026EA07062662276A01F059
:1063A000030602FA00F0721E3843012AC1F3810C81
:1063B000C1F300182062C1F3411137D900242246ED
:1063C00001274FF0030E03E0102A04F1020426D047
:1063D00007FA02F0A84302F10102F5D1D3F800C098
:1063E0000EFA04F0C04300EA0C0CC3F800C0D3F866
:1063F000008006FA04FC4CEA080CC3F800C0D3F88D
:106400000CC000EA0C00D860D3F80CC001FA04F00C
:1064100040EA0C00102AD86004F10204D8D1BDE88B
:10642000F08F2E4C666C35436564A5E7002002466C
:106430004FF0010E4FF0030904E00132102A00F181
:1064400002003CD00EFA02F737EA0504F5D1D3F882
:1064500000A009FA00F4E4430AEA040AC3F800A021
:10646000D3F800B006FA00FA4AEA0B0AC3F800A013
:10647000D3F808A004EA0A0AC3F808A0D3F808B0C1
:106480000CFA00FA4AEA0B0AC3F808A0D3F804A0F1
:106490002AEA07075F60D3F804A008FA02F747EA80
:1064A0000A075F60DF683C40DC60DF6801FA00F4E7
:1064B00001323C43102ADC6000F10200C2D1BDE889
:1064C000F08F064C266B3543256355E7034C266C4D
:1064D0003543256450E700BFE4DA03080038024082
:1064E000026802F13F4303F57E032DE9F04F9B0A5A
:1064F000544DEB5C03F01F055B090124032B04FAE8
:1065000005F400F09980042B00F09180022B3ED01E
:1065100001F00306731E012BC1F3810CC1F30018B7
:106520008588C1F3411137D90024234601274FF054
:10653000030E03E0102B04F1020426D007FA03F047
:10654000A84303F10103F5D1D2F800C00EFA04F01C
:10655000C04300EA0C0CC2F800C0D2F8008006FA72
:1065600004FC4CEA080CC2F800C0D2F80CC000EAE7
:106570000C00D060D2F80CC001FA04F040EA0C0024
:10658000102BD06004F10204D8D1BDE8F08F2E4B5F
:106590005D6C2C435C64BBE7002003464FF0010EAA
:1065A0004FF0030904E00133102B00F102003CD04E
:1065B0000EFA03F737EA0504F5D1D2F800A009FA7C
:1065C00000F4E4430AEA040AC2F800A0D2F800B0DA
:1065D00006FA00FA4AEA0B0AC2F800A0D2F808A0AC
:1065E00004EA0A0AC2F808A0D2F808B00CFA00FAC5
:1065F0004AEA0B0AC2F808A0D2F804A02AEA070760
:106600005760D2F804A008FA03F747EA0A07576070
:10661000D7683C40D460D76801FA00F401333C43AA
:10662000102BD46000F10200C2D1BDE8F08F064B00
:106630001D6B2C431C636BE7034B1D6C2C431C64CC
:1066400066E700BFE4DA03080038024010B5040929
:10665000013C032C17D80D4B33F8142000F00F0029
:1066600042FA00F313F001030DD0012303FA00F006
:106670000138104021F05EFD054A064B125D1044C2
:1066800003EBC00010BD002010BD00BFE8D203081E
:10669000E4D20308407700202DE9F04F4A484B49E7
:1066A0004B4B4C4C4FF0010A4FF002094FF00408DD
:1066B0004FF0080C4FF0100E20274026802530F8B0
:1066C000022B12F0010F03D01960A3F804A00833C5
:1066D00012F0020F03D01960A3F80490083312F0EF
:1066E000040F03D01960A3F80480083312F0080FD8
:1066F00003D01960A3F804C0083312F0100F03D0C0
:106700001960A3F804E0083312F0200F02D01960DA
:106710009F80083312F0400F02D019609E8008332A
:1067200012F0800F02D019609D80083312F4807F30
:1067300005D04FF4807B1960A3F804B0083312F43D
:10674000007F05D04FF4007B1960A3F804B0083334
:1067500012F4806F05D04FF4806B1960A3F804B079
:10676000083312F4006F05D04FF4006B1960A3F8E2
:1067700004B0083312F4805F05D04FF4805B1960D9
:10678000A3F804B0083312F4005F05D04FF4005BA7
:106790001960A3F804B0083312F4804F05D04FF409
:1067A000804B1960A3F804B00833D20B04D04FF427
:1067B000004219609A80083301F58061A1427FF49C
:1067C0007EAFBDE8F08F00BFE8D2030800000240B2
:1067D000407700200010024000286AD003682DE9AD
:1067E000F04F03F13F4404F57E045F4EA40A0125F7
:1067F000345D04F01F066409032C05FA06F559D030
:10680000042C00F0AC80022C59D08588B5FA85F0B4
:10681000C0F11F0080B2C40803EB840400F007003D
:10682000266A80000F27874026EA07062662276A25
:1068300001F003068240701E3A430128C1F3810C27
:10684000C1F300182262C1F341113DD90024224650
:1068500001274FF0030E03E0102A04F1020426D0B2
:1068600007FA02F0A84302F10102F5D1D3F800C003
:106870000EFA04F0C04300EA0C0CC3F800C0D3F8D1
:10688000008006FA04FC4CEA080CC3F800C0D3F8F8
:106890000CC000EA0C00D860D3F80CC001FA04F078
:1068A00040EA0C00102AD86004F10204D8D1BDE8F7
:1068B000F08F70472D4C266C35432564A5E72B4C93
:1068C000666C35436564A0E7002002464FF0010E78
:1068D0004FF0030904E00132102A00F102003CD01D
:1068E0000EFA02F737EA0504F5D1D3F800A009FA49
:1068F00000F4E4430AEA040AC3F800A0D3F800B0A5
:1069000006FA00FA4AEA0B0AC3F800A0D3F808A076
:1069100004EA0A0AC3F808A0D3F808B00CFA00FA8F
:106920004AEA0B0AC3F808A0D3F804A02AEA07072A
:106930005F60D3F804A008FA02F747EA0A075F602D
:10694000DF683C40DC60DF6801FA00F401323C4360
:10695000102ADC6000F10200C2D1BDE8F08F034CC8
:10696000266B3543256350E7E4DA0308003802401C
:10697000002855D0026802F13F4303F57E032DE95C
:10698000F04F9B0A544DEB5C03F01F055B0901249B
:10699000032B04FA05F444D0042B00F09780022B5B
:1069A00044D001F00306731E012BC1F3810CC1F327
:1069B00000188588C1F341113DD9002423460127E1
:1069C0004FF0030E03E0102B04F1020426D007FA67
:1069D00003F0A84303F10103F5D1D2F800C00EFA89
:1069E00004F0C04300EA0C0CC2F800C0D2F80080EA
:1069F00006FA04FC4CEA080CC2F800C0D2F80CC03D
:106A000000EA0C00D060D2F80CC001FA04F040EAB1
:106A10000C00102BD06004F10204D8D1BDE8F08F37
:106A200070472E4B1D6C2C431C64BAE72B4B5D6CDE
:106A30002C435C64B5E7002003464FF0010E4FF095
:106A4000030904E00133102B00F102003CD00EFAE0
:106A500003F737EA0504F5D1D2F800A009FA00F4EB
:106A6000E4430AEA040AC2F800A0D2F800B006FA29
:106A700000FA4AEA0B0AC2F800A0D2F808A004EA19
:106A80000A0AC2F808A0D2F808B00CFA00FA4AEADA
:106A90000B0AC2F808A0D2F804A02AEA0707576038
:106AA000D2F804A008FA03F747EA0A075760D76844
:106AB0003C40D460D76801FA00F401333C43102B0A
:106AC000D46000F10200C2D1BDE8F08F034B1D6B12
:106AD0002C431C6365E700BFE4DA0308003802407A
:106AE00010B1036882885A83704700BF10B10368F1
:106AF00082881A83704700BF18B10368828809B979
:106B00005A8370471A83704710B40A4B0A4A1C789C
:106B100001238340234052F8200029B9B3FA83F1BE
:106B200049095DF8044BE7E7191C18BF01215DF81E
:106B3000044BE1E7567900205879002030B1036812
:106B400082881B691A4214BF01200020704700BFD1
:106B50002DE9F0410B4E346873691C400FD0DFF80B
:106B600028800127B4FA84F3C3F11F0307FA03F561
:106B700058F8230003689847AC437561F2D1BDE82B
:106B8000F08100BF003C0140C87800202DE9F041B1
:106B90000B4E346873691C400FD0DFF82880012742
:106BA000B4FA84F3C3F11F0307FA03F558F823007E
:106BB00003689847AC437561F2D1BDE8F08100BF2E
:106BC000003C0140C87800202DE9F0410B4E3468AC
:106BD00073691C400FD0DFF828800127B4FA84F3D2
:106BE000C3F11F0307FA03F558F823000368984719
:106BF000AC437561F2D1BDE8F08100BF003C0140BB
:106C0000C87800202DE9F0410B4E346873691C40B0
:106C10000FD0DFF828800127B4FA84F3C3F11F03F3
:106C200007FA03F558F8230003689847AC437561E9
:106C3000F2D1BDE8F08100BF003C0140C8780020DF
:106C40002DE9F0410B4E346873691C400FD0DFF81A
:106C500028800127B4FA84F3C3F11F0307FA03F570
:106C600058F8230003689847AC437561F2D1BDE83A
:106C7000F08100BF003C0140C87800202DE9F041C0
:106C80000B4E346873691C400FD0DFF82880012751
:106C9000B4FA84F3C3F11F0307FA03F558F823008D
:106CA00003689847AC437561F2D1BDE8F08100BF3D
:106CB000003C0140C87800202DE9F0410B4E3468BB
:106CC00073691C400FD0DFF828800127B4FA84F3E1
:106CD000C3F11F0307FA03F558F823000368984728
:106CE000AC437561F2D1BDE8F08100BF003C0140CA
:106CF000C8780020084A094808B5536C43F480431B
:106D000053640021402223F008FF054B4FF0FF326F
:106D10001A60C3F8032008BD00380240C87800207C
:106D20000879002003685B6A184700BF2DE9F0412D
:106D3000044618460D461646984620F051FD276831
:106D4000E6722844A07229467D69434632462046B1
:106D5000AC46BDE8F0416047036810B504461B68C7
:106D60009847236820469B689847A37B0133A37309
:106D700010BD00BF10B5036804469B689847FF2309
:106D800001226373227310BD08B5FFF75FFC38B1B1
:106D90002C2282710022C2712021BDE80840E7E563
:106DA00008BD00BF40F2E93300E0A3B10289013B16
:106DB00012F0020F9BB2F8D089B2818140F2E93320
:106DC00000E043B10289013B12F0010F9BB2F8D001
:106DD0008089C0B27047094A904205D0084B98425A
:106DE00001D0FF2070470223064A02EB03135A89A1
:106DF000013292B25A815889C0B2704700300140C6
:106E0000003C0040286F0020144B984224D003F52A
:106E10008063984220D0028822F040021204120CB3
:106E20000280028822F038031B041B0C59B141F484
:106E30008071002991FAA1F2B2FA82F108BF4FF0F5
:106E4000FF310139C9000B439BB2038003889BB219
:106E500043F04003038070474908DCE700380040F6
:106E6000F0B484894FF6FF764FF47A7443B3002967
:106E700038D00F78013101E0B4421AD00589013CC5
:106E800015F00205A4B2F7D0BCB284814FF47A7435
:106E900002E0BCB2B4420CD0058915F0010504F142
:106EA000FF37F6D08589ADB20AB115700132013BCA
:106EB000DCE70D4B984207D0A3F57443984202D00B
:106EC0000120F0BC70470225084B03EB05156B89C8
:106ED00001339BB26B81688980B2003018BF0120FA
:106EE000F0BC7047FF27C9E700300140286F002041
:106EF00070B50546806810B104688088608341F0F1
:106F00008001686840F2E93400E0E4B10689013CA0
:106F100016F0020FA4B2F8D089B2818140F2E931B3
:106F200000E009B30489013914F0010F89B2F8D0E7
:106F300081890021FFF794FFAB6813B11A689B8821
:106F40001383012070BD1049884204D0A1F574411B
:106F50008842EED102240D4901EB0414618901310C
:106F600089B261816189E4E7074CA04203D00849F6
:106F70008842DED10221054C04EB01114C89013419
:106F8000A4B24C814989D4E700300140286F002029
:106F9000003C004038B50B4C23688BB15A68821A0C
:106FA000002A054604DA0CE05A68AA1A002A07DB10
:106FB0009A68226018461A6890472368002BF3D11C
:106FC00038BD38BD943600200D4B042100228907BE
:106FD00010B4027203F1600402D5197981540132B0
:106FE0009C4203F1180308D0072A06DC9979890727
:106FF000F3D49C4203F11803F6D15DF8044B7047BB
:107000006CD2030810B4104C0423214613F0010382
:107010004FF0000201F1180108D10132052A0ED00B
:107020008B7913F0010301F11801F6D002EB420253
:1070300004EBC2025DF8044B1379037070470370D0
:107040005DF8044B704700BF6CD203080122322365
:1070500002704370704700BF232203230270437005
:10706000704700BF08B50FF0DDFCF5F78FFC00BFDF
:10707000024A034B127819780DF0DEBC88210020FB
:1070800089210020038A2DE9F0478589ADB21D4092
:1070900029D00F4606464FF000484FF00009B5FAD8
:1070A00085F328FA03F2D24391B21B3B154031829B
:1070B000042B16D8DFE803F03129211903007B6A7D
:1070C000002B32D003F1FF3A1FFA8AFAC7F8249056
:1070D0003C6A34B123682046514698476468002CC6
:1070E000F8D1002DDBD1BDE8F0873868716B0368FB
:1070F00089B29847002DD2D1F5E77868B16B036863
:1071000089B29847002DCAD1EDE7B868F16B0368E2
:1071100089B29847002DC2D1E5E7F868316C036861
:1071200089B29847002DBAD1DDE7F36A1FFA83FAD6
:10713000CEE700BF08B501210220FFF7E5FC094BAF
:107140001B7803F00503052B08D000210120FFF771
:10715000DBFC00210846FFF7D7FCFEE70FF0F4FC4C
:10716000F3E700BF10330020022828BF022010B42C
:10717000084C094B207000EB8002C0EBC2020749AB
:107180005DF8044B013003EB4203C0B20B6003F027
:107190006DBF00BF1C5C00203E5C0020305C002006
:1071A00008B509F06FFAF4F7CDFABDE8084009F028
:1071B00051BA00BF38B5484B5A899989914224BFCA
:1071C00000225A81198ADA89914224BF0022DA8189
:1071D000DA78CAB1072A41496AD091F85700404D80
:1071E000012400210A282C709C70D9715DD00C28D4
:1071F00007D0002A6CD0DFED3B7A072A0ED00A2890
:1072000062D0DFED397A09E0344A92F857000A2853
:1072100056D00C285BD1D979DFED347A344C9FED10
:10722000350AA278002918BFF0EE407A062A04D861
:10723000314901EB820191ED000A217979B1013ADE
:10724000032A0BD8F7EE007A87EE800A21F05AFB6A
:107250002388984228BF1846208038BD38BD9B78C7
:107260001F4A07EE103A1178B8EEC77A67EE277A10
:1072700007EE101AB8EEC77A27EE277AB4EEC70ADF
:10728000F1EE10FAEADD80EE277AFDEEC77A17EE0E
:10729000903A102BA8BF1023012BB8BF0123DBB2FB
:1072A0008B4238BF0B46137038BDDFED147AA4E76C
:1072B00091F857000A2803D00C28ACD0D9799AE766
:1072C000D979DFED0E7AA9E7DFED0D7AA6E7D97956
:1072D000DFED047AA2E700BF086A0020586F0020A3
:1072E000A86500206F1203396F12833A0AD7A339B9
:1072F000D86600206F12033834B403085304E93809
:107300000F506E3A38B50D4C0D4DAC4206D2616847
:1073100020461434F4F7A2F9AC42F8D3094B0A4CD6
:107320000A4A0B4D1D6000230A49A3711370537064
:1073300009480860BDE8384012F0FCB88801000830
:10734000D4050008305C0020D85B00201C5C0020C5
:107350003E5C0020989E0020465D002008B5FFF7A7
:10736000D1FF09F08FF9F4F7EDF9BDE8084009F015
:1073700071B900BFF0B50C2934D8DFE801F08933CA
:1073800033335E333333343333330700048C96891D
:10739000B2F802E01788734D24F480542404240CBE
:1073A0000484038C8488818B23F4005321F4E64108
:1073B0001B0409041B0C46EA0E06090C43EA0633BB
:1073C00041EA0721A8429BB2A4B289B200F09E8094
:1073D00005F58065A84200F09980926884808183D9
:1073E00002640384F0BD048C9589B2F802C0B2F83F
:1073F00000E05C4F24F480742404240C0484038C87
:107400008688818B23F400731B0421F073011B0C0D
:1074100045EA0C04090443EA0423090CB8429BB270
:10742000B6B241EA0E015CD04F4CA04259D09268EE
:1074300086808183C2630384F0BD048C9589B2F891
:1074400002C0B2F800E0474E24F010042404240CDB
:107450000484038C8788018B23F0200321F4E64108
:107460001B0409041B0C45EA0C04090C43EA041331
:1074700041EA0E21B0429BB2BFB289B25DD03A4C14
:10748000A0425AD092688780018382630384F0BD52
:10749000048C9789B2F802E01688324D24F001047A
:1074A0002404240C0484038C8488018B23F00203BD
:1074B0001B0421F073011B0C47EA0E0709043B4330
:1074C000090CA8429BB2A4B241EA060125D005F5F9
:1074D0008065A84221D0926884800183426303843E
:1074E000F0BDD589148A578A23F4006343EA052541
:1074F0004FF6FF332B40958826F440563C4343EA31
:10750000052346EA04169BB2B6B290E7158A24F426
:10751000804444EA8514A4B25FE7D689158A578A65
:1075200023F00803334324F4407496883D4323F04A
:1075300004032C433343A4B2CDE7D489158A568A79
:1075400023F0800343EA04134FF6BF741C40938872
:1075500027F44067354344EA031347EA85079BB2A3
:10756000BFB28FE700000140000401402DE9F04F59
:107570007822002183B0C248C24CDFF82493C24D68
:10758000C24EC34FDFF81C8323F0C7FAC148C2497B
:10759000DFF814E3DFF814C30022A358834200F09D
:1075A000D481B3F1804F00F0D281AB4200F0D181A1
:1075B000B34200F0D081BB4200F0CF81734500F0B0
:1075C000CE81634500F0CD81434500F0CC81DFF8EA
:1075D000E0A2534500F0C9810AF5806A534500F0E6
:1075E000C6810AF5806A534500F0C381AAF5983A2E
:1075F000534500F0C0810AF5806A534500F083814D
:107600000AF5806A534508BF0D2300F07D811832CA
:10761000782AC2D11320FFF719F8002840D001685A
:107620009E4C01F13F4303F57E039A0A0123A25CBD
:1076300002F01F045209032A03FA04F300F09D81AB
:10764000042A00F0B881022A03D1934A546C2343E0
:10765000536483880093B3FA83F3C3F11F039BB28F
:10766000DA0801EB820203F00703106A9B000F2483
